:100000000C946A100C948B100C948B100C948B1025
:100010000C948B100C948B100C948B100C948B10F4
:100020000C948B100C948B100C9497600C948B1088
:100030000C948B100C948B100C948B100C948B10D4
:100040000C948B100C948B100C948B100C948B10C4
:100050000C948B100C948B100C948B100C948B10B4
:100060000C948B100C949B570C948B100C94DC59B3
:100070000C948B100C948B100C948B100C948B1094
:100080000C948B100C948B100C948B100C948B1084
:100090000C948B100C948B100C948B100C948B1074
:1000A0000C948B100C948B100C948B100C948B1064
:1000B0000C948B100C948B100C948B100C948B1054
:1000C0000C948B100C948B100C948B100C948B1044
:1000D0000C948B100C948B100C948B100C948B1034
:1000E0000C948B100C948B100C94EB570C948B107D
:1000F0000C942C5A0C948B100C948B100C948B1029
:100100000C948B100C948B100C948B100C948B1003
:100110000C948B100C948B100C948B100C948B10F3
:100120000C948B100C948B100C948B100C948B10E3
:100130000C948B100C948B100C948B100C948B10D3
:100140000C948B100C948B100C948B100C948B10C3
:100150000C948B100C948B100C948B100C948B10B3
:100160000C94C3570C948B100C94045A0C948B1061
:100170000C948B100C948B100C948B100C948B1093
:100180000C948B100C948B100C948B100C948B1083
:100190000C948B100C948B100C948B100C948B1073
:1001A0000C94463F0C948B100C948B100C948B1079
:1001B0000C948B100C948B100C948B100C948B1053
:1001C0000C948B100C948B100C948B100C948B1043
:1001D0000C948B100C948B100C948B100C94135863
:1001E0000C948B100C94545A000000000100661B04
:1001F000010205000100020000000000161C291C7D
:10020000341C401C4C1C5B1C8F1C971CAF1CBD1C61
:10021000111E151E191E1D1E941E941E941E941E42
:10022000941E941E941E941E941E941E941E211EB1
:10023000241E941E941E941E941E941E941E941E9E
:10024000941E941E941E941E941E941E941E271E8B
:100250002B1E941E941E941E941E941E941E941E77
:10026000941E941E941E941E941E941E941E2F1E63
:100270003F1E431E461E491E961E961E961E961E25
:10028000961E961E961E961E961E961E961E961ECE
:100290004C1E4F1E521E551E961E961E961E961ED4
:1002A000961E961E961E961E961E961E961E581EEC
:1002B000731E761E9A1E9A1E9A1E9A1E9A1E9A1EC9
:1002C0009A1E9A1E9A1E9A1E9A1E9A1E9A1E791E8F
:1002D0007D1E811E851E9A1E9A1E9A1E9A1E9A1EA9
:1002E0009A1E9A1E9A1E9A1E9A1E9A1E9A1E891E5F
:1002F0009A1E9A1E9A1E9A1E9A1E9A1E9A1E9A1E3E
:100300009A1E9A1E9A1E9A1E9A1E9A1E9A1E8C1E3B
:100310009A1E9A1E9A1E9A1E9A1E9A1E9A1E9A1E1D
:100320009A1E9A1E9A1E9A1E9A1E9A1E9A1E8F1E18
:10033000F41FD61FDB1FE01FE51FEA1FEF1FC82AAF
:10034000D32ADF2A242BE82B142C432C4D2C7F3965
:10035000E7390B3A3A3A483A5B3A6C3A8B3AC13D44
:10036000F13D063E173E283E553E723E673E7F3EBB
:100370002A426142A242F6428E43C7432C4469445A
:10038000FE4403451245214530453F4550456B45E8
:100390008645A145BC45D745F545174630463F46FD
:1003A0004E465C466E46BF4AED4A294BB84BED4B74
:1003B000434C764CA74CEB4C464D5C4D694D7F4D04
:1003C000904DA54D014E0E4E1A4E7252625264521D
:1003D000665268526A526C526E5270528E52B452C9
:1003E000C952A1523953DE52F5520C532353F65BD6
:1003F0002C5C9E5C125DAD5DB25ED55EEE5E496EBC
:1004000076616C696420435243206465746563744B
:100410006564206F6E20726563656976656420701F
:1004200061636B65740D0A000D0A52657365742073
:100430005265706F7274696E6720496E64657820CA
:10044000436F6D6D616E64205265636569766564A6
:10045000210D0A0D0A00496E76616C696420436FB4
:100460006E66696775726174696F6E21210D0A008D
:10047000436F6E66696775726174696F6E2055703F
:1004800064617465640D0A00496E76616C6964206C
:10049000436F6E66696775726174696F6E2C206E4A
:1004A0006F2075706461746520636F6D706C657426
:1004B000656421210D0A00436F6E6669677572617C
:1004C00074696F6E20557064617465640D0A00492B
:1004D00072696469756D204D65737361676520533A
:1004E000656E64204661696C6564210D0A0049727D
:1004F000696469756D204D65737361676520536527
:100500006E74210D0A004972696469756D20476532
:1005100074204D657373616765202D20496E636F8C
:100520006D696E6720436F6D6D616E6420506172FE
:10053000736564210D0A000D0A000D0A5472616E84
:10054000736D697373696F6E204F7074696F6E732A
:100550003A20000D0A537572666163696E67205315
:10056000657474696E673A20000D0A4E756D2046F9
:100570006978657320506572204D61696C626F788F
:1005800020436865636B3A20000D0A4E756D204666
:10059000697865732050657220586D69743A20003F
:1005A00046697820496E74657276616C3A20000D58
:1005B0000A0D0A002E002E000D0A4669726D776141
:1005C00072653A20000D0A53657269616C204E75A0
:1005D0006D6265723A200029002028000D0A000D86
:1005E0000A0D0A0020736563200030005454463A17
:1005F0002000206D2C20003000454850453A200056
:100600002C200030003030003030300030303030BE
:10061000003030303030003030303030300030306A
:100620003030303030002E0020002030002B002DE4
:10063000002C2000300030300030303000303030BE
:10064000300030303030300030303030303000303A
:10065000303030303030002E0020002030002B00B1
:100660002D002C20003000303000303030002E00C3
:1006700030003030003A0030003030003A003000B6
:1006800030300020002F0030003030002F003000CC
:10069000303000556E6B6E776E2C20004E6F20460A
:1006A00069782C200033442C202020202000324464
:1006B0002C202020202000345356204B462C200094
:1006C000335356204B462C2000325356204B462C99
:1006D0002000315356204B462C200056616C696433
:1006E0002C20004E6F5369672C20005265636F7297
:1006F00064205772697474656E20746F204C6F6744
:10070000210D0A005472616E736D697373696F6EA7
:10071000204572726F722121210D0A005472616EA0
:10072000736D697373696F6E20436F6D706C657460
:1007300065210D0A00446F776E6C6F61642045720D
:10074000726F722121210D0A00446F776E6C6F6108
:100750006420436F6D706C657465210D0A00446FF1
:10076000776E6C6F61642054696D656F7574205489
:1007700072616E736D697474696E67205061636B2A
:1007800065742121210D0A00436C656172204D655D
:100790006D6F7279205374617465204572726F7247
:1007A0002121210D0A004F7574676F696E67204D16
:1007B00065737361676520616464656420746F208C
:1007C0004F7574626F780D0A000D0A002C005254A8
:1007D00043205265676973746572733A20005254FE
:1007E0004320557064617465640D0A005254435F80
:1007F000434C4B4F55542044697361626C65640DE2
:100800000A00416C61726D20496E74657272757078
:100810007420456E61626C65640D0A00416C617202
:100820006D2053657420746F204D61782076616C63
:100830007565206F66203220646179730D0A00446B
:1008400061792C20486F75722C2026204D696E75B9
:10085000746520416C61726D205365740D0A004807
:100860006F75722026204D696E75746520416C612C
:10087000726D205365740D0A004D696E75746520A4
:10088000416C61726D205365740D0A00426C756590
:10089000746F6F74682044697361626C6564210DC4
:1008A0000A00426C7565746F6F7468204E616D65E7
:1008B00020536574210D0A00426C7565746F6F7466
:1008C0006820456E61626C6564210D0A000000219C
:1008D00010422063308440A550C660E7700881292B
:1008E000914AA16BB18CC1ADD1CEE1EFF1311210C3
:1008F0000273325222B5529442F772D6623993187B
:10090000837BB35AA3BDD39CC3FFF3DEE3622443CE
:100910003420040114E664C774A44485546AA54BCA
:10092000B528850995EEE5CFF5ACC58DD553367262
:100930002611163006D776F6669556B4465BB77A1A
:10094000A719973887DFF7FEE79DD7BCC7C448E5EE
:10095000588668A7784008611802282338CCC9ED6A
:10096000D98EE9AFF9488969990AA92BB9F55AD402
:100970004AB77A966A711A500A333A122AFDDBDCBA
:10098000CBBFFB9EEB799B588B3BBB1AABA66C870E
:100990007CE44CC55C222C033C600C411CAEED8F0A
:1009A000FDECCDCDDD2AAD0BBD688D499D977EB6A2
:1009B0006ED55EF44E133E322E511E700E9FFFBE5A
:1009C000EFDDDFFCCF1BBF3AAF599F788F8891A92D
:1009D00081CAB1EBA10CD12DC14EF16FE18010A104
:1009E00000C230E3200450254046706760B9839808
:1009F00093FBA3DAB33DC31CD37FE35EF3B1029054
:100A000012F322D2323542145277625672EAB5CBD3
:100A1000A5A89589856EF54FE52CD50DC5E234C3A3
:100A200024A01481046674476424540544DBA7FAA7
:100A3000B79987B8975FE77EF71DC73CD7D326F2F3
:100A4000369106B01657667676154634564CD96DF3
:100A5000C90EF92FE9C899E9898AB9ABA944586543
:100A60004806782768C018E1088238A3287DCB5C47
:100A7000DB3FEB1EFBF98BD89BBBAB9ABB754A5493
:100A80005A376A167AF10AD01AB32A923A2EFD0F13
:100A9000ED6CDD4DCDAABD8BADE89DC98D267C07E3
:100AA0006C645C454CA23C832CE01CC10C1FEF3EE7
:100AB000FF5DCF7CDF9BAFBABFD98FF89F176E3633
:100AC0007E554E745E932EB23ED10EF01E466C6182
:100AD0007368206D656D6F72793A204944207265A4
:100AE0006164204641494C4544210D0A00466C6131
:100AF0007368206D656D6F72793A20494420726584
:100B000061642053554343455353210D0A00475018
:100B10005320416E74656E6E612053656C6563741D
:100B200065642E2E2E2E2E2E2E200D0A004972695F
:100B30006469756D20416E74656E6E612053656CDD
:100B400065637465642E2E2E2E2E2E200D0A00B0A5
:100B5000B300A0A2000D0A002A0024004750532031
:100B60005365747570204552524F52210D0A004151
:100B70007474656D7074696E6720475053204261CC
:100B800075643A20343830300D0A00417474656D54
:100B90007074696E672047505320426175643A2033
:100BA000323430300D0A00417474656D7074696EB2
:100BB000672047505320426175643A2035373630FC
:100BC000300D0A00417474656D7074696E6720475A
:100BD000505320426175643A2031393230300D0A69
:100BE00000417474656D7074696E672047505320BE
:100BF000426175643A20393630300D0A0053656E13
:100C000064696E67204F535020496E697469616C46
:100C1000697A6174696F6E20636F6D6D616E642EA9
:100C20002E2E0D0A0053656E64696E6720636F6D2A
:100C30006D616E6420746F206368616E6765204724
:100C400050532050726F746F636F6C20746F204F1D
:100C500053502E2E2E0D0A004750532053657475A5
:100C6000702054696D656F75743A20417474656DB8
:100C70007074696E67206E6577206261756420729A
:100C80006174652E2E2E0D0A004750532050726F4E
:100C9000746F636F6C2044657465637465643A2097
:100CA0004F53500D0A004750532050726F746F63BA
:100CB0006F6C2044657465637465643A204E4D45DD
:100CC000410D0A004750532053687574646F776E66
:100CD00020436F6D706C657465210D0A0047505399
:100CE00020506F7765722052656D6F7665640D0ACE
:100CF0000053656E64204750532053687574646FC9
:100D0000776E20436F6D6D616E640D0A004750531E
:100D100020536F6674776172652056657273696FD0
:100D20006E20496E666F726D6174696F6E205265D8
:100D30006365697665640D0A00207365636F6E6490
:100D400073005454463A20004750532054696D654F
:100D50006F75740D0A00475053204552524F52216F
:100D60002121212121212121212121212121202075
:100D7000200D0A0047505320436F6E6669677572F5
:100D80006174696F6E20436F6D706C657465210DC1
:100D90000A0047505320454550524F4D205570642E
:100DA00061746520436F6D706C657465210D0A0078
:100DB00047505320537769746368696E6720667281
:100DC0006F6D2048796265726E61746520746F2062
:100DD0004163746976652E2E2E0D0A004E6F2070C9
:100DE00061636B6574732072656365697665642001
:100DF00066726F6D20475053207265636569766532
:100E000072206C6174656C792C20726573746172E8
:100E100074696E672E2E2E0D0A00475053204550E0
:100E200050524F4D20557064617465205265717544
:100E300065737465642E2E2E0D0A00436F6E66690D
:100E4000677572696E67204750532E2E2E0D0A006B
:100E5000475053205475726E696E67204F6E2E2E68
:100E60002E0D0A0047505320416E74656E6E61204E
:100E700053656C6563746564202D2054696D656FDE
:100E8000757420666F72204972696469756D2055AA
:100E90007365200D0A00A0A2000038A0A2005B2903
:100EA000A0A2000212A0A200020CA0A200020BA0AD
:100EB000A2000909A0A2000006A0A200BC04A0A2F2
:100EC000002902505352463135302C0047504753C9
:100ED000562C0047504753412C0047504747412C60
:100EE000004750524D432C00505352463130302C65
:100EF000302C31393230302C382C312C300000027B
:100F0000CD10000284000008A600040100000000CB
:100F10000008A6002901000000000008A602000049
:100F20000000000000198000000000000000000028
:100F3000000000000000000000000000000C005352
:100F40005049204572726F723A2054696D656F7511
:100F500074206F6E205374726F62652042756666EE
:100F600065720D0A00535049204572726F723A2023
:100F700054696D656F7574206F6E205374726F6263
:100F80006520427974650D0A004D616E6167656D7B
:100F9000656E742054696D65205265636569766578
:100FA000640D0A004D616E6167656D656E74205455
:100FB000696D6520636F756C64206E6F7420626567
:100FC0002064657465726D696E65640D0A004D611B
:100FD0006E6167656D656E742054696D6520697317
:100FE0002056616C69640D0A004D54202D204D651A
:100FF0007373616765205472616E736665726564B0
:10100000205375636365737366756C6C79206672C3
:101010006F6D204761746577617920746F204D6F23
:1010200064656D2E2E2E2E2E20200D0A0053656E27
:1010300064204D657373616765205472616E7366D9
:101040006572204661696C65642E2E2E2E2E20203E
:101050000D0A004D4F202D204D657373616765208B
:101060005472616E73666572204661696C656420B6
:1010700064756520746F2074726166666963206DA3
:10108000616E6167656D656E74207468696E6779FD
:10109000212E2E2E2E2E20200D0A004D65737361F9
:1010A00067657320617265205175657565642E2EC4
:1010B0002E20200D0A005570646174652053746100
:1010C000747573202D2055706461746520457272AB
:1010D0006F720D0A005570646174652053746174F9
:1010E0007573202D2055706461746520436F6D7099
:1010F0006C6574650D0A00557064617465205374E5
:1011000061747573202D2052657175657374204E5E
:101110006574776F726B2054696D650D0A005570A8
:101120006461746520537461747573202D20526559
:10113000717565737420534244535820537461741D
:1011400075730D0A00557064617465205374617481
:101150007573202D205265676973746572696E67B7
:10116000206F6E204E6574776F726B0D0A0055709C
:101170006461746520537461747573202D20526509
:101180007175657374205369676E616C2053747256
:10119000656E6774680D0A00204972696469756D2F
:1011A000202D205573652050726F66696C65203064
:1011B000204F6E2052657365740D0A00526574727B
:1011C000792074696D657220657870697265642E26
:1011D0002E2E0D0A004E6F204E6574776F726B20B5
:1011E000417661696C61626C65202D2043616E27D8
:1011F0007420676574206D65737361676520617421
:1012000020746869732074696D6521200D0A00528D
:10121000657472792074696D656F7574202D207204
:101220006573656E6420636C6561725F6D65737371
:101230006167655F627566665F4D542E2E2E0D0ADE
:101240000042756666657220636C65617265642034
:101250007375636365737366756C6C792E2E2E0DD2
:101260000A0052657472792074696D656F75742017
:101270002D20726573656E6420636C6561725F6DAD
:101280006573736167655F627566665F4D542E2E88
:101290002E0D0A0057652077657265206E6F7420E9
:1012A00061626C6520746F206765742074686520C6
:1012B000726561645F62696E6172795F64617461B5
:1012C0005F726573706F6E7365202D205265747246
:1012D000792074696D657220657870697265642E15
:1012E0002E2E0D0A004D5347207265616420616EF9
:1012F0006420636865636B73756D206572726F72CD
:101300002E2E2E0D0A004D53472072656164206118
:101310006E642070617273656420737563636573B6
:101320007366756C6C792E2E2E0D0A0052657472E0
:10133000792074696D656F7574202D2072657365F1
:101340006E6420636C6561725F6D65737361676560
:101350005F627566665F4D542E2E2E0D0A00526533
:101360007472792074696D65722065787069726530
:10137000642E2E2E0D0A004C6574732077616974FB
:1013800020612062697420746F207365652069662E
:1013900020776520676574204E6574776F726B20C7
:1013A000536572766963652E2E2E0D0A00476574AB
:1013B000206D657373616765205342444958206608
:1013C00061696C2E2E2E0D0A00476574206D6573C1
:1013D00073616765205342444958207375636365A0
:1013E00073732E2E2E0D0A00526574727920746963
:1013F0006D657220657870697265642E2E2E0D0AF7
:10140000004C65747320776169742061206269748F
:1014100020746F2073656520696620776520676595
:1014200074204E6574776F726B20536572766963B2
:10143000652E2E2E0D0A0053656E642041542B53E9
:10144000424449582E2E2E0D0A004D657373616774
:101450006520616C7265616479206F627461696E88
:101460006564202D20676F20746F2050617273694E
:101470006E672E2E2E0D0A004972696469756D2003
:1014800053656E64204D65737361676520457272A4
:101490006F7220537461746520526561636865647E
:1014A000210D0A0052657472792074696D6572208D
:1014B000657870697265642C20636C6561722020A8
:1014C0004D4F2062756666657220636F6D6D616E4B
:1014D000642E2E2E0D0A004E6F204E6574776F72AB
:1014E0006B20417661696C61626C65202D204361DF
:1014F0006E27742073656E64206D65737361676514
:1015000020617420746869732074696D6521200DF1
:101510000A0052657472792074696D65722065786D
:1015200070697265642C20726573656E64696E679C
:10153000205342444C4F4520636F6D6D616E642EA5
:101540002E2E0D0A004C657473207761697420613A
:101550002062697420746F20736565206966207746
:101560006520676574204E6574776F726B205365D4
:1015700072766963652E2E2E0D0A005472616666BE
:101580006963204D616E6167656D656E742077617A
:10159000697420706572696F64206973206C6F6E66
:1015A00067202D2043616E27742073656E64206D63
:1015B0006573736167652061742074686973207452
:1015C000696D6521200D0A00526574727920746975
:1015D0006D657220657870697265642C2072657320
:1015E000656E64696E67204D4F2062756666657230
:1015F00020636C65617220636F6D6D616E642E2E69
:101600002E0D0A0052657472792074696D6572201E
:10161000657870697265642C20726573656E6469A3
:101620006E672041542B534244495820636F6D6DBF
:10163000616E642E2E2E0D0A004C65747320776146
:10164000697420612062697420746F20736565205D
:10165000696620776520676574204E6574776F72C0
:101660006B20536572766963652E2E2E0D0A004E2F
:101670006574776F726B20697320617661696C6144
:10168000626C6520736F206C6574732074727920AE
:10169000746F20726573656E64202E2E2E0D0A0005
:1016A000534244495820526573706F6E73652069C8
:1016B0006E64696361746564206661696C757265E6
:1016C000202E2E2E0D0A0052657175657374696E99
:1016D000672074726166666963206D616E6167651B
:1016E0006D656E7420706572696F642E2E2E0D0A02
:1016F0000053656E64204D65737361676520537593
:10170000636365737321200D0A005265747279203A
:1017100074696D657220657870697265642C2072D9
:101720006573656E64696E672042696E61727920C7
:10173000446174612E2E2E0D0A004E6F204E65748A
:10174000776F726B20617661696C61626C65206A8B
:10175000757374207965742C20736F206C657473B5
:101760002077616974206120626974202E2E2E0D0D
:101770000A0052657472792074696D65722065780B
:1017800070697265642C20726573656E64696E673A
:1017900020534244574220436F6D6D616E642E2E7C
:1017A0002E0D0A004E6577204972696469756D20B7
:1017B0004D65737361676520686173206265656E4E
:1017C000207375636365737366756C6C79207265DD
:1017D0007472696576656420616E64206865616411
:1017E000696E6720746F20706172736572202E2E8F
:1017F0002E2E200D0A004572726F72205265736F93
:101800006E73652072656365697665642066726FC4
:101810006D204972696469756D204D6F64756C65E2
:10182000202E2E2E2E200D0A0048617264776172E0
:1018300065204661696C757265205265736F6E73C1
:10184000652072656365697665642066726F6D20D8
:101850004972696469756D204D6F64756C65202EE1
:101860002E2E2E200D0A004E6574776F726B205558
:101870006E617661696C61626C65202E2E2E2E2061
:101880000D0A004E6574776F726B20417661696C4A
:1018900061626C65202E2E2E2E200D0A004E65747E
:1018A000776F726B20556E617661696C61626C65F1
:1018B000202E2E2E2E200D0A004E6574776F726B2F
:1018C00020417661696C61626C65202E2E2E2E207F
:1018D0000D0A0052494E47212052494E47212052BD
:1018E000494E47212052494E47212052494E472117
:1018F0002052494E4721200D0A00497269646975DA
:101900006D204552524F5221212121210D0A0045BF
:10191000786974696E67204972696469756D2047DA
:101920006574204D657373616765205374617465D8
:10193000204D616368696E652E2E2E0D0A00457874
:101940006974696E67204972696469756D205365B1
:101950006E64204D657373616765205374617465AF
:10196000204D616368696E652E2E2E0D0A00497246
:10197000696469756D205374617475732055706462
:10198000617465202F204D61696C626F7820436817
:1019900065636B20436F6D706C6574652E2E2E0D24
:1019A0000A004972696469756D20454550524F4D72
:1019B0002055706461746520537461727465642E7F
:1019C0002E2E0D0A004972696469756D2053746189
:1019D00074757320557064617465202F204D6169A2
:1019E0006C626F7820436865636B20537461727416
:1019F00065642E2E2E0D0A00456E746572696E6741
:101A0000204972696469756D20476574204D65735E
:101A100073616765205374617465204D6163686903
:101A20006E652E2E2E0D0A00456E746572696E6706
:101A3000204972696469756D2053656E64204D6537
:101A40007373616765205374617465204D616368C9
:101A5000696E652E2E2E0D0A004972696469756DD6
:101A60002053687574646F776E2073746172746547
:101A7000642E2E2E0D0A004972696469756D205519
:101A8000706461746520537461747573202F204DE8
:101A900061696C626F7820436865636B2053746181
:101AA0007274696E672E2E2E0D0A00497269646980
:101AB000756D20536574757020436F6D706C65741F
:101AC000652E2E2E0D0A004972696469756D204CD1
:101AD0006F6E6720536574757020537461727465FE
:101AE00064202E2E2E0D0A004972696469756D20DE
:101AF00053687574646F776E20636F6D706C657476
:101B000065202E2E2E0D0A004972696469756D20BC
:101B1000506F77657220557020436F6D706C6574DF
:101B200065210D0A004972696469756D20506F77EF
:101B3000657220557020537461727465642E2E2E68
:101B40000D0A004972696469756D20506F7765727E
:101B5000205570205265747279210D0A004972690E
:101B60006469756D20506F776572204572726F726F
:101B7000202D204578636565646564204D61786932
:101B80006D756D2052657472696573210D0A004D83
:101B90005353544D3A0053424453583A005342442D
:101BA0004C4F453A0053424449583A00534244523C
:101BB000494E47005245414459004F4B004841525D
:101BC0004457415245204641494C5552453A0045FB
:101BD00052524F52004353513A00434945563A300E
:101BE0002C00434945563A322C0041542B53424471
:101BF00057423D0041542659300041542B53424432
:101C00004958410041542B53424449580041542BF8
:101C10004950523D360041542657300041542B5311
:101C200042444D54413D310041542B5342445245AE
:101C3000470041542B53424452420041542B5342DB
:101C4000444C4F450041542D4D5353544D00415485
:101C500049330041542B4353510041542B534244C8
:101C6000535800415449340041542B43474D4D00D3
:101C700041542B43474D490041542B4347534E0099
:101C800041544937004154493600415449350041D7
:101C900054264B300041542B434945523D302C30A3
:101CA0002C302C302C300041542B434945523D31CF
:101CB0002C312C312C312C300041542A4600415417
:101CC000453000415426443000300041542B5342EB
:101CD0004444310041542B53424444300041542B7E
:101CE000534244443200556E61626C6520746F202B
:101CF0007365742052544320416C61726D2C2077BF
:101D000061746368646F672077696C6C20726573B7
:101D100065742073797374656D2E2E2E0D0A004143
:101D20006C61726D2054696D653A20004375727262
:101D3000656E742054696D653A2000537461727445
:101D40002053797374656D2053687574646F776E72
:101D50000D0A0056616C6964204669782C2073680E
:101D6000757474696E6720646F776E204750532EC8
:101D70002E2E0D0A004750532054696D656F7574FF
:101D80002C207368757474696E6720646F776E2099
:101D90004750532E2E2E0D0A000D0A000D0A204D1D
:101DA00061696C626F7820436F756E743D000D0A37
:101DB000205472616E736D697420436F756E743D4B
:101DC000002046697820436F756E743D00426C7543
:101DD00065746F6F746820697320656E61626C65ED
:101DE000642C2073687574646F776E2077696C6CEF
:101DF0002062652064656C61796564210D0A0020AC
:101E00007365636F6E64730D0A004E6578742063AA
:101E100079636C6520696E20636F6E6669677572A1
:101E200065642047505320696E74657276616C3A20
:101E30002000292C206E657874206379636C6520FE
:101E4000696E2035206D696E757465732E2E2E0DAA
:101E50000A0054657374204D6F6465206163746972
:101E600076652028000D0A53687574646F776E20BC
:101E7000726561736F6E3A204E6F20475053205346
:101E800069676E616C2E2E2E0D0A00426C756574AA
:101E90006F6F746820697320656E61626C65642C75
:101EA0002073687574646F776E2077696C6C20623C
:101EB000652064656C61796564210D0A0020736595
:101EC000636F6E64730D0A004E65787420637963E6
:101ED0006C6520696E20636F6E66696775726564F4
:101EE0002047505320696E74657276616C3A200009
:101EF000292C206E657874206379636C6520696E87
:101F00002035206D696E757465732E2E2E0D0A00B6
:101F100054657374204D6F646520616374697665E0
:101F20002028000D0A576174657220537769746325
:101F3000682044697361626C65642C205379737402
:101F4000656D20746F20537461727475700D0A0092
:101F50000D0A576174657220537769746368206451
:101F6000657465726D696E65642053797374656D0F
:101F700020746F20537461727475700D0A002073A1
:101F800065636F6E64730D0A004E65787420637923
:101F9000636C6520696E20636F6E66696775726534
:101FA000642047505320696E74657276616C3A20E4
:101FB00000292C206E657874206379636C65206934
:101FC0006E2035206D696E757465732E2E2E0D0A88
:101FD0000054657374204D6F646520616374697685
:101FE000652028000D0A53687574646F776E20723F
:101FF0006561736F6E3A205761746572205377691B
:102000007463680D0A000D0A4D61676E6574204E99
:102010006F742050726573656E740D0A000D0A535B
:10202000687574646F776E20726561736F6E3A20A5
:102030004D61676E6574205377697463680D0A009B
:1020400057617465722053776974636820446973BB
:1020500061626C65640D0A00576174657220537784
:102060006974636820456E61626C65640D0A00578F
:1020700061746572205377697463682053616D7071
:102080006C6564206173205375626D657267656469
:102090000D0A005761746572205377697463682074
:1020A00053616D706C65642061732041626F766569
:1020B0002057617465720D0A005761746572205370
:1020C00077697463682053616D706C696E672E2E3A
:1020D0002E0D0A0011241FBECFEFCDBFDFE5DEBFFE
:1020E00000E00CBF14E2A0E0B0E2EEEEFDEC00E098
:1020F0000BBF02C007900D92A433B107D9F724E4B7
:10210000A4E3B4E201C01D92A03FB207E1F70E9430
:1021100090510C94F5660C9400007F928F929F92E0
:10212000AF92BF92CF92DF92EF92FF920F931F93E5
:10213000CF93DF9391E0E0E0F6E09583833008F001
:10214000ADC090E0FC01EE0FFF1F9C01220F331F7A
:10215000220F331F220F331FE20FF31FE259FC4DF2
:102160000481158122E0D8012C93768011967C920F
:102170001197278112962C93129725E014962C9391
:102180001497208590962C939097218591962C9367
:10219000EFE4F3EC3197F1F700C00000E12CF12CF3
:1021A000812C912C5401C8EED3E06C01CC0CDD1CC9
:1021B000880F991F880F991F880F991F8C0D9D1DDF
:1021C0009C0122593C4D6901D8018C9181608C930E
:1021D0008C9184608C9316968C9180FD19C0CE01F1
:1021E0000197CD2B91F0EC01E3EFF1E03197F1F79E
:1021F00000C00000D80116968C9180FD09C0CE0168
:102200000197CD2B21F0EC01EFCFEC0101C0EC01E7
:10221000F8018681816086831082209759F1F8E069
:10222000EF16F104F4F0D80150966D917C9151971E
:1022300080E090E00E949962F60120813181428124
:1022400053810E94006220E030E040E85CE30E949D
:1022500027639B01AC01C501B4010E949C614B0145
:102260005C01FFEFEF1AFF0A28E4E216F10409F01F
:10227000ABCF03C0812C912C540174FC12C020916F
:102280003424309135244091362450913724C501AF
:10229000B4010E949B614B015C0103C0812C912C15
:1022A000540181E0E0E0F6E08683C501B401DF91EE
:1022B000CF911F910F91FF90EF90DF90CF90BF9043
:1022C000AF909F908F907F900895CF92DF92EF9282
:1022D000FF921092342410923524109236241092DA
:1022E000372480E01ADF6B017C0181E016DF9B015F
:1022F000AC01C701B6010E949B61609334247093C6
:1023000035248093362490933724FF90EF90DF900C
:10231000CF900895E0E0F6E081E08183868382E05B
:102320008093CA01E0E2F0E0E491A0E0B2E01C9604
:10233000EC931C97E1E2F0E0E4911D96EC93E4E26B
:10234000F0E0E491A0E4B2E01C96EC931C97E5E287
:10235000F0E0E4911D96EC93EEE2F0E06491EFE2A0
:10236000F0E0E49170E07E2B80E090E00E949962C2
:1023700020E030E040E859E30E942763609338246E
:102380007093392480933A2490933B241092CA018D
:102390009CCF0895C2DE22E53BE844E252E40C946F
:1023A00027630895CF92DF92EF92FF92CF93C82FC9
:1023B0002091342430913524409136245091372493
:1023C000609138247091392480913A2490913B2473
:1023D0000E949B619B01AC0163E373E183EB93E497
:1023E0000E9400626B017C018C2F97DEA701960191
:1023F0000E94276323E333E948E853E40E949B618A
:10240000CF91FF90EF90DF90CF900895E4E4F4E255
:102410008CE295E2DF0118971C92108211821282E1
:1024200013821482158216821782108611861286F4
:1024300013861486158616861786108A118A128AC4
:10244000138A148A7D96E817F90721F781E0089529
:1024500048EE50E06CE374E28BE591E00E94C553D6
:1024600081E008950F931F93CF93DF938B01883002
:10247000B0F59DE1899FE0011124C45CDB4DCE01E4
:102480000E943864F8018085888781859285A385BC
:10249000B48589879A87AB87BC8785859685A7850C
:1024A000B0898D879E87AF87B88B81899289A389F0
:1024B000B489898B9A8BAB8BBC8B4589568967898C
:1024C000708D4D8B5E8B6F8B788F418D528D638DB0
:1024D000748D498F5A8F6B8F7C8F81E001C080E0B3
:1024E000DF91CF911F910F910895FC0180818F3F63
:1024F00081F14585568567857089413055496A4B1C
:102500007A4048F541895289638974894130554937
:102510006A4B7A4010F5458956896789708D41303C
:102520005A4265477541D8F4418D528D638D748D43
:1025300041305A4265477541A0F481E0418552859A
:1025400063857485403452446F40710558F080E0D3
:10255000089580E0089580E0089580E0089580E087
:10256000089580E008950F931F93CF93DF9348EE73
:1025700050E06CE374E28BE591E00E94B853CCE349
:10258000D4E204E215E2CE01B0DF882329F06D9693
:10259000C017D107C1F702C080E001C081E0DF9120
:1025A000CF911F910F910895809124250895FC01EA
:1025B000108208958F929F92AF92BF92CF92DF9236
:1025C000EF92FF920F931F93CF93DF93CDB7DEB7B8
:1025D0002D97CDBFDEBF7C015B016A018AEA89834A
:1025E00085E58A831B821C82F70181818D8382812C
:1025F00080688E8393819F83188619869FEF9A87C0
:102600009CEC9B879081913069F48283C70104968A
:102610000E942F64B6016D5F7F4FC70101960E9433
:102620001D2E4FC0CA0103969B8383E0840F8C83C9
:10263000AE01445F5F4F61E08FEF0E9453348E0123
:102640000D5F1F4F4E01F8E08F0E911CAE01445FED
:102650005F4F60E0F80181918F010E9453340815AB
:102660001905A1F7C114D10481F0850145018C0C35
:102670009D1CAE01445F5F4F60E0F80181918F01C6
:102680000E94533408151905A1F78C859D859887FC
:10269000898747E050E0BE016F5F7F4FF70180817F
:1026A0000E94C158A601B501F70180810E94C1585E
:1026B00044E050E0BE01685F7F4FF70180810E94D7
:1026C000C15881E02D96CDBFDEBFDF91CF911F9124
:1026D0000F91FF90EF90DF90CF90BF90AF909F90C1
:1026E0008F900895EF92FF920F931F93CF93DF93F4
:1026F000CDB7DEB7CA5FD109CDBFDEBF8C01CE0139
:1027000001960E94C937CE0183599F4F0E941B41F9
:1027100082EE92E40E9486250F2EFAEFEF2EF2E46D
:10272000FF2EF02DF701608171818281938144E059
:102730000E941351F70160837183828393830F2E6C
:10274000F0E0EF2EF3E4FF2EF02DF70160817181B0
:1027500080E090E042E00E941351F70160837183B2
:1027600082E193E40E94123F82E093E40E94434F8F
:1027700040E850E062EE72E4C8011CDFC650DF4F53
:10278000CDBFDEBFDF91CF911F910F91FF90EF90F2
:1027900008950F931F93CF93DF93CDB7DEB72D9797
:1027A000CDBFDEBF8C01CE0101960E94E12F698171
:1027B0007A818B819C8144E00E94135169837A83E2
:1027C0008B839C8380E0E6DD20E030E040E251E452
:1027D0000E9427630E946D6242E00E9413516D8344
:1027E0007E8382E0DFDD0E9468626F83188619862F
:1027F0001A861B861C861D864DE050E0BE016F5F69
:102800007F4FC801D7DE2D96CDBFDEBFDF91CF91C0
:102810001F910F9108950F931F93CF93DF93CDB71F
:10282000DEB7CD54D140CDBFDEBF8C01CE010196C5
:102830000E94E12F69817A818B819C8144E00E9412
:10284000135169837A838B839C8380E0A3DD20E02E
:1028500030E040E251E40E9427630E946D6242E052
:102860000E9413516D837E8382E09CDD0E9468622A
:102870006F830E94DF2D8887CE018E519F4F0E946B
:10288000C937CE018C5A9F4F0E941B41CE51DF4F5A
:102890008881C25ED0408987CD51DF4F8881C35E79
:1028A000D0408A87CC51DF4F8881C45ED0408B876F
:1028B000CB51DF4F8881C55ED0408C8765968FAD48
:1028C00065978D8766968FAD66978E8769968FAD73
:1028D00069978F876A968FAD6A97888B6E966CAD75
:1028E0007DAD8EAD9FAD6E97698B7A8B8B8B9C8BFC
:1028F00044E00E941351698B7A8B8B8B9C8B6F9673
:102900008FAD6F978D8BA0968FADA0978E8BA49671
:102910008CAD9DADAEADBFADA4978F8B988FA98FB9
:10292000BA8FA6968EAD9FADA6978B8F9C8FA796DC
:102930008FADA7978D8FA8968FADA8978E8FAA96EB
:102940008EAD9FADAA978F8F98A3FE01ED52FF4FDA
:10295000DE019196CE018E519F4F21912D93E81764
:10296000F907D9F744E050E0BE01605D7F4F83E393
:102970009EE00E94332468A979A98AA99BA944E012
:102980000E94135168AB79AB8AAB9BAB44E050E03B
:10299000BE016C5C7F4F83E39DE00E9433246CA9F1
:1029A0007DA98EA99FA944E00E9413516CAB7DAB19
:1029B0008EAB9FAB44E050E0BE01685C7F4F83E389
:1029C0009CE00E94332468AD79AD8AAD9BAD44E0B4
:1029D0000E94135168AF79AF8AAF9BAFCE01CC96FE
:1029E0000E946F32CE018F5B9F4F0E94CD2D0E94BF
:1029F000146063968FAF6397D7DD64968FAF64974B
:102A000043E550E0BE016F5F7F4FC801D3DDC35B7C
:102A1000DE4FCDBFDEBFDF91CF911F910F910895A3
:102A2000CF93DF93CDB7DEB72597CDBFDEBF25E0CF
:102A3000E2E6F3E2DE01119601900D922A95E1F7AC
:102A400045E050E0BE016F5F7F4FB4DD2596CDBFFE
:102A5000DEBFDF91CF9108950F931F93CF93DF9344
:102A600000D01F92CDB7DEB78C01CE0101960E9437
:102A7000E12F69817A818B819C8144E00E9413510E
:102A800069837A838B839C8344E050E0BE016F5F4F
:102A90007F4FC8018FDD2496CDBFDEBFDF91CF9180
:102AA0001F910F910895AF92BF92CF92DF92EF9254
:102AB000FF920F931F93CF93DF93CDB7DEB761974C
:102AC000CDBFDEBF8C017C0184E0E80EF11CF80173
:102AD000648175818681978144E00E941351F801D9
:102AE0006483758386839783CE0109960E94E12FC4
:102AF00081E08D87F80184819581A681B781498520
:102B00005A856B857C8584179507A607B70728F437
:102B1000481B590B6A0B7B0B08C05C016D01A41AA2
:102B2000B50AC60AD70AB601A5014E875F87688B2A
:102B3000798BBE016E5F7F4FC7010E942430CE01AA
:102B400002960E94F52E91E0813009F490E0919573
:102B5000998341E050E0BE016F5F7F4FC8012ADDDD
:102B600045E050E0BE01635F7F4F8FE00E94EC289C
:102B70006196CDBFDEBFDF91CF911F910F91FF9086
:102B8000EF90DF90CF90BF90AF9008950F931F9379
:102B9000CF93DF931F92CDB7DEB78C018FEF898380
:102BA000F801EC5FFE4F60817181613581E078074B
:102BB00040F46D5F7F4FC80101960E941D2E811168
:102BC000198241E050E0BE016F5F7F4FC801F2DC27
:102BD0000F90DF91CF911F910F910895DF92EF92A7
:102BE000FF920F931F93CF93DF93CDB7DEB7C45BF4
:102BF000D109CDBFDEBF7C01FC0184818A3008F0A1
:102C000048C08983BE016E5F7F4F0E94F02C6A81AD
:102C10007B818C819D8144E00E9413516A837B8378
:102C20008C839D836E817F818885998544E00E9495
:102C300013516E837F83888799876C857D8580E0BB
:102C400090E042E00E9413516C877D876A857B8506
:102C500080E090E042E00E9413516A877B87698997
:102C60007A8980E090E042E00E941351698B7A8B70
:102C70006F85788980E090E042E00E9413516F8771
:102C8000788B42E150E0BE016F5F7F4FC70192DC5D
:102C900064C08F3F09F05AC08E010E5F1F4FD12CC8
:102CA000F8013197D082B8018D2D0E94F02CF801E7
:102CB000608171818281938144E00E941351F80107
:102CC0006083718382839383648175818681978118
:102CD00044E00E941351F8016483758386839783CF
:102CE0006285738580E090E042E00E941351F80114
:102CF000628773876085718580E090E042E00E9482
:102D00001351F801608771876785708980E090E0D2
:102D100042E00E941351F8016787708B65857685C4
:102D200080E090E042E00E941351F80165877687C9
:102D3000D3940E5E1F4FFAE0DF12B2CF44EB50E0A7
:102D4000BE016F5F7F4FC70135DC07C042E150E035
:102D5000BE016F5F7F4FC7012DDCCC54DF4FCDBF6D
:102D6000DEBFDF91CF911F910F91FF90EF90DF9029
:102D70000895DF92EF92FF920F931F93CF93DF930B
:102D8000CDB7DEB7E097CDBFDEBF7C01FC0184810B
:102D90008830C8F48983BE016E5F7F4F0E940B327A
:102DA0006A817B818C819D8144E00E9413516A83FA
:102DB0007B838C839D8346E050E0BE016F5F7F4F35
:102DC000C701F8DB2FC08F3F31F58E010E5F1F4F1B
:102DD000D12CF8013197D082B8018D2D0E940B3291
:102DE000F801608171818281938144E00E941351D6
:102DF000F8016083718382839383D3940A5F1F4FAA
:102E0000F8E0DF12E6CF40E350E0BE016F5F7F4F96
:102E1000C701D0DB07C046E050E0BE016F5F7F4FC7
:102E2000C701C8DBE096CDBFDEBFDF91CF911F9118
:102E30000F91FF90EF90DF9008950F931F93CF9322
:102E4000DF93CDB7DEB76E97CDBFDEBF8C01FE013D
:102E500031968EE1DF011D928A95E9F78FEF898324
:102E6000F8018481883008F045C08983FDE18F9F97
:102E7000C00111244DE150E0BE016E5F7F4F855AC5
:102E80009E4F0E94B8536F85788989899A8944E05A
:102E90000E9413516F87788B898B9A8B6F89788DFD
:102EA000898D9A8D44E00E9413516F8B788F898FA2
:102EB0009A8F6B897C898D899E8944E00E94135189
:102EC0006B8B7C8B8D8B9E8B6B8D7C8D8D8D9E8D7E
:102ED00044E00E9413516B8F7C8F8D8F9E8F6B858A
:102EE0007C858D859E8544E00E9413516B877C878D
:102EF0008D879E874EE150E0BE016F5F7F4FC80116
:102F000059DB6E96CDBFDEBFDF91CF911F910F9140
:102F100008950F931F93CF93DF93CDB7DEB76297DA
:102F2000CDBFDEBF8C01FE01319682E1DF011D9233
:102F30008A95E9F78FEF8983F8018481883020F53D
:102F40008983F1E18F9FC001112441E150E0BE016E
:102F50006E5F7F4F8D5B9D4F0E94B8536B857C8564
:102F60008D859E8544E00E9413516B877C878D87F9
:102F70009E876F85788989899A8944E00E941351D8
:102F80006F87788B898B9A8B42E150E0BE016F5F2F
:102F90007F4FC8010FDB6296CDBFDEBFDF91CF91BF
:102FA0001F910F9108957F928F929F92AF92BF923F
:102FB000CF92DF92EF92FF920F931F93CF93DF9305
:102FC000CDB7DEB7C55BD109CDBFDEBF5C018FEFEA
:102FD000CB54DF4F8883C55BD040F50184818A30B4
:102FE00008F071C0EC5FFE4F80819181429709F03B
:102FF0006AC082E1FA95DE01119601900D928A95E0
:10300000E1F76A817B818C819D8144E00E941351AC
:103010006A837B838C839D836E817F81888599857C
:1030200044E00E9413516E837F83888799876A8565
:103030007B8580E090E042E00E9413516A877B87A5
:103040006C857D8580E090E042E00E9413516C87A2
:103050007D876F85788980E090E042E00E9413517F
:103060006F87788B69897A8980E090E042E00E94DE
:103070001351698B7A8BCE0102960E94562D8130B6
:10308000B1F4BE016E5F7F4F89810E941A2DF50158
:1030900080810E94002D0E94585B67EB74E081E004
:1030A000FAD6CB54DF4F1882C55BD04004C068E825
:1030B00074E081E0F0D641E050E0BE016B547F4FF8
:1030C000C50178DA9AC0F501EC5FFE4F80819181ED
:1030D000843B910509F08AC08E010F5F1F4F750177
:1030E000F4E0EF0EF11C6E0185EBC80ED11C0F2E23
:1030F000F4EB7F2EF02DF701D801872D01900D9272
:103100008A95E1F7F801618172818381948144E0BD
:103110000E941351F80161837283838394836581D4
:1031200076818781908544E00E941351F801658380
:103130007683878390876385748580E090E042E0A2
:103140000E941351F801638774876185728580E05E
:1031500090E042E00E941351F80161877287608914
:10316000718980E090E042E00E941351F801608B89
:10317000718B6685778580E090E042E00E94135174
:10318000F801668777874801FFEF8F1A9F0AC4010D
:103190000E94562D813061F4B401F80180810E94B3
:1031A0001A2D0E94585B60E774E081E074D604C079
:1031B00066E574E081E06FD60E5E1F4FF4EBEF0E14
:1031C000F11C0C151D0509F096CFF50180810E94B8
:1031D000002DCB54DF4F1882C55BD04041E050E05A
:1031E000BE016B547F4FC501E5D907C041E050E0F7
:1031F000BE016B547F4FC501DDD9CB54DF4FCDBF2E
:10320000DEBFDF91CF911F910F91FF90EF90DF9084
:10321000CF90BF90AF909F908F907F9008959F9296
:10322000AF92BF92CF92DF92EF92FF920F931F93D4
:10323000CF93DF93CDB7DEB7E197CDBFDEBF6C0193
:103240008FEF89ABF6018481883050F5EC5FFE4F3B
:1032500080819181069721F586E0FA95DE0111962D
:1032600001900D928A95E1F76A817B818C819D8125
:1032700044E00E9413516A837B838C839D83BE014B
:103280006E5F7F4F89810E9429320E941F3219AAE6
:1032900041E050E0BE016F5C7F4FC6018BD94AC050
:1032A000F601EC5FFE4F80819181C097E1F58E01C0
:1032B0000F5F1F4F7601F4E0EF0EF11C5E0181E31A
:1032C000A80EB11C0F2EF0E39F2EF02DF701D801B0
:1032D000892D01900D928A95E1F7F8016181728143
:1032E0008381948144E00E941351F80161837283C9
:1032F00083839483B8016F5F7F4F80810E9429325E
:103300000A5F1F4FF0E3EF0EF11C0A151B05F1F6E3
:103310000E941F3219AA41E050E0BE016F5C7F4F4E
:10332000C60148D907C041E050E0BE016F5C7F4F45
:10333000C60140D9E196CDBFDEBFDF91CF911F918D
:103340000F91FF90EF90DF90CF90BF90AF909F9044
:1033500008950F931F93CF93DF93CDB7DEB76F9789
:10336000CDBFDEBF8C01FE0131968EE1DF011D92E3
:103370008A95E9F78FEF89838F8FF80184818830F0
:1033800008F05AC0EC5FFE4F808191814E9709F0A2
:1033900053C08EE1FA95DE01119601900D928A9547
:1033A000E1F76F85788989899A8944E00E941351F1
:1033B0006F87788B898B9A8B6F89788D898D9A8DA1
:1033C00044E00E9413516F8B788F898F9A8F6B899D
:1033D0007C898D899E8944E00E9413516B8B7C8B84
:1033E0008D8B9E8B6B8D7C8D8D8D9E8D44E00E9490
:1033F00013516B8F7C8F8D8F9E8F6B857C858D8518
:103400009E8544E00E9413516B877C878D879E8741
:103410008981FDE18F9FC00111244DE150E0BE0183
:103420006E5F7F4F855A9E4F0E94C553BE016E5FEF
:103430007F4F898117D81F8E41E050E0BE01615E49
:103440007F4FC801B7D86F96CDBFDEBFDF91CF9158
:103450001F910F9108950F931F93CF93DF93CDB7D3
:10346000DEB76397CDBFDEBF8C01FE01319682E1EE
:10347000DF011D928A95E9F78FEF89838B8BF80125
:1034800084818830C8F5EC5FFE4F8081918142973E
:1034900099F582E1FA95DE01119601900D928A95D7
:1034A000E1F76B857C858D859E8544E00E941351F4
:1034B0006B877C878D879E876F85788989899A89B4
:1034C00044E00E9413516F87788B898B9A8B898196
:1034D000F1E18F9FC001112441E150E0BE016E5F18
:1034E0007F4F8D5B9D4F0E94C553BE016E5F7F4F26
:1034F00089810E94B25F1B8A41E050E0BE016D5E8F
:103500007F4FC80157D86396CDBFDEBFDF91CF9103
:103510001F910F9108950F931F93CF93DF931F92E5
:10352000CDB7DEB78C018FEF8983F80184818430B9
:1035300010F484D4198241E050E0BE016F5F7F4FE8
:10354000C80138D80F90DF91CF911F910F91089546
:103550000F931F93CF93DF931F921F92CDB7DEB7C8
:103560008C011982FC0180818A8341E050E0BE0118
:103570006E5F7F4F80E090E00E94C55341E050E0D5
:10358000BE016F5F7F4FC80115D801C00000F80170
:1035900080810E9400578823C9F38FE493EC019740
:1035A000F1F700C00000F89481E08CBFE0E0F4EF98
:1035B00019950F900F90DF91CF911F910F91089562
:1035C0000F931F93CF93DF93CDB7DEB76097CDBF37
:1035D000DEBF8C0144E050E0BE016F5F7F4F83E3AC
:1035E0009EE00E94332469817A818B819C8144E032
:1035F0000E94135169837A838B839C8344E050E05B
:10360000BE016B5F7F4F83E39DE00E9433246D8199
:103610007E818F81988544E00E9413516D837E8363
:103620008F83988744E060E070E0CB010E941351E3
:1036300069877A878B879C8744E060E070E0CB01E4
:103640000E9413516D877E878F87988B40E150E0F1
:10365000BE016F5F7F4FC8010E94DA126096CDBF36
:10366000DEBFDF91CF911F910F910895CF93DF932C
:1036700000D01F92CDB7DEB719821A821B821C823E
:1036800044E050E0BE016F5F7F4F0E94DA12249643
:10369000CDBFDEBFDF91CF910895CF92DF92EF9241
:1036A0000F93CF93DF93CDB7DEB72997CDBFDEBFA2
:1036B0006C01862FF601EC5FFE4F208131812830AE
:1036C000310521F4B6016C5F7F4F02C060E070E00D
:1036D000F601E08003819E012A5F3F4FAE014E5FFD
:1036E0005F4F0E9456298130C1F46A817B818C81B1
:1036F0009D8144E00E9413516A837B838C839D8368
:103700006E817F818885998544E00E9413516E8384
:103710007F838887998719820AC01A821B821C823C
:103720001D821E821F82188619868FEF898349E0C9
:1037300050E0BE016F5F7F4FC6010E94DA122996EA
:10374000CDBFDEBFDF91CF910F91EF90DF90CF9093
:1037500008950F931F93CF93DF931F92CDB7DEB7DA
:103760008C010E94492A91E0813009F490E0919502
:10377000998341E050E0BE016F5F7F4FC8010E9416
:10378000DA120F90DF91CF911F910F9108950F934F
:103790001F93CF93DF931F92CDB7DEB78C018FEFCE
:1037A0008983F801608183810E94DE28813009F4D9
:1037B000198241E050E0BE016F5F7F4FC8010E9457
:1037C000DA120F90DF91CF911F910F9108950F930F
:1037D0001F93CF93DF931F92CDB7DEB78C01198271
:1037E00068E274E081E057D3F80180810E94692C7F
:1037F00041E050E0BE016F5F7F4FC8010E94DA12C6
:103800000F90DF91CF911F910F9108951F93CF9348
:10381000DF93EC01162F488150E04A30510508F043
:10382000BBC0FA01E250FF4F0C94EA631B8219827D
:103830001A821E821F82FC01E45FFE4F10821182F9
:1038400081E08883AE01405F5E4F61E08FEF0E94B0
:1038500053341A3A39F480E09AEA8C839D8382E0EB
:1038600088839BC0188299C0153541F48C819D8155
:1038700085658C839D8383E088838FC018828DC08B
:103880001E821F83AC01405F5E4F60E0812F0E946B
:10389000533484E0888381C08E819F81812B8E8305
:1038A0009F83AE01405F5E4F60E0812F0E945334E2
:1038B00085E0888372C029813A81C9010196898394
:1038C0009A832130310539F020F02230310529F07A
:1038D00006C0198712C01A8710C01B870EC0FE01D0
:1038E000E45FFE4F808191819C012F5F3F4F2083D9
:1038F0003183FE01E80FF91F1487AE01405F5E4F70
:1039000060E0812F0E94533429813A818E819F810A
:103910002817390708F441C086E088833EC0FC01BF
:10392000E25FFE4F1082118387E0888336C0FC017E
:10393000E25FFE4F20813181C901812B8083918319
:103940003296208131818217930719F488E08883A9
:1039500024C06EEF73E081E09ED218821EC01F3F2C
:1039600051F480E09FEFFE01EE5EFE4F8083918375
:1039700089E0888312C0188210C01C3C59F4FC01F5
:10398000EE5EFE4F808191818C6C8083918381E01B
:103990008B8303C0188201C018828B81DF91CF9185
:1039A0001F910895AF92BF92CF92DF92EF92FF9254
:1039B0000F931F93CF93DF93CDB7DEB72797CDBF7C
:1039C000DEBF5C018B01FB01818592858E839F8325
:1039D00083858D8384858C8385858B8386858A8387
:1039E00027853089369527953695279536952795DD
:1039F000A5ECB0E20E94F063929582958F708927C2
:103A00009F7089278983B501CE0101960E943C2FC2
:103A1000F501608171818281938144E00E9413519C
:103A2000F5016083718382839383F80144A18DEC57
:103A3000489F412D1124469546954770406823A123
:103A400030E02350310927703327C901880F991FAF
:103A5000880F991F880F991F842BF5018483F80123
:103A600061897289838994890F2EFAE0CF2ED12C37
:103A7000E12CF12CF02DA70196010E94CE63CA0122
:103A8000B9016058754B824A9A4F44E00E94135125
:103A9000F5016583768387839087F8016589768948
:103AA0008789908DA70196010E94CE63CA01B90152
:103AB0007B568544954F44E00E941351F501618780
:103AC000728783879487F801838D948DA58DB68D39
:103AD0008F3F9105A105B10511F008F08FEFF501B9
:103AE0008687F801818D928D8F3F910511F008F046
:103AF0008FEFF5018587F801838194818F3F9105D0
:103B000011F008F08FEFF5018787F801818181308E
:103B1000C9F4C5010E94E12FF501608171818281A4
:103B2000938144E00E941351F50160837183828385
:103B3000938389E08483F80183A18B3008F080E0CF
:103B4000F501878781E02796CDBFDEBFDF91CF915A
:103B50001F910F91FF90EF90DF90CF90BF90AF90AB
:103B600008950F931F93CF93DF93CDB7DEB7E597FB
:103B7000CDBFDEBF8C0160E0CE0141960E94A73729
:103B8000BE016F5E7F4FCE0101960CDF40E150E039
:103B9000BE016F5F7F4FC8010E94DA12E596CDBF6C
:103BA000DEBFDF91CF911F910F9108950F931F9367
:103BB000CF93DF931F92CDB7DEB78C0181E089836D
:103BC0000E94585BC801CDDF41E050E0BE016F5F4D
:103BD0007F4F80E10E94EC280F90DF91CF911F91E1
:103BE0000F910895CF93DF93EC01262F688389818D
:103BF0008530C9F118F4833041F094C0873009F45E
:103C00005AC0893009F464C08DC08A8190E0FC01FB
:103C10003197E033F10508F087C0E85FFE4F0C9460
:103C2000EA63CE010E947213ACC0CE010E94C91398
:103C3000A8C0CE010E941015A4C0CE010E940B1492
:103C4000A0C0CE018EDF9DC0CE01B0DF9AC0CE01F4
:103C50000E942C1596C0CE010E94531592C0CE0131
:103C60000E94C6158EC04A8150E0FA013197E032B9
:103C7000F10508F05BC0E85CFE4F0C94EA63CE01EE
:103C80000E94EE157EC0CE0174D87BC0CE01D5D87F
:103C900078C0CE013ED975C0CE0185D972C0CE01A3
:103CA000BEDA6FC0CE0155DB6CC0CE01D4DB69C07B
:103CB000CE0131DC66C08A81813008F43EC0843098
:103CC00008F436C0843009F038C0CE0141DC59C058
:103CD0004A8150E0FA013197E034F10558F5E85A8D
:103CE000FE4F0C94EA63CE016BDC4BC0CE01BEDC10
:103CF00048C060E0CE01D1DC44C061E0CE01CDDC43
:103D000040C062E0CE01C9DC3CC063E0CE01C5DC4E
:103D100038C0CE011EDD35C0CE0139DD32C0CE0146
:103D200056DD2FC080E007C080E005C080E003C002
:103D300081E001C080E0811124C0213011F50E9492
:103D4000A132813069F4FE01EC5FFE4F4081518168
:103D50004D5F5F4FBE016F5F7F4F80E00E94C15893
:103D60000E94F032813069F4FE01EC5FFE4F408129
:103D700051814D5F5F4FBE016F5F7F4F83E00E94B7
:103D8000C158DF91CF910895CF93DF93CDB7DEB7C0
:103D9000C650D140CDBFDEBFBE016B5F7E4FCE01AE
:103DA00002960E94DC40882341F061E0CE0101963A
:103DB00019DF66E075E081E06ED00E94652A81110E
:103DC00014C00E948940823019F0833041F00DC048
:103DD0000E94954F6EEE74E081E05DD006C00E94B7
:103DE000954F6FEC74E081E056D0CA5FDE4FCDBFD7
:103DF000DEBFDF91CF9108950E94AC2D811105C0E7
:103E00000E94C22C80E00E94002D0E944E3281113F
:103E100004C00E94F9310E941F320E94B312811126
:103E200004C00E9406120E9428120E94F35F8111B2
:103E300004C00E948B5F0C94A85F08958093252591
:103E40000895CF93DF93EB0190912525981700F10A
:103E50000E94A132813061F4FE0101900020E9F757
:103E60003197AF014C1B5D0BBE0180E00E94C15831
:103E70000E94F032813061F4FE0101900020E9F7E8
:103E80003197AF014C1B5D0BBE0183E00E94C1580E
:103E9000DF91CF910895CF93DF93EB01909125258A
:103EA0009817C0F00E94A132813041F4CE010E94E7
:103EB0002664AC01BE0180E00E94AF590E94F0323E
:103EC000813041F4CE010E942664AC01BE0183E042
:103ED0000E94AF59DF91CF910895CF93C82F809161
:103EE00025258C1740F082EE93E40E94B44F62EED9
:103EF00073E48C2FA6DFCF9108952F923F924F92BB
:103F00005F926F927F928F929F92AF92BF92CF9269
:103F1000DF92EF92FF920F931F93CF93DF93CDB772
:103F2000DEB76697CDBFDEBFFC0180818D877280D2
:103F300023803480A185B285AD8BBE8B4384B4854C
:103F4000BC8B85858B8B96859A8B07851089C1885C
:103F5000D288E388F48885889688A788B08C838D7A
:103F6000948DA58DB68D8E879F87A88BB98B0E9467
:103F7000A037882309F42EC30E941B3F811105C07E
:103F800063EE76E081E087DF8EC29D85992321F084
:103F90006BED76E081E07FDF872D90E08730910543
:103FA00040F5FC01E856FE4F0C94EA6362ED76E0C2
:103FB00081E071DF22C069EC76E081E06CDF1DC03A
:103FC00060EC76E081E067DF18C067EB76E081E0C7
:103FD00062DF13C06EEA76E081E05DDF0EC065EA65
:103FE00076E081E058DF09C06CE976E081E053DFDC
:103FF00004C063E976E081E04EDF512C612C712C26
:10400000411451046104710429F460E976E081E00F
:1040100042DF0CC0AAE04A1651046104710408F0A2
:104020004FC26EE876E081E036DF4AC26CE876E0A7
:1040300081E031DFBC894B2E512C612C712C411455
:1040400051046104710429F469E876E081E023DF1A
:104050000CC08AE0481651046104710408F03CC2A7
:1040600067E876E081E017DF37C265E876E081E057
:1040700012DFAD89BE89AD0160E070E0CE0101962E
:104080000E94B44FBE016F5F7F4F81E0DADE63E8CC
:1040900076E081E000DFBB894B2E512C612C712C26
:1040A000411451046104710429F460E876E081E070
:1040B000F2DE0CC08AE0481651046104710408F075
:1040C00017C26EE776E081E0E6DE12C26CE776E0CA
:1040D00081E0E1DE9A89492E512C612C712C41142A
:1040E00051046104710429F469E776E081E0D3DECC
:1040F0000CC0AAE04A1651046104710408F004C21D
:1041000067E776E081E0C7DEFFC165E776E081E042
:10411000C2DE9801369527953695279536952795D1
:10412000A5ECB0E20E94F063929582958F7089278A
:104130009F7089272C01612C712C4114510461045A
:10414000710429F462E776E081E0A5DE0CC0BAE0F4
:104150004B1651046104710408F0E2C160E776E097
:1041600081E099DEDDC16EE676E081E094DEA8EEC6
:10417000B3E0A30192010E94FF632801612C712C1E
:10418000461A570A680A790A29F46AE676E081E055
:1041900082DE17C08AE0481651046104710428F4D5
:1041A00067E676E081E077DEC7C194E64916510400
:1041B0006104710408F0C0C165E676E081E06BDE61
:1041C000BBC162E676E081E066DEFF206CF460E66B
:1041D00076E081E060DEF094E094D094C094C11C5D
:1041E000D11CE11CF11C04C06EE576E081E053DED9
:1041F000C701B60120E836E948E950E00E94CE63E5
:10420000722E632E042F152F822F932FA42FB52FDC
:104210000097A105B10529F46BE576E081E03BDE6E
:104220000AC00A97A105B10508F092C169E576E0D8
:1042300081E031DE8DC167E576E081E02CDE272D5F
:10424000362D402F512F60E876E988E990E00E94F2
:104250008A63C61AD70AE80AF90A29F46FE476E0F5
:1042600081E019DE49C0AAE0CA16D104E104F104D4
:1042700028F468E476E081E00EDE78C1B4E6CB167F
:10428000D104E104F10428F462E476E081E003DE85
:104290006DC188EEC81683E0D806E104F10428F465
:1042A0006DE376E081E0F7DD61C190E1C91697E248
:1042B000D906E104F10428F469E376E081E0EBDD5E
:1042C00055C1A0EACA16A6E8DA06A1E0EA06F1049A
:1042D00028F466E376E081E0DEDD48C1B0E4CB1689
:1042E000B2E4DB06BFE0EB06F10408F03FC164E393
:1042F00076E081E0D0DD3AC161E376E081E0CBDDBC
:10430000BB206CF46FE276E081E0C5DDB094A09450
:1043100090948094811C911CA11CB11C04C06DE27E
:1043200076E081E0B8DDC501B40120E836E948E96E
:1043300050E00E94CE63E22EF32E042F152F822F21
:10434000932FA42FB52F0097A105B10529F46AE298
:1043500076E081E0A0DD0AC00A97A105B10508F06A
:1043600011C168E276E081E096DD0CC166E276E09C
:1043700081E091DD2E2D3F2D402F512F60E876E911
:1043800088E990E00E948A6375016401C61AD70A21
:10439000E80AF90A29F46EE176E081E07CDD49C0A3
:1043A0008AE0C816D104E104F10428F467E176E05C
:1043B00081E071DDF5C094E6C916D104E104F10491
:1043C00028F461E176E081E066DDEAC0A8EECA1675
:1043D000A3E0DA06E104F10428F46CE076E081E081
:1043E0005ADDDEC0B0E1CB16B7E2DB06E104F10432
:1043F00028F468E076E081E04EDDD2C080EAC8169D
:1044000086E8D80681E0E806F10428F465E076E065
:1044100081E041DDC5C090E4C91692E4D9069FE071
:10442000E906F10408F0BCC063E076E081E033DD2A
:10443000B7C060E076E081E02EDD69EF75E081E0F5
:104440002ADD8E859F85A889B989892B8A2B8B2B9C
:1044500009F0B2C067EF75E081E01DDD62EF75E045
:1044600081E019DD6CEE75E081E015DD2114310489
:1044700029F46AEE75E081E00EDD11C0A10160E073
:1044800070E0411551056105710549F0CE010196B5
:104490000E94B44FBE016F5F7F4F81E0D2DC64EEBB
:1044A00075E081E0F8DC9D85992329F06FED75E0DA
:1044B00081E0F1DC8FC06CED75E081E0ECDC8AC05E
:1044C000B301A201CE0101960E94B44FBE016F5FFD
:1044D0007F4F81E0B6DCAACDB301A201CE010196E7
:1044E0000E94B44FBE016F5F7F4F81E0AADCBDCD5B
:1044F000B301A201CE0101960E94B44FBE016F5FCD
:104500007F4F81E09EDCE2CDB301A201CE01019696
:104510000E94B44FBE016F5F7F4F81E092DCF5CD0A
:10452000B301A201CE0101960E94B44FBE016F5F9C
:104530007F4F81E086DC17CEB301A201CE01019648
:104540000E94B44FBE016F5F7F4F81E07ADC39CEAD
:10455000472D562D602F712FCE0101960E94B44F2A
:10456000BE016F5F7F4F81E06CDC65CEB701A601B5
:10457000CE0101960E94B44FBE016F5F7F4F81E074
:1045800060DCBACE4E2D5F2D602F712FCE010196CB
:104590000E94B44FBE016F5F7F4F81E052DCE6CED8
:1045A000B701A601CE0101960E94B44FBE016F5F14
:1045B0007F4F81E046DC3DCF4E855F8568897989F4
:1045C000CE0101960E94B44FBE016F5F7F4F81E024
:1045D00038DC44CF6696CDBFDEBFDF91CF911F910F
:1045E0000F91FF90EF90DF90CF90BF90AF909F9092
:1045F0008F907F906F905F904F903F902F90089595
:10460000CF93DF93CDB7DEB72797CDBFDEBFBE0117
:104610006F5F7F4F0E9424304D8150E060E070E07A
:1046200081E05BDC6CE873E281E00BDC4C8150E004
:1046300060E070E081E051DC6CE873E281E001DC75
:104640004E815F8160E070E081E047DC6EE873E2FC
:1046500081E0F7DB4B8150E060E070E081E03DDC21
:1046600060E973E281E0EDDB4A8150E060E070E0F8
:1046700081E033DC60E973E281E0E3DB498150E013
:1046800060E070E081E029DC6EEF73E281E0D9DB6D
:104690002796CDBFDEBFDF91CF9108950F931F9373
:1046A000CF93DF93CDB7DEB72897CDBFDEBF8E01A6
:1046B0000F5F1F4F88E0F80111928A95E9F782E6B3
:1046C00093E424D2C8012BD262E673E481E0B9DB23
:1046D00069ED75E081E0DFDBB80181E0B2DB67ED19
:1046E00075E081E0D8DB65EC75E081E0D4DB4091DA
:1046F0007A4350917B4360917C4370917D4381E08C
:10470000ECDB68EB75E081E0C6DB40917E4350E076
:1047100060E070E081E0E1DB66EB75E081E0BBDB4F
:1047200040917F4350E060E070E081E0D6DB64EBD5
:1047300075E081E0B0DB409180435091814360E0BF
:1047400070E081E0CADB6FEA75E081E0A4DB60EA3B
:1047500075E081E0A0DB0E948B2CAB01BC0181E005
:10476000BCDB69E875E081E096DB0E94AD2CAC0112
:1047700060E070E081E0B1DB69E675E081E08BDB51
:104780000E94982CAC0160E070E081E0A6DB63E55C
:1047900075E081E080DB0E94A32C482F50E060E0B0
:1047A00070E081E09ADB6AE375E081E074DB0E94EF
:1047B000B82C482F50E060E070E081E08EDB67E3CA
:1047C00075E081E068DB2896CDBFDEBFDF91CF9139
:1047D0001F910F910895CF92DF92EF92FF920F9366
:1047E0001F93CF93DF931F92CDB7DEB77C018B0170
:1047F00041E050E0BE016F5F7F4FC801C3970E9448
:10480000B85302531109D12CC98041E050E0BE01D8
:104810006F5F7F4FC8010E94B85381E08C0D998172
:10482000891739F0E114F10489F0F701C0828D2D68
:1048300010C0D3940F5F1F4FF2E3DF12E5CFE114F6
:10484000F10431F0F701808382E303C08D2D01C0B4
:1048500082E30F90DF91CF911F910F91FF90EF9026
:10486000DF90CF900895CF92DF92EF92FF920F9357
:104870001F93CF93DF931F92CDB7DEB78C016B01EF
:104880007A01BC01CE010196A6DF282F2E9DC00122
:104890002F9D900D1124A701B601800F911F0E943A
:1048A000B8530F90DF91CF911F910F91FF90EF9030
:1048B000DF90CF900895AF92BF92CF92DF92EF92A8
:1048C000FF920F931F93CF93DF931F92CDB7DEB765
:1048D0008C015B016A01BC01CE0101967CDF8F5F18
:1048E000833308F080E099819F5F9983E82EF12C53
:1048F000EC9CC001ED9C900DFC9C900D1124A60138
:10490000B501800F911F0E94C553C801C39741E0B4
:1049100050E0BE016F5F7F4F8E0D9F1D0E94C553FB
:104920000F90DF91CF911F910F91FF90EF90DF904B
:10493000CF90BF90AF900895CF93DF93CDB7DEB700
:10494000C258D109CDBFDEBF40E850E0BE016F5F65
:104950007F4F80E090E00E9452546EE770E0CE01FD
:1049600001960E947434C158DF4F28813981CF5796
:10497000D0402817390709F05EC089819A810197D4
:1049800009F043C08B8180933025813071F018F09D
:104990008230A9F01EC088E0E2E9F3E2A1E3B5E2CB
:1049A00001900D928A95E1F71DC088E0EAE9F3E2F3
:1049B000A1E3B5E201900D928A95E1F713C088E07A
:1049C000E2EAF3E2A1E3B5E201900D928A95E1F704
:1049D00009C088E0EAEAF3E2A1E3B5E201900D92B2
:1049E0008A95E1F78D819E81AF81B88580934925B5
:1049F00090934A25A0934B25B0934C2589859A85A1
:104A000080932E2590932F252DC088E0EAEAF3E2CB
:104A1000A1E3B5E201900D928A95E1F71092492544
:104A200010924A2510924B2510924C2510922E255B
:104A300010922F2517C088E0E2E9F3E2A1E3B5E286
:104A400001900D928A95E1F744E050E069E475E247
:104A500089E190E00E94B85382E090E080932E2597
:104A600090932F2542E050E06EEE71E0CE018F571B
:104A70009F4F0E941D64CE57DF4F8881C258D0409F
:104A80008F93CF57DF4F8881C158D0408F9382EBEF
:104A900093E29F938F9386E295E29F938F930E9478
:104AA0003F6444E050E060EF71E08DE495E20E94E5
:104AB0001D6481E595E20E94434F0F900F900F9087
:104AC0000F900F900F90809151258F3F41F4E1E5B9
:104AD000F5E288E595E21192E817F907E1F781E63A
:104AE00095E20E94123F809161258F3F41F4E1E6FB
:104AF000F5E28FE695E21192E817F907E1F7CE5754
:104B0000DF4FCDBFDEBFDF91CF91089520E8E1E315
:104B1000F5E2DC0101900D922A95E1F7089528E075
:104B2000E6E2F5E2DC0101900D922A95E1F70895A5
:104B3000809130250895E0E8F6E082E08183868365
:104B40001092B4251092B6251092B72587EB95E206
:104B50000E9417601092B52508958091B62588238C
:104B600009F462C08091B4258130C1F0823009F42B
:104B70003DC08091B525882309F456C08091B725A2
:104B8000811152C08091B3258093B72582E0E0E87F
:104B9000F6E0858381E08093B42508958091B72560
:104BA000811142C08091B225882349F08093B725B6
:104BB00082E0E0E8F6E086838093B4250895809152
:104BC000B125882359F081508093B1258091B32578
:104BD0008093B72581E08093B42508951092B52580
:104BE0008CE08093B7251092B42508958091B72565
:104BF00081111AC08091B125882379F0815080936A
:104C0000B1258091B3258093B72581E08093B425A9
:104C100082E0E0E8F6E0858308951092B5258CE007
:104C20008093B7251092B42508958091B6258111FF
:104C30000DC081E08093B62582E0E0E8F6E086834F
:104C40001092B4251092B7251092B5250895CF93F0
:104C5000DF9300D01F92CDB7DEB744E050E0BE0135
:104C60006F5F7F4F83E39EE0FEDD89819A81AB8198
:104C7000BC810097A105BF4F60F019821A821B8288
:104C80001C8244E050E0BE016F5F7F4F83E39EE0F3
:104C900012DE44E050E0BE016F5F7F4F83E39DE092
:104CA000E2DD89819A81AB81BC810097A105BF4F6C
:104CB00060F019821A821B821C8244E050E0BE011F
:104CC0006F5F7F4F83E39DE0F6DD44E050E0BE017F
:104CD0006F5F7F4F83E39CE0C6DD89819A81AB8162
:104CE000BC810097A105BF4F60F019821A821B8218
:104CF0001C8244E050E0BE016F5F7F4F83E39CE085
:104D0000DADD8DE697E20E94176083E597E20E9464
:104D100017602496CDBFDEBFDF91CF910895CF936A
:104D2000DF93CDB7DEB7CB50D140CDBFDEBF809192
:104D30004F27882319F0813061F05BC080915427A0
:104D4000813009F05CC080934F2784E08093532723
:104D500056C080915327811152C084E0809353271D
:104D6000CE01895F9E4F0E940735C95FDE4F888163
:104D7000C750D14080FD43C0C85FDE4F1882198202
:104D80001A821B82C850D14044E050E0BE01685FE7
:104D90007E4F83E39EE08FDD44E050E0BE01685F1C
:104DA0007E4F83E39DE087DD44E050E0BE01685F15
:104DB0007E4F83E39CE07FDD89E08A838EEF8B83E7
:104DC000809152278C83809151278983C95FDE4F60
:104DD0001882C750D14041E050E0BE01695F7E4F6C
:104DE000CE0101960E94DA121092542710924F279A
:104DF00006C010924F2768E877E081E04CD8C55F85
:104E0000DE4FCDBFDEBFDF91CF910895CF92DF920D
:104E1000EF92FF920F931F93CF93DF93CDB7DEB73F
:104E2000C650D140CDBFDEBF80914E27823009F4FD
:104E3000F4C028F4882361F0813059F155C18430E1
:104E400009F438C108F415C1853009F444C14CC1D6
:104E500080916C27813009F047C110926C27109225
:104E60006B278091662790916727A0916827B09162
:104E7000692780934A2790934B27A0934C27B093A0
:104E80004D2781E080934E2780936E27109249270B
:104E90002BC160914A2770914B2780914C279091AC
:104EA0004D2700916227109163272091642730914C
:104EB0006527061717072807390708F498C0011552
:104EC00011052105310509F492C06B017C014CE00C
:104ED000C40ED11CE11CF11C0C151D052E053F054F
:104EE00038F080EC90E0809347279093482719C0D2
:104EF0000F5F1F4F2F4F3F4F68017901C61AD70A26
:104F0000E80AF90AD701C60182959295907F982701
:104F1000807F9827809347279093482781E080934C
:104F20006B27209147273091482780914A279091FD
:104F30004B27A0914C27B0914D27880F991FAA1F8E
:104F4000BB1F880F991FAA1FBB1FBC01CD01660F95
:104F5000771F881F991F660F771F881F991F47E8C3
:104F600056E20E94EC348823A9F160914A2770919F
:104F70004B2780914C2790914D2744E00E9413517C
:104F8000609383267093842680938526909386264B
:104F90002091472730914827329522952F7023275B
:104FA0003F70232780914A2790914B27A0914C274F
:104FB000B0914D27820F931FA11DB11D80934A27E9
:104FC00090934B27A0934C27B0934D2782E080937A
:104FD0004E278AC08091492791E0980F90934927E6
:104FE0008B3008F481C085E080934E277DC044E07B
:104FF0000E941351609383267093842680938526A4
:1050000090938626109247271092482781E080933C
:105010006B2782E080934E2767C089E08A838FEFF9
:105020008B83809161278C83809160278983809115
:105030006B27813059F4E3E8F6E280819181A28107
:10504000B381806880839183A283B3834091472793
:10505000509148274C5F5F4F63E876E2CE0101969E
:105060000E94DA1288E080936D2783E080934E27B8
:105070003BC0809160270E940057813071F480917D
:105080006B27813031F410926B2784E080934E2798
:105090002BC081E080934E2727C080916D2781111E
:1050A00023C06EE577E081E00E944B1F85E080938E
:1050B0004E271AC044E050E06AE477E283E39DE0C3
:1050C000FADB69E477E081E00E944B1F10924E27E3
:1050D00010926E2709C065E377E081E00E944B1FC4
:1050E00010924E2710926E27CA5FDE4FCDBFDEBFF3
:1050F000DF91CF911F910F91FF90EF90DF90CF90B4
:105100000895EF92FF920F931F93CF93DF9300D0F8
:105110001F92CDB7DEB78C017B018091542781119E
:1051200040C044E050E0BE016F5F7F4F83E39EE0EC
:105130009ADB89819A81AB81BC81880F991FAA1F54
:10514000BB1F880F991FAA1FBB1F880F991FAA1F7B
:10515000BB1F880F991FAA1FBB1FBC01CD01607F19
:1051600099279701A8010E9438358130E1F489819F
:105170009A81AB81BC810196A11DB11D89839A835F
:10518000AB83BC8344E050E0BE016F5F7F4F83E39D
:105190009EE091DB6BEE76E081E00E944B1F81E0A8
:1051A00003C080E001C080E02496CDBFDEBFDF9168
:1051B000CF911F910F91FF90EF90089591E0909300
:1051C000542780935227609351270C9424350895D7
:1051D00060E170E096CF0895DF92EF92FF920F9317
:1051E0001F93CF93DF93CDB7DEB76097CDBFDEBF00
:1051F000D82E7B018A01FE01319680E1DF011D92EC
:105200008A95E9F7CF01DDD669817A818B819C810E
:1052100044E00E94135169837A838B839C83DD82EF
:105220000115110559F0A8010C30110510F04BE0E3
:1052300050E0B701CE0106960E942F6460E170E055
:10524000CE0101965EDF6096CDBFDEBFDF91CF91CC
:105250001F910F91FF90EF90DF900895CF93DF9310
:1052600000D0CDB7DEB780E00E94CA1120E030E068
:1052700040E251E40E9427630E946D6242E00E9476
:10528000135169837A8382E00E94D2110E9468627E
:105290006B8343E050E0BE016F5F7F4F83E09CDF94
:1052A0002396CDBFDEBFDF91CF910895CF92DF92DD
:1052B000EF920F931F93CF93DF936A01E9019091CF
:1052C0006E279111B4C0843008F0B3C09091542778
:1052D0009111B1C091E090936C2780936A2700935D
:1052E0006127E0926027813089F138F0823009F43B
:1052F00055C0833009F47DC0A0C01092662710927B
:105300006727109268271092692744E050E062E610
:1053100077E283E39EE0A7DA80916227909163278A
:10532000A0916427B09165270097A105B10509F404
:1053300086C00197A109B1098093622790936327E2
:10534000A0936427B093652781E082C044E050E0D9
:1053500066E677E283E39DE086DA44E050E062E6C9
:1053600077E283E39EE07FDA809162279091632762
:10537000A0916427B09165270097A105B10509F4B4
:1053800060C00197A109B1098093622790936327B8
:10539000A0936427B093652781E05AC0672B09F476
:1053A00052C01092662710926727109268271092B9
:1053B000692744E050E062E677E283E39EE053DA57
:1053C0008091622790916327A0916427B09165270F
:1053D0000097A105B105C9F10197A109B109809311
:1053E000622790936327A0936427B093652781E099
:1053F0002FC06115710559F1FB01808190E0A0E09B
:10540000B0E08093662790936727A0936827B093B6
:105410006927848190E0A0E0B0E0809362279093B8
:105420006327A0936427B093652781E011C080E0D3
:105430000FC080E00DC080E00BC080E009C081E0BB
:1054400007C081E005C080E003C081E001C080E0CA
:10545000009166271091672720916827309169276E
:10546000F601008311832283338340916227509198
:1054700063276091642770916527488359836A8305
:105480007B83DF91CF911F910F91EF90DF90CF90B1
:10549000089580916E27813019F480936B270895C9
:1054A00080E0089590916E2791110EC0909154273D
:1054B00091110AC090915F27911106C091E09093DD
:1054C0005F27817080935D27089580915F270895FD
:1054D00080916E27813059F080915427813049F0B6
:1054E00081E090915F27913029F080E0089581E07C
:1054F000089581E00895CF93DF9300D01F92CDB738
:10550000DEB790915027992301F190916F2799234D
:1055100011F08823E1F044E050E0BE016F5F7F4F5F
:1055200083E39EE0A0D944E050E0BE016F5F7F4F6F
:1055300083E39CE0C0D940E050E060E070E086E1A9
:105540004BDE1092502781E003C080E001C080E074
:105550002496CDBFDEBFDF91CF910895CF92DF9229
:10556000EF92FF920F931F93CF93DF93CDB7DEB7E8
:10557000C650D140CDBFDEBF80916F2790E088300C
:10558000910508F093C1FC01E156FE4F0C94EA63CB
:1055900080915F27813009F089C110925E2782E0F7
:1055A00080936F2783C181E0A6DF882321F082E00A
:1055B00080936F277BC183E080936F2777C144E09E
:1055C00050E069E577E283E39CE04DD944E050E0A8
:1055D00065E577E283E39EE046D980915527909177
:1055E0005627A0915727B09158270097A105B105DC
:1055F000B9F00197A109B1098093552790935627D7
:10560000A0935727B093582720915D27213041F46C
:105610008093592790935A27A0935B27B0935C27D8
:105620008091592790915A27A0915B27B0915C27D0
:1056300080937F2690938026A0938126B093822624
:1056400083E080936F2732C160917F26709180261E
:10565000809181269091822600915527109156279E
:105660002091572730915827061717072807390721
:1056700008F498C0011511052105310509F492C0FF
:105680006B017C014CE0C40ED11CE11CF11C0C151B
:105690001D052E053F0538F080EC90E080937D26B7
:1056A00090937E2619C00F5F1F4F2F4F3F4F680109
:1056B0007901C61AD70AE80AF90AD701C601829504
:1056C0009295907F9827807F982780937D2690934E
:1056D0007E2681E080935E2720917D2630917E2674
:1056E00080917F2690918026A0918126B09182267C
:1056F000880F991FAA1FBB1F880F991FAA1FBB1FC6
:10570000BC01CD01660F771F881F991F660F771F99
:10571000881F991F4DEB55E20E94EC348823A9F1B4
:1057200060917F26709180268091812690918226BB
:1057300044E00E9413516093B9257093BA25809379
:10574000BB259093BC2520917D2630917E263295F5
:1057500022952F7023273F70232780917F269091D9
:105760008026A0918126B0918226820F931FA11DD1
:10577000B11D80937F2690938026A0938126B093BD
:10578000822684E080936F2791C08091B82591E0B4
:10579000980F9093B8258B3008F488C087E08093E9
:1057A0006F2784C044E00E9413516093B925709321
:1057B000BA258093BB259093BC2510927D2610922C
:1057C0007E2681E080935E2784E080936F276EC001
:1057D00081E08A838DEF8B831C8280915E278130EC
:1057E00059F4E9EBF5E280819181A281B38180686F
:1057F00080839183A283B38300917D2610917E26BE
:10580000A8016DEB75E2CE0105960E942F64B801E8
:105810006D5F7F4FCE01029610D2882309F446C0F7
:1058200085E080936F2742C00E9489408230D9F47E
:105830000E94954F80915D27811107C044E050E0A0
:105840006FE776E283E39CE036D880915E27813073
:1058500031F410925E2786E080936F2727C081E0A5
:1058600080936F2723C00E9489408330F9F40E94FF
:10587000954F80915E27813011F410925E2786E06B
:1058800080936F2713C06CE177E081E00E944B1F8B
:1058900010926F2710925F2709C064E077E081E0E3
:1058A0000E944B1F10926F2710925F2780E023DE2B
:1058B000CA5FDE4FCDBFDEBFDF91CF911F910F9149
:1058C000FF90EF90DF90CF90089529DA9FDA46CECF
:1058D0000895CF93DF931F92CDB7DEB7898381E020
:1058E0008093502741E050E0BE016F5F7F4F85E11C
:1058F00073DC80E000DE0F90DF91CF91089580E2AD
:10590000E0E8F6E082830895E0E8F6E0808585FB34
:10591000882780F90895E091702781E1E89FF001E0
:105920001124E050F04E648175818681978108953D
:10593000E091702781E1E89FF0011124E050F04EE2
:10594000828593850895E091702781E1E89FF001B9
:105950001124E050F04E84850895E091702781E194
:10596000E89FF0011124E050F04E8785908908955A
:10597000E091702781E1E89FF0011124E050F04EA2
:1059800085850895CF93DF93D3D8E0E0F0E2ACE0D3
:10599000B0E2CAEAD0E24CE251E060E070E021E01F
:1059A00030E0108211821282138244835583668311
:1059B000778322873387108611862787308B258748
:1059C0003687813011F494E001C091E09C93719688
:1059D0005196EC17FD0729F781E0DF91CF910895EB
:1059E0008A3060F421E1829FC001112441E150E03E
:1059F0008F579F4F0E94B85381E0089580E008952B
:105A0000CF93DF931F92CDB7DEB789834AEA50E088
:105A100060E070E281E890E00E94C55341E050E010
:105A2000BE016F5F7F4F87E0D7DB81E00F90DF9192
:105A3000CF910895FB018A30B8F540815181628190
:105A4000738191E1899FD0011124A050B04E4D93F4
:105A50005D936D937C931397448155816681778123
:105A600014964D935D936D937C93179782859385E0
:105A70001A968D939C931B978085918518968D938C
:105A80009C93199784851C968C931C978785908985
:105A90001F968D939C935097858596851D968D9323
:105AA0009C931E9781E0089580E00895CF92DF9245
:105AB000EF92FF92CF93DF93EC013AD8E82FCC809E
:105AC000DD80EE80FF80B701A601485751096109CA
:105AD00071094938524A6240710570F5AF85B8893D
:105AE000109779F0A70196010E94FF63AB01BC01FA
:105AF00048575109610971094938524A6240710594
:105B0000E8F4AA85BB85A70196010E94FF63DC012A
:105B1000CB0188579109A109B1098938924AA2405D
:105B2000B10570F49C85963068F4E13069F481E049
:105B3000913059F480E009C080E007C080E005C0E2
:105B400080E003C080E001C081E0DF91CF91FF9051
:105B5000EF90DF90CF9008950F931F93CF93DF9333
:105B60004AEA50E060E070E281E890E00E94B853B9
:105B7000C0E0D0E20AEA10E2CE0198DF882329F0E3
:105B80006196C017D107C1F702C080E001C081E073
:105B9000DF91CF911F910F910895E091702721E13E
:105BA000E29FF0011124E050F04E21E1DC01019070
:105BB0000D922A95E1F708958091702708958091BC
:105BC00071270895CF93DF9380917627813049F034
:105BD000EDECF8E281E090E0EC012081213021F54C
:105BE00002C0C0E0D0E027E531E0C29FC001C39F02
:105BF000900DD29F900D1124FC01E553F74D60816B
:105C000071818958984D0E948C40813099F487E5C4
:105C100091E0C89FF001C99FF00DD89FF00D1124AD
:105C2000EA58F84D108206C00196E95AFE4F8530B9
:105C3000910591F6DF91CF910895CF92DF92EF9287
:105C4000FF920F931F93CF93DF937C01EB01653598
:105C500081E07807B8F580917627882349F0EDEC4C
:105C6000F8E221E030E089018081811123C002C087
:105C700000E010E066EA77E081E00E944B1F87E5D4
:105C800091E0089F6001099FD00C189FD00C11244F
:105C9000AE01B701C6018958984D0E942F64F601E4
:105CA000EA58F84DDF01AB5ABE4FCD93DC9381E04B
:105CB00080830BC02F5F3F4FE95AFE4F25303105DF
:105CC00091F602C080E001C080E0DF91CF911F918A
:105CD0000F91FF90EF90DF90CF900895E6E7F7E205
:105CE00029E23EE280E09081913009F48F5FE95A29
:105CF000FE4FE217F307B9F70895E82F8230C1F499
:105D0000862F8370A9F489E2689F812D11248295E2
:105D10008F70962F24E6829F9019112491110DC047
:105D2000862F90E060E971E00E949963892B39F039
:105D3000F0E0E754FC4D808108958DE108958DE1F8
:105D400008958091292E0895BF92CF92DF92EF920D
:105D5000FF920F931F93CF93DF93B82EEB017A013D
:105D6000690160E080E00E94803F8823F1F080E2DA
:105D7000E0E6F6E085838B2D0E94B43FB701CE01AB
:105D80000E94F33F813049F4B801C6010E94CD3F23
:105D9000C1E0813019F0C0E001C0C0E080E2E0E67F
:105DA000F6E086830E94723F01C0C0E08C2FDF9135
:105DB000CF911F910F91FF90EF90DF90CF90BF9008
:105DC00008950F931F9300E110E02AE23EE240E0C5
:105DD00050E060E070E080E9B7DF91E0813009F0E9
:105DE00090E0892F1F910F9108950F931F93CF93E8
:105DF000DF93CDB7DEB72797CDBFDEBF8C01FC01A7
:105E000080810E94EE508983F80181810E94EE50CA
:105E10008A83F80182810E94EE508B83F80183818E
:105E20000E94EE508C831D82F80184810E94EE5006
:105E30008E83F8018581805D0E94EE508F8300E0A3
:105E400010E020E030E047E050E0BE016F5F7F4FA0
:105E500082E17ADF813039F46EED77E083E00E94F1
:105E60004B1F81E001C080E02796CDBFDEBFDF91F0
:105E7000CF911F910F910895CF92DF92EF92FF92F1
:105E8000CF93DF93EC01FB01ED80FE80A701405D25
:105E900057405695479556954795B7016C5B7740A7
:105EA0002DE631E0629FC001639F900D729F900DBF
:105EB0001124480F591F6A0166E0C60ED11CC701A4
:105EC00083709927892B99F59701369527953695F3
:105ED0002795ABE7B4E10E94F0639695879564E659
:105EE000689F9001699F300D1124E216F306C1F4FA
:105EF0009701329522952F7023273F702327AEE319
:105F0000BAE00E94F06320E931E0BC01629FC00169
:105F1000639F900D729F900D1124E816F90639F4D5
:105F20008C81833020F46A0175E0C70ED11C4B814F
:105F300050E0415051094C0D5D1D2C8130E0215045
:105F40003109121613067CF480E090E060E0DC0179
:105F5000A654BC4D8C91480F511D6F5F862F90E069
:105F600082179307A4F32A8130E0A0E1BEE00E94EB
:105F7000F0636B017C01298130E0ACE3B0E00E946A
:105F8000F063C60ED71EE81EF91E8881C80ED11C0C
:105F9000E11CF11CDA01159720E831E541E050E001
:105FA0000E94FF63C60ED71EE81EF91EC082D18272
:105FB000E282F382DF91CF91FF90EF90DF90CF905C
:105FC00008950F931F93CF93DF93CDB7DEB7279735
:105FD000CDBFDEBF8C01F5DE813049F580912C2EDE
:105FE0008F770E94E350898380912D2E8F770E94B6
:105FF000E3508A8380912E2E0E94E3508B83809100
:106000002F2E0E94E3508C838091312E0E94E3500A
:106010008D838091322E0E94E35090E08053984F00
:106020008E839F83B801CE01019626DF05C0F8015B
:1060300010821182128213822796CDBFDEBFDF91BC
:10604000CF911F910F9108956F927F928F929F929F
:10605000AF92BF92CF92DF92EF92FF920F931F9376
:10606000CF93DF93EB01FC01608171818281938189
:1060700020E831E541E050E00E94AC634B015C0157
:106080008CEB97E08D839E8381E08C8369017A019C
:10609000F5E0CF0ED11CE11CF11C772473940FC0E6
:1060A000C41AD50AE60AF70A81E0860D8D3010F48D
:1060B0008C8305C07C820F5F1F4F0D831E830D8173
:1060C0001E816C80602F862D18DE482F50E060E026
:1060D00070E04C155D056E057F0510F3CB82C501A0
:1060E000B40120E13EE040E050E00E94AC632A832E
:1060F0000F2EFCE3CF2ED12CE12CF12CF02DC5017D
:10610000B401A70196010E94AC63162FCA01B90120
:10611000A70196010E94AC6369831883DF91CF9138
:106120001F910F91FF90EF90DF90CF90BF90AF90B5
:106130009F908F907F906F900895CF92DF92EF9213
:10614000FF920F931F93CF93DF93CDB7DEB7639783
:10615000CDBFDEBF8B0120E829832A832B832C83CC
:10616000FB01C080D180E280F380FC01408151813D
:10617000628173814C155D056E057F0508F090C046
:10618000C41AD50AE60AF70ABE016A5F7F4F5CDFD0
:10619000BE01635F7F4FC80157DFF0E1CF16FEE01D
:1061A000DF06E104F10458F48E850E94EE508D83E1
:1061B000898369E778E081E00E944B1F51C080E845
:1061C000C81681E5D80681E0E806F10480F48F85E1
:1061D0000E94EE508D838A838E850E94EE508D83BF
:1061E00089836FE578E081E00E944B1F39C0C114BC
:1061F000E3EADE06E2E0EE06F104A8F488890E94F4
:10620000EE508D838B838F850E94EE508D838A8321
:106210008E850E94EE508D8389836FE378E081E064
:106220000E944B1F1DC01985612F8A8566DD412F95
:1062300050E04E5F5F4F282F30E02417350724F4DD
:106240001E5F181B1D8302C01E5F1D838D810E946F
:10625000EE508D838B836CE178E081E00E944B1FD0
:1062600000E010E020E030E044E050E0BE016F5F6D
:106270007F4F89E169DD8130A9F482E08D8320E0E0
:1062800030E041E050E0BE016B5F7F4F81E15CDDBB
:10629000813051F462E078E00E944B1F81E005C03C
:1062A00080E003C080E001C080E06396CDBFDEBF28
:1062B000DF91CF911F910F91FF90EF90DF90CF90E2
:1062C0000895EF92FF920F931F93CF93DF93CDB773
:1062D000DEB72897CDBFDEBF74DD6EEC77E081E0DE
:1062E0000E944B1F0AE21EE20F2EFAE3EF2EFEE29F
:1062F000FF2EF02DF80161918F0170E0CE01019623
:106300000E941C50BE016F5F7F4F81E00E94211FE1
:106310006CEC77E081E00E944B1F0E151F0551F7D2
:1063200069EC77E081E00E944B1F2896CDBFDEBF6D
:10633000DF91CF911F910F91FF90EF9008950F93F0
:106340001F93CF93DF93CDB7DEB72997CDBFDEBFC5
:1063500087E0E7E6F3E2DE01129601900D928A955E
:10636000E1F7E0E6F6E080E28683818381E08093D6
:10637000292E27DD813069F48091382E833711F47E
:106380001092292E80912C2E88231CF481E080937A
:10639000292E97DF8091292E8823B9F0CE0102960D
:1063A00024DD83E7898700E010E020E030E041E071
:1063B00050E0BE01675F7F4F8EE1C6DC813029F47B
:1063C0006CEE77E082E00E944B1F198200E010E043
:1063D00020E030E041E050E0BE016F5F7F4F81E19F
:1063E000B3DC2996CDBFDEBFDF91CF911F910F9116
:1063F0000895EEE3FEE286E69EE2DF0114971D9229
:106400001D921D921C92139710823596E817F9077A
:10641000A1F781E00895883080F490E09C01220F7C
:10642000331F220F331F820F931F45E050E0855D1D
:106430009E4F0E94B85381E0089580E0089548E29D
:1064400050E06AE37EE28BE291E00E94C55381E076
:106450000895FB018830C0F490E040815181628151
:106460007381DC01AA0FBB1FAA0FBB1FA80FB91FA6
:10647000A65CB14D4D935D936D937C93139784818E
:1064800014968C9381E0089580E00895FC01948136
:106490009A5081E0953F08F480E008950F931F9390
:1064A000CF93DF9348E250E06AE37EE28BE291E033
:1064B0000E94B853CAE3DEE202E61EE2CE01E6DF46
:1064C000882329F02596C017D107C1F702C080E0C4
:1064D00001C081E0DF91CF911F910F910895CF937B
:1064E000DF93EC0169DB282F30E0F901EE0FFF1F8D
:1064F000EE0FFF1F2E0F3F1FF901E65CF14D85E007
:10650000DE0101900D928A95E1F7DF91CF91089518
:10651000E0E4F6E080E18183858381E08093973138
:10652000089540E05BE460E070E080E00E94375551
:1065300080E00E94CE54ECDF88E991E30C94176070
:106540000895809197310895CF93DF931F92CDB72F
:10655000DEB780E00E947C56892BF1F041E050E0EC
:10656000BE016F5F7F4F80E00E94C85581111CC043
:1065700083E080939831698187E79FE20E94061C3F
:10658000813091F460E08FE79FE20E94F21D87E77F
:106590009FE20E94D71208C080919831813021F487
:1065A00087E79FE20E94D7120F90DF91CF91089565
:1065B000E0E2F6E081E081838683109293311092CD
:1065C00094311092953186E991E30E94176084E935
:1065D00091E30C944360089581E080939331089592
:1065E000809193310895CF92DF92EF92FF920F93B3
:1065F0001F93CF93DF931F92CDB7DEB78091762F95
:10660000813019F130F08230E9F1833009F4F5C0BE
:1066100040C180919331813009F03BC111E0E0E24B
:10662000F6E0158340E855E260E070E083E00E9408
:10663000375583E00E94CE5484E090E080939431FB
:10664000909395311093762F24C18091943190913D
:106650009531892B09F01DC147E050E062EB70E2F3
:1066600083E00E94C15868EB78E081E00E944B1FF4
:1066700084E090E0809394319093953182E0809310
:10668000762F07C18091943190919531892B09F033
:1066900000C148E750E06BE970E380E09FE00E94B2
:1066A000B85301E910E387E0ECE0F1E3D801019091
:1066B0000D928A95E1F71092983083E191E30E9460
:1066C0008625D8010D900020E9F711979D012159E9
:1066D00030430F2EF3E1CF2EF1E3DF2EF02DD60164
:1066E0000D900020E9F71197A351B1430F2EFCEA5A
:1066F000EF2EF0E2FF2EF02DF70101900020E9F7D8
:106700003197CF018C5A9042A20F8A0F92E0980FD6
:1067100090938E3093E0980F90938C3010928D3040
:1067200092E590938F3094E090939030875A8093C5
:106730008B3041E050E061EB70E283E00E94C15891
:1067400042E050E06FE870E383E00E94C15842E00D
:1067500050E06CE870E383E00E94C15841E050E0F3
:106760006BE870E383E00E94C15841E050E06EE8BE
:1067700070E383E00E94C158F60101900020E9F720
:106780003197AF0143515143B60183E00E94C15894
:10679000D7010D900020E9F71197AD014C5A5042F6
:1067A000B70183E00E94C158F80101900020E9F789
:1067B0003197AF0141595043B80183E00E94C1585D
:1067C00042E050E06AEA70E283E00E94C15841E092
:1067D00050E06FEA70E283E00E94C15862EA78E01C
:1067E00081E00E944B1F80E699E080939431909362
:1067F000953183E08093762F4CC0809194319091B5
:106800009531892B19F41092933104C08091933102
:1068100081110EC081E0E0E2F6E0868383E00E9411
:106820007B546CE878E081E00E944B1F1092762F39
:1068300083E00E947C56892B21F141E050E0BE01AB
:106840006F5F7F4F83E00E94C855811122C083E0B3
:1068500080939631698182E69EE20E94061C813017
:10686000C1F463E08AE69EE20E94F21D82E69EE2A7
:106870000E94D71280E699E08093943190939531ED
:1068800008C080919631813021F482E69EE20E9418
:10689000D7120F90DF91CF911F910F91FF90EF9042
:1068A000DF90CF900895DA01611116C04C911196D6
:1068B000EC911197F0E0E827FF27EE0FFF1FE3535D
:1068C000F74F2591349180E090E0942F8227932711
:1068D0008D939C93119705C08FEF9FEF8D939C93A1
:1068E00011978D919C910895CF92DF92EF92FF9234
:1068F0000F931F93CF93DF931F921F92CDB7DEB7F5
:106900006C017B01AE014F5F5F4F61E08FEFCBDF2A
:10691000E114F10471F08601EC0CFD1CAE014F5F37
:106920005F4F60E0F80181918F01BDDF0E151F05FB
:10693000A9F789819A810F900F90DF91CF911F91D4
:106940000F91FF90EF90DF90CF900895E0E6F6E092
:1069500082E0868381E0858383E081830895BF920E
:10696000CF92DF92EF92FF920F931F93CF93DF931B
:10697000B82EEB017A01690160E080E00E94803F5F
:106980008823F1F081E0E0E6F6E086838B2D0E941B
:10699000B43FB701CE010E94F33F813049F4B80102
:1069A000C6010E94CD3FC1E0813019F0C0E001C0B6
:1069B000C0E081E0E0E6F6E085830E94723F01C01E
:1069C000C0E08C2FDF91CF911F910F91FF90EF903E
:1069D000DF90CF90BF9008950F931F93CF93DF93D5
:1069E00000D0CDB7DEB789837A836B8389019A01A2
:1069F00043E050E0BE016F5F7F4F83E0B0DF23963E
:106A0000CDBFDEBFDF91CF911F910F9108950F93FE
:106A10001F9300E010E020E030E041E050E0BC01D6
:106A200085E09DDF1F910F9108950F931F9300E064
:106A300010E020E030E040E050E060E070E086E010
:106A40008EDF1F910F9108950F931F93EEDF81301A
:106A500059F400E010E020E030E040E050E060E079
:106A600070E087EC7CDF01C080E01F910F910895FA
:106A70000F931F93CF93DF93CDB7DEB7A397CDBF0F
:106A8000DEBFFA01890121323105C8F489837A8396
:106A90006B83A901BF01CE0104960E942F64C5DF5C
:106AA000813079F4A8014D5F5F4F00E010E020E0F5
:106AB00030E0BE016F5F7F4F82E051DF03C080E0B6
:106AC00001C080E0A396CDBFDEBFDF91CF911F91C3
:106AD0000F9108950F931F93653150F4062F10E026
:106AE0009C0140E050E060E070E08FE938DF01C0D9
:106AF00080E01F910F910895CF93DF93CDB7DEB75C
:106B00006597CDBFDEBF22DFCE01019680DF8130E9
:106B1000B9F464E1CE010296DDDF813089F48A8127
:106B2000803249F48B818B3B31F46DEE7AE081E069
:106B30000E944B1F05C06DEC7AE081E00E944B1F64
:106B40006596CDBFDEBFDF91CF910895CF93DF93E0
:106B50008091F13290E0A0E0B0E0BA2FA92F982FF9
:106B600088272091F232822B8093A3319093A43115
:106B70002091F3328091F43290E0A0E0B0E0DC01AB
:106B800099278827B22B2091F632822B2091F5325B
:106B9000922B8093A5319093A631A093A731B09307
:106BA000A8318091F7328093A931882309F441C03C
:106BB000CCEAD1E36CEF72E3982F990F890F382F4D
:106BC000330F330F830F35E1380F25E1DB011497C5
:106BD0008C91DE0112978C93DB0113978C91DE016F
:106BE00011978C93DB0112978C91888311968C916D
:106BF00090E0A0E0B0E0BA2FA92F982F882746EFA9
:106C0000420FFB015081852B89839A83522FDE012D
:106C100013964F5F842F90E08F509D4CFC01808134
:106C20008D934513F6CF215F2F96615F7F4F23131E
:106C3000CDCFDF91CF910895CF92DF92EF92FF9267
:106C40008091F33290E0A0E0B0E0BA2FA92F982F06
:106C500088272091F4322770822B809360328450F1
:106C6000833030F481E080935E3210925F3234C022
:106C70008091F6339091F733892B59F468E47DE0E5
:106C800081E00E944B1F81E080935E3280935F32EF
:106C900023C062E47DE082E00E944B1F8091F633C6
:106CA0009091F73340EB54E060E070E0481B590BE3
:106CB000610971097695679557954795769567951A
:106CC0005795479582E00E946D1F69E37DE082E061
:106CD0000E944B1F10925E322091F7328091F83261
:106CE00090E0A0E0B0E0DC0199278827B22B20914A
:106CF000FA32822B2091F932922B80936332909357
:106D00006432A0936532B09366328091FB3290E09A
:106D1000A0E0B0E0BA2FA92F982F88272091FC324D
:106D2000822B80936732909368328091FD328093FA
:106D300069328091FE3280936A328091FF32809373
:106D40006B328091003380936C328091013390E0FC
:106D5000A0E0B0E0BA2FA92F982F88272091023306
:106D6000822B80936D3290936E3220910733809105
:106D7000083390E0A0E0B0E0DC0199278827B22B2F
:106D800020910A33822B20910933922B80936F320A
:106D900090937032A0937132B093723220910B3382
:106DA00080910C3390E0A0E0B0E0DC0199278827C7
:106DB000B22B20910E33822B20910D33922B809396
:106DC000733290937432A0937532B093763260919F
:106DD0001833862F90E0A0E0B0E0BA2FA92F982FAB
:106DE000882720911933BC01CD01622B0F2EF4E6C8
:106DF000CF2ED12CE12CF12CF02DA70196010E9471
:106E0000AC632093773230937832209122336091B3
:106E10002333862F90E0A0E0B0E0DC01992788279B
:106E2000B22B20912533822B20912433BC01CD013C
:106E3000722BA70196010E94AC63209379323093A4
:106E40007A3240937B3250937C32233331054105B3
:106E5000510540F08091F6339091F733899710F007
:106E600010925E32209126338091273390E0A0E08B
:106E7000B0E0DC0199278827B22B20912933822B9F
:106E800020912833922B80937D3290937E32A09371
:106E90007F32B093803220914833822B80938132AD
:106EA00020914933822B8093823281E08093F032AB
:106EB00080915E328130F9F42091F6333091F733CE
:106EC00080EB94E0A0E0B0E0821B930BA109B10934
:106ED000B695A79597958795B695A7959795879514
:106EE0000196809361329093623280EB94E08093BC
:106EF000F6339093F733FF90EF90DF90CF900895A3
:106F000081E080938432109283321092853208950A
:106F100088E08093833208958091833281110FC07D
:106F200080918432811105C0EBDF81E0809385324E
:106F3000089581E08093853282E0809383320895C2
:106F400081E090918332911101C080E00895662321
:106F500051F0613031F42091F032213071F080E055
:106F6000089580E0089525E2EEE5F2E3DC0101906A
:106F70000D922A95E1F781E0089525E2EEE5F2E32E
:106F8000DC0101900D922A95E1F71092F03281E038
:106F900008952CE6E3E8F2E3DC0101900D922A95D6
:106FA000E1F70895EF92FF920F931F93CF93DF9332
:106FB00000D0CDB7DEB78C010E9426647C0100971B
:106FC00069F0F801D801A80FB91F60E070E0849162
:106FD00068273196EA17FB07D1F702C060E070E03E
:106FE000CE0101960E941C5041E050E06AE57BE032
:106FF00082E00E94AF59A701B80182E00E94AF5918
:1070000041E050E068E57BE082E00E94AF5943E058
:1070100050E0BE016F5F7F4F82E00E94C15842E0A6
:1070200050E065E57BE082E00E94AF592396CDBF3A
:10703000DEBFDF91CF911F910F91FF90EF900895E8
:10704000EF92FF920F931F93CF93DF93CDB7DEB7ED
:107050002897CDBFDEBF8C0119821A82FC01859171
:1070600094918B839C8342E0BE016D5F7F4FCE0184
:1070700001960E9432501D821E821F8218868981CD
:107080009A810097A1F040E050E020E030E0B801A4
:107090006E5F7F4FFB01E20FF31FE4914E0F511D16
:1070A0002F5F3F4F28173907A8F34F83588742E0D7
:1070B000BE01695F7F4FCE0105960E94325042E0CB
:1070C00050E062E57BE082E00E94AF5949815A813D
:1070D0004E5F5F4FB80182E00E94AF5942E050E03E
:1070E000BE016B5F7F4F82E00E94C15842E050E0DA
:1070F0006FE47BE082E00E94AF592896CDBFDEBFEF
:10710000DF91CF911F910F91FF90EF9008958091A3
:107110009F318230B9F128F4882359F08130C9F0C9
:1071200066C0843009F44DC0C0F1853009F452C006
:107130005EC08EEF9EE084DF80EE91E08093F233BC
:107140009093F33381E080939F3161EF7CE00E9464
:107150004B1F82E00E940057882349F084E190E0B1
:107160008093F2339093F33382E080939F31809148
:10717000F2339091F333892BF1F586E080939F31C0
:1071800080E008958091F2339091F333892BA9F533
:1071900083E080939F3180E0089580E2E0EAF6E0AA
:1071A0008683E0E0F6E0868388E28093F93384E02A
:1071B00080939F316DED7CE081E00E944B1F80E069
:1071C00008958091F93381111AC085E080939F3131
:1071D00080E00895109284321092853210929F318F
:1071E00064EC7CE081E00E944B1F81E008951092E6
:1071F0009F3182E0089580E0089580E0089580E066
:1072000008958091A1318130A1F018F0823029F1E8
:107210005BC08091A0318F5F843620F48093A031D1
:1072200080E008951092A03181E08093A13180E048
:1072300008951092152110921B2110921E21109278
:107240001F2182E09FE0FCDE80EE91E08093F2332C
:107250009093F33382E08093A13180911B218823A6
:1072600041F16DE07DE081E00E944B1F40911C21C7
:1072700050911D214150510961EF72E38EE992E373
:107280000E942F6487E1E6ECF3E2A8E8B2E3019004
:107290000D928A95E1F71092873248E650E067E850
:1072A00072E388E79FE00E94C5531092A13181E00C
:1072B00008958091F2339091F333892B49F481E062
:1072C0008093A13180E008951092A13182E0089569
:1072D00080E00895CF93DF93EC01A62F488150E022
:1072E000FA013197E830F10520F4E955FE4F0C948E
:1072F000EA631E821D821F82188681E0888389814D
:10730000813081F58D816C81861750F52A813B8112
:10731000F901E80FF11DE491EA1320C08F5F8D831E
:107320006813F9C01B861C8619861A8670E06115E1
:10733000710579F040E050E080E090E0F901E80F5D
:10734000F91FE4914E27019686179707B8F34B87EC
:107350005C8719861A8682E08883DDC01882DBC0CC
:107360001882D9C0823089F58D819C81891758F5A2
:10737000EA81FB81E80FF11DE491AE1729F082301C
:1073800029F08330F1F409C0823029F41F82A887E4
:1073900083E08D83C0C0833041F48F8198858A2B30
:1073A0008F83988784E08D83B6C08F5F8D83981319
:1073B000B2C0B0E0AB87BC8719861A8683E08883A9
:1073C000AAC01882A8C01882A6C01882A4C0AA3277
:1073D000A9F089859A858F3F910509F048F4FC0151
:1073E000EF50FD4CA0838B859C858A278B879C87DB
:1073F00089859A85019689879A878DC06B857C855A
:107400000B960E941C5089859A8501968F839887D8
:1074100084E0888380C089859A85AC014F5F5F4F87
:107420002F8138854217530798F48F3F910509F053
:1074300050F4FC01EF50FD4CA0838B859C858A0F96
:10744000911D8B879C8789859A85019689879A8764
:1074500029853A852F5F3F4F8F81988528173907F7
:1074600009F059C084E088838B859C859F778B8742
:107470009C8751C08981813021F4B0E0AD87BE87FF
:1074800004C0823011F41D86AE8785E0888343C036
:107490008981813031F48D859E859A2B8D879E87D9
:1074A00007C0823029F48D859E858A2B8D879E8723
:1074B00086E0888330C0AD3021F48981813049F481
:1074C00005C0A03B31F48981823019F487E08883BC
:1074D00022C018821E821FC0AA3021F48981813007
:1074E000C1F405C0A33BA9F48981823091F42B85B6
:1074F0003C858D859E852817390741F488E7809360
:10750000F83388E0888381E08E8305C018821E826C
:1075100002C018821E828E81DF91CF910895109251
:107520007E2110928421109287211092882110923E
:107530006F2110927521109278211092792110926A
:107540006021109266211092692110926A21109296
:1075500051211092572110925A2110925B211092C2
:1075600042211092482110924B2110924C211092EE
:1075700033211092392110923C2110923D2110921A
:10758000242110922A2110922D2110922E21109246
:10759000152110921B2110921E2110921F21109272
:1075A000062110920C2110920F211092102110929E
:1075B000CA201092D0201092D3201092D420109282
:1075C000BB201092C1201092C4201092C5200895B3
:1075D000E0EAF6E081E0828391859C7F916091876B
:1075E000108A82871092F13382E6818382E2868359
:1075F00080E486831092F9331092F8331092F233BC
:107600001092F3331092F4331092F5331092F63354
:107610001092F73389EF93E30E94176088EF93E3AA
:107620000E94176086EF93E30E94436082EF93E32A
:107630000E94436084EF93E30E9443601092833280
:1076400010928432109285321092EF32109286326C
:1076500048E650E067E872E388E79FE00E94B8538D
:107660001092F0325CCF08958091BA20823009F4F4
:1076700086C028F4882361F0813089F05BC18430B2
:1076800009F4C0C008F49BC0853009F4CEC052C1D3
:1076900010929E3181E08093BA2080E0089580911D
:1076A000842181110CC080917521811108C08091C5
:1076B0006621811104C0809157218823B9F08091FF
:1076C0009E31811113C081E080939E3182E08093CE
:1076D000BA2085E090E08093F2339093F33366EA2A
:1076E0007CE082E00E944B1F80E008958091392168
:1076F000811118C080911B21811114C080910C212F
:10770000811110C08091FD2081110CC08091EE206C
:10771000811108C08091DF20811104C08091D020A8
:107720008823E1F082E08093EF3284E08093BA20F6
:1077300085E090E08093F2339093F33369E87CE046
:1077400082E00E944B1F8AE19FE07ADC80E19FE0AB
:1077500077DC86E09FE074DC80E008958091F2336E
:107760009091F333892B09F0EFC068E57CE081E06C
:107770000E944B1F85E08093BA2080E0089580919D
:10778000F2339091F333892B09F0E0C065E27CE09D
:1077900082E00E944B1F88EE9EE004DC80E09BE4C8
:1077A000A0E0B0E080939A3190939B31A0939C31FC
:1077B000B0939D3183E08093BA2080E0089582E009
:1077C0000E940057882309F4C3C082E00E947B54C2
:1077D00040919A3150919B3160919C3170919D31D3
:1077E00082E00E94375582E00E94CE5480EE91E004
:1077F0008093F2339093F33381E08093BA208FDE4D
:1078000080E008958091F2339091F333892B09F051
:10781000A1C06DEF7BE082E00E944B1F84E29FE0FD
:107820000FDC1092BA2081E0089580919931813067
:10783000D9F030F0823069F1833009F43FC053C091
:1078400080E895E2A0E0B0E080939A3190939B317C
:10785000A0939C31B0939D3181E08093993161EE8A
:107860007BE00E944B1F52C080E09BE4A0E0B0E0B0
:1078700080939A3190939B31A0939C31B0939D312A
:1078800082E08093993164EC7BE081E00E944B1FA1
:107890003DC080E091EEA0E0B0E080939A319093FB
:1078A0009B31A0939C31B0939D3183E080939931BB
:1078B00067EA7BE081E00E944B1F28C080E699E0E8
:1078C000A0E0B0E080939A3190939B31A0939C31DB
:1078D000B0939D3184E0809399316BE87BE081E047
:1078E0000E944B1F13C080EC92E1A0E0B0E08093B7
:1078F0009A3190939B31A0939C31B0939D3110921B
:1079000099316FE67BE081E00E944B1F80919931B5
:10791000882351F080EE91E08093F2339093F3331B
:1079200083E08093BA2003C087E08093BA20F7DD1C
:1079300080E008956CE57BE081E00E944B1F81E0D0
:107940008093BA2082E0089580E0089580E0089551
:1079500080E0089580E008958091F1338F5F8093F7
:10796000F13308958823B9F080918632811122C0C5
:1079700081E08093863280E4E0EAF6E085836DE280
:107980007BE081E00E944B1F80E19EE08093F43316
:107990009093F5330FC080918632882359F010926E
:1079A000863280E4E0EAF6E086836EE07BE081E008
:1079B0000E944B1F81E008950F931F93CF93DF9395
:1079C000CDB7DEB76B97CDBFDEBFCE010F960E945D
:1079D000E12FBE016F5F7F4FCE010F960E942430D2
:1079E00080916032882309F49DC080916732909124
:1079F00068328D879E87809169328C8780916A3248
:107A00008B8780916B328A8780916C328987209135
:107A10006D3230916E32369527953695279536958D
:107A20002795A5ECB0E20E94F063929582958F7045
:107A300089279F7089278887BE016D5E7F4FCE01A1
:107A400008960E943C2F8B899C89AD89BE894F8501
:107A5000588969897A8984179507A607B70760F05E
:107A60008C019D01041B150B260B370B0B301105E8
:107A70002105310568F456C08A019B01081B190BCA
:107A80002A0B3B0B0B3011052105310508F44AC0C8
:107A90001F8A481759076A077B0728F4841B950B30
:107AA000A60BB70B08C08A019B01081B190B2A0BF8
:107AB0003B0BD901C801888F998FAA8FBB8F80910A
:107AC0006732909168328E839F83809169328D8373
:107AD00080916A328C8380916B328B8380916C327F
:107AE0008A8320916D3230916E3236952795369586
:107AF000279536952795A5ECB0E20E94F063929504
:107B000082958F7089279F7089278983CE0101967E
:107B10000E94F52E45E050E0BE01695E7F4F8FE088
:107B20000E94EC286B96CDBFDEBFDF91CF911F91F5
:107B30000F9108951F93CF93DF931F92CDB7DEB7B8
:107B40008091F4339091F533892B79F480918632CA
:107B5000882359F01092863280E4E0EAF6E08683CA
:107B600064E67EE081E00E944B1F8091833290E0CA
:107B70008930910508F0D0C0FC01E155FE4F0C940E
:107B8000EA6380918432882309F4D6C080E2E0EA77
:107B9000F6E08583E0E0F6E0858311E01093833220
:107BA00040EC52E160E070E082E00E94375582E0F4
:107BB0000E94CE541092EF32B2DC1092F133109347
:107BC000A23180EB94E08093F6339093F7331092D8
:107BD0005E321092A93160E57EE081E00E944B1F89
:107BE000ABC08091F133823008F4A6C08091853219
:107BF000882321F082E0809383329EC085E08093C9
:107C000083321092F6331092F73396C01092F1330C
:107C100082E0E0EAF6E0858385EB8150F1F782E0CF
:107C2000E0EAF6E0868383E08093833285C080912A
:107C3000F133882309F480C080918532882321F0B4
:107C400084E08093833278C085E08093833274C06F
:107C50008091A231813079F486E08093833280EE86
:107C600091E08093F2339093F3336BE37EE081E015
:107C70000E944B1F61C0809187328F3F49F487E09B
:107C8000809383326AE17EE081E00E944B1F54C002
:107C90008091F833811150C088E0809383326CED7D
:107CA0007DE081E00E944B1F47C081E080938532D8
:107CB00084E08093833280EB94E08093F63390935A
:107CC000F73360EB7DE081E00E944B1F35C099DA0D
:107CD000813069F562E97DE00E944B1F84E080936A
:107CE00083322AC0C1DC813011F564E77DE00E9457
:107CF0004B1F84E0809383321092A2311DC007DABB
:107D00008130A9F482E00E947B5410925E3210927E
:107D100083321092A93110C066E57DE081E00E94B7
:107D20004B1F82E00E947B541092833205C0823048
:107D300019F489E08093833282E00E947C56892B7B
:107D400009F46BC041E050E0BE016F5F7F4F82E0FD
:107D50000E94C855811161C08091EF32823031F5A7
:107D600069818AEC90E2B6DA882359F00E941C36C9
:107D70001092CA201092D0201092D3201092D420BA
:107D80001BDE698184E291E2A5DA882351F00E942A
:107D9000A6351092242110922A2110922D211092A2
:107DA0002E21698185E191E295DA37C0813069F44D
:107DB00069818FE691E28EDA698180E691E28ADA62
:107DC00069818EE791E286DA28C0698183E391E2D6
:107DD00081DA698184E291E27DDA698186E091E26B
:107DE00079DA69818AEC90E275DA69818BEB90E24D
:107DF00071DA69818EE791E26DDA69818FE691E24D
:107E000069DA698180E691E265DA698181E591E26A
:107E100061DA698182E491E25DDA0F90DF91CF91BE
:107E20001F9108952EE0E0EAF2E3DC0101900D924B
:107E30002A95E1F708952091A9312D3008F02CE022
:107E40002223E1F080EB91E321504FE0249F900149
:107E5000112421543E4C0AC05191511111C04F5F61
:107E60004A30D1F70F968217930761F0FC013197E2
:107E70004081411109C0FC0141E0EECF80E008954E
:107E800081E0089580E0089581E008951F920F92A7
:107E90000FB60F9211240BB60F922F933F934F936F
:107EA0005F936F937F938F939F93AF93BF93EF9362
:107EB000FF9352DDFF91EF91BF91AF919F918F9111
:107EC0007F916F915F914F913F912F910F900BBEDA
:107ED0000F900FBE0F901F9018958AEF93E30C94AC
:107EE000176008951092C008E0E7F0E08381886091
:107EF000838308958091C00886FB882780F90895C0
:107F0000823031F0833031F0813031F080E005C0D3
:107F100088E003C08CE001C084E0633079F028F48D
:107F20006130A1F0623041F005C0653059F040F099
:107F3000663051F020E80BC021E809C021E007C0FD
:107F400022E805C022E003C023E001C020E0E0E712
:107F5000F0E09381977F9383E0ECF8E011828065F5
:107F6000822B8083C7CF089592E09093FA33E0ECA0
:107F7000F8E083830BC08091FA33811107C065E676
:107F80007FE082E00E944B1F8FEF0895828188235B
:107F900094F7E0ECF8E08381089561157105F9F03C
:107FA000DC01680F791F22E0E0ECF8E09FEF2093FE
:107FB000FA3393830BC08091FA33811107C06DEDC2
:107FC00073E282E00E94211F80E00895828188236D
:107FD00094F783818D93A617B70749F702C081E014
:107FE000089581E00895CF93DF936115710509F13C
:107FF000DC01680F791F92E0E0ECF8E09093FA332F
:10800000ED018C9183830BC08091FA33811107C0FD
:108010006FE37FE082E00E944B1F80E00DC0828111
:10802000882394F7838188831196A617B70731F7C1
:1080300002C081E001C081E0DF91CF910895E0EAC4
:10804000F6E080E181838683E0E6F6E08183868343
:1080500040E05BE460E070E081E00E9437558FE330
:1080600098E30E94176080E498E30E9443601092B6
:1080700040381092413810923F3810920C341092D0
:10808000113410921234109213341092143410924E
:10809000163410921534109217341092183410922E
:1080A000193410921A3410921B3410921C3410920E
:1080B0001D3410921E3410921F34109220341092EE
:1080C00021341092223410922334109224341092CE
:1080D0002534109226341092103410920F341092DE
:1080E0000E3410920D3448E750E067E274E380E00C
:1080F0009FE00C94B853089581E080931234089562
:10810000109212340895809112340895809123348E
:10811000089580911B340895EF92FF920F931F935F
:10812000CF93DF931F921F92CDB7DEB78B011982D9
:108130001A8220911B34211133C06E3021E0720766
:1081400088F521E020931B3461157105D1F020E002
:1081500030E0AFEAB5E3E82EF92EAB0141555A4CB9
:10816000C701F70161917F016D93FC018081B90125
:10817000680F711DA417B50711F09B01F1CF69833A
:108180007A8342E0BE016F5F7F4FC80181559A4CF0
:108190000E943250009321341093223481E003C0B6
:1081A00080E001C080E00F900F90DF91CF911F9190
:1081B0000F91FF90EF900895EF92FF920F931F930E
:1081C000CF93DF938C01EB0180912334823029F52A
:1081D00064EA77E181E00E944B1F0F2EF5E2EF2E5B
:1081E000F4E3FF2EF02DF701408151816FE974E334
:1081F000C8010E942F64F7018081918103978883D1
:10820000998380912434882321F081E08093233462
:108210000BC01092233481E007C0833021F4109208
:10822000233480E001C080E0DF91CF911F910F9156
:10823000FF90EF9008952EE8E1E1F4E3DC01019076
:108240000D922A95E1F70895EF92FF920F931F93F5
:10825000CF93DF93EC018B018881813031F008F4FA
:1082600066C0823009F45AC05FC0FB0110821582DB
:10827000F2E2CA3BDF0709F441C0EB80F12C29810F
:108280003A812093023430930334E114F10491F0E5
:10829000AFECB7E3C7018153984CF90144914D937A
:1082A0003196A817B907D1F72E0D3F1D2093023440
:1082B000309303344C815D814115510559F06E8135
:1082C0007F81C7018153984C0E942F648C819D81CE
:1082D000E80EF91EF701E153F84C8DE080838AE047
:1082E0008183A7014E5F5F4FFA01E153F84C108282
:1082F0006FEC77E381E00E94C1580EC04091BE222E
:108300005091BF224115510539F06091C022709102
:10831000C12281E00E94C15882E08883F8018581F2
:10832000813039F4188206C0188282E003C080E0F0
:1083300001C080E0DF91CF911F910F91FF90EF90EE
:10834000089580910A34813091F028F08230F9F05C
:108350008330B1F166C080E1E0EAF6E085831092F7
:10836000093488E080933F3881E080930A3480911B
:108370003F3881115AC080E1E0E6F6E0858388E06D
:1083800080933F3882E080930A3480E008958091A2
:108390003F3881114CC040E05BE460E070E081E078
:1083A0000E94375581E00E94CE5481E080939A224A
:1083B00088E280933F3883E080930A3480E0089518
:1083C00068EB71E28AE992E23FDF813019F41092A2
:1083D0000A340895823029F484E080930A3480E0DE
:1083E000089580913F38811124C0809109348330F1
:1083F00048F084E080930A346DE57BE181E00E94DF
:108400004B1F03C082E080930A34809109348F5F50
:108410008093093463E47BE181E00E944B1F80E09C
:10842000089510920A3482E0089580E0089580E073
:10843000089580E00895CF93DF9380918D2190E09F
:10844000FC013197E830F10508F085C2E854FE4F91
:108450000C94EA63409121345091223460E070E042
:1084600083E398E30E94B44F80913338882361F00E
:10847000E4E3F8E380E090E0DC010196A11DB11D8A
:1084800021912111FACF03C080E090E0DC0123E3C9
:1084900038E32093E8213093E9218093E6219093FB
:1084A000E72181E08093E22182E080938D2188E7BB
:1084B00090E0809340389093413810920834D0E097
:1084C0007FC261EB71E282EE91E2BEDEC82F8130A5
:1084D000E9F48FEA95E38093C0229093C1228091C2
:1084E00021349091223402968093BE229093BF2231
:1084F00081E08093BA2283E080938D2188E790E029
:10850000809340389093413810920834209140383D
:1085100030914138232B09F04CC281E08093E22155
:1085200088E790E0809340389093413862E777E1A4
:1085300081E00E944B1F809108348F5F8093083444
:10854000D0E03CC268EB71E28AEB92E27DDEC82F9C
:10855000813061F51092103410920F3480911534EF
:10856000882379F081E08093FA2184E080938D2143
:1085700088E790E080934038909341381092083417
:1085800015C06AE377E181E00E944B1F81E0EAD9E0
:1085900080ED92E0809340389093413887E080935B
:1085A0008D21809108348F5F80930834209140386A
:1085B00030914138232B09F0FEC11092B82110925E
:1085C000BD2181E08093BA2288E790E08093403813
:1085D000909341386AE077E181E00E944B1F8091DF
:1085E00008348F5F80930834D0E0E8C168EB71E213
:1085F0008AEF91E229DE80911034882309F46EC05D
:1086000080910F348823C1F061EF76E181E00E9410
:108610004B1F85E080938D211092103410920F34FF
:1086200081E08093D22288E790E080934038909355
:1086300041381092083452C080911C348823C1F014
:1086400067EC76E181E00E944B1F86E080938D21EC
:108650001092103481E080932A2210920D3488E722
:1086600090E080934038909341381092083436C09F
:1086700060EA76E181E00E944B1F809115348823E7
:10868000C1F06FE676E181E00E944B1F109210343A
:1086900010920F3481E08093FA2188E790E0809374
:1086A000403890934138809108348F5F809308342C
:1086B00015C069E376E181E00E944B1F81E052D949
:1086C00080ED92E0809340389093413887E080932A
:1086D0008D21809108348F5F8093083480914038D9
:1086E00090914138892B09F073C110921034109287
:1086F0000F3481E08093FA2188E790E0809340383E
:108700009093413864E076E181E00E944B1F8091B4
:1087100008348F5F80930834D0E052C168EB71E277
:1087200082ED92E291DDC82F8130B1F481E0809337
:108730008D2182E080931B3410921D3410921E34E0
:1087400010921F341092203410921C341092103466
:1087500010920F34D1E001C0D0E020914038309128
:108760004138232B09F02AC181E08093D22228E7E7
:1087700030E0209340383093413868EC75E10E9436
:108780004B1F809108348F5F8093083417C16CE9C8
:1087900071E28AE292E258DDC82F80910D34813077
:1087A000E9F540911D3450911E3460911F34709151
:1087B0002034413D524061057105F0F088E080931E
:1087C0008D216BE775E181E00E944B1F10921D34F3
:1087D00010921E3410921F341092203481E0809346
:1087E000D22288E790E080934038909341381092ED
:1087F000083410920D3412C065E475E181E00E94E6
:108800004B1F80911D3490911E348093403890937B
:10881000413887E080938D2110920D3420914038AB
:1088200030914138232B09F0C8C010920D3481E0FB
:1088300080932A2288E790E08093403890934138D3
:1088400062E175E181E00E944B1F809108348F5FE7
:1088500080930834D0E0B2C0809115348823E9F0C9
:1088600080911C34882339F08091403890914138B0
:10887000892B09F0AFC01092103410920F3481E0B0
:108880008093FA2184E080938D2188E790E08093A3
:10889000403890934138D0E093C080914038909117
:1088A0004138892B09F098C088E080938D2167EDCD
:1088B00074E181E00E944B1F81E08093D22288E71F
:1088C00090E0809340389093413810920834D0E083
:1088D00077C068EB71E282ED92E2B6DCC82F81309E
:1088E000F9F410920B3441E050E06BE074E38AE05D
:1088F0000E94EC2883E080931B3481E080938D21DB
:1089000010921D3410921E3410921F341092203495
:1089100010921C341092103410920F34D1E001C028
:10892000D0E02091403830914138232B09F046C0E7
:1089300081E08093D22228E730E0209340383093C2
:10894000413864EA74E10E944B1F809108348F5FC4
:108950008093083433C08091403890914138049717
:1089600010F081E001C082E080930B3441E050E0E0
:108970006BE074E38AE00E94EC2883E080931B3470
:1089800081E080938D211092083410921D34109252
:108990001E3410921F341092203410921C34109206
:1089A000103410920F3468E774E10E944B1FD1E03D
:1089B00007C0D0E003C0D0E001C0D0E0C23021F059
:1089C00080910834843050F089E080938D2106C076
:1089D000D0E0F6CFD0E0F4CFD0E0F2CF8D2FDF9112
:1089E000CF9108958091053490E08331910508F08E
:1089F0008AC1FC01E054FE4F0C94EA6381E080934D
:108A000002228093053468EB71E282E092E21CDC82
:108A1000813009F07CC18093AA2282E080930534E2
:108A200080E0089568EB71E28AEA92E20DDC813021
:108A300009F06DC18093B22283E08093053480E019
:108A4000089568EB71E282EB92E2FEDB813009F07F
:108A50005EC180938A2284E08093053480E008958B
:108A600068EB71E28AE892E2EFDB813009F04FC1F6
:108A70008093922285E08093053480E0089568EB2E
:108A800071E282E992E2E0DB813009F040C180933B
:108A90004F388093622286E08093053480E0089509
:108AA00069E478E382E692E2CFDB813009F02FC1FE
:108AB00087E0EFEBF6E3A8E2B4E301900D928A952C
:108AC000E1F781E080934F3880935A2287E08093CA
:108AD000053480E0089569E478E38AE592E2B4DB46
:108AE000813009F014C183E2EFEBF6E3AFE2B4E3C7
:108AF00001900D928A95E1F781E080934F38809341
:108B0000722288E08093053480E0089569E478E378
:108B100082E792E299DB813009F0F9C08DE1EFEB59
:108B2000F6E3A2E5B4E301900D928A95E1F781E0C6
:108B300080934F3880933A2289E08093053480E017
:108B4000089569E478E38AE392E27EDB813009F0FC
:108B5000DEC087E0EFEBF6E3AFE6B4E301900D9201
:108B60008A95E1F781E080934F38809352228AE022
:108B70008093053480E0089569E478E382E592E229
:108B800063DB813009F0C3C083E1EFEBF6E3A6E7D6
:108B9000B4E301900D928A95E1F781E080934F381C
:108BA00080937A228BE08093053480E0089569E415
:108BB00078E38AE792E248DB813009F0A8C080912F
:108BC000BF369091C036A091C1368093893490937E
:108BD0008A34A0938B3481E080934F388093822233
:108BE0008CE08093053480E0089569E478E382E8BE
:108BF00092E22ADB813009F08AC08091BF369091E1
:108C0000C036A091C136B091C23680938C34909317
:108C10008D34A0938E34B0938F3481E080934F389D
:108C200080936A228DE08093053480E0089569E4A2
:108C300078E38AE692E208DB813009F068C08FE0D1
:108C4000EFEBF6E3A0E9B4E301900D928A95E1F72A
:108C500081E080939A228EE08093053480E008952D
:108C600068EB71E28AE992E2EFDA813009F04FC0F5
:108C7000809312228FE08093053480E0089568EBA2
:108C800071E282E192E2E0DA813009F040C0809343
:108C9000CA2280E18093053480E0089568EB71E298
:108CA0008AEC92E2D1DA813091F580930A2281E157
:108CB0008093053480E0089568EB71E28AE092E2E7
:108CC000C3DA813021F58093EA2168E971E10E94DD
:108CD0004B1F82E18093053480E0089568EB71E2D8
:108CE0008AEE91E2B1DA813091F41092273448E7AC
:108CF00050E067E274E380E09FE00E94C553109269
:108D0000053481E008951092053482E008958230A0
:108D100029F483E18093053480E0089580E008958C
:108D2000CF93809104348230B1F028F4882349F045
:108D3000813021F157C08330A1F1843009F443C060
:108D400051C081E0809342226EE671E10E944B1F88
:108D500082E08093043468EB71E282E492E274DA98
:108D6000813009F052C0C1E0C0931A2265E471E17C
:108D70000E944B1FC093043480E04FC068EB71E247
:108D80008AE192E261DA813009F03FC080934A22A1
:108D90006EE171E10E944B1F83E08093043480E018
:108DA0003CC068EB71E28AE492E24EDA813069F508
:108DB0008093322267EF70E10E944B1F84E0809322
:108DC000043480E02AC068EB71E282E392E23CDA8C
:108DD0008130D9F41092043465ED70E10E944B1F8C
:108DE00081E01BC086E080930B3441E050E06BE0F3
:108DF00074E38AE00E94EC2866EB70E181E00E9457
:108E00004B1F1092043482E008C0823029F485E0C0
:108E10008093043480E001C080E0CF910895DC01AC
:108E20008C91833009F4E2C030F4813091F08230CB
:108E300009F467C006C0843009F40AC1853009F41A
:108E40002BC115961C92159714961C92149781E0CD
:108E50008C9388E3A234B807E9F4809148388823DA
:108E6000B1F06230A0F46093BF3681E090E080936F
:108E700000349093013482E0809342381092FE33A4
:108E80001092FF331092FC331092FD3305C1109203
:108E9000423802C188E3A934B80789F480914F3879
:108EA000882351F0109200341092013483E08093B3
:108EB00049381092FB33F0C010924938EDC0149637
:108EC0008C91149713969C9113978917C0F411965F
:108ED000ED91FC911297E80FF11DE4916E130DC016
:108EE0008F5F14968C9314979813D6C01092003409
:108EF0001092013482E08C93CFC01C92CDC01C92A2
:108F0000CBC088E3A234B80709F04FC08091FE338C
:108F10009091FF33009749F5E0910034F0910134CE
:108F2000E154F94C60833197808190E08093FC3369
:108F30009093FD33982F8827862B8093FE33909350
:108F4000FF3380932534909326341092003410928E
:108F50000134892B09F0A0C081E08093473885E077
:108F6000809342381092483897C020910034309155
:108F70000134F901E154F94C60832F5F3F4F209396
:108F800000343093013401978093FE339093FF3384
:108F9000892B09F081C084E08093423882E090E020
:108FA0008093FE339093FF3377C06D3009F474C023
:108FB0006A3071F08091003490910134FC01E154E9
:108FC000F94C60830196809300349093013464C01F
:108FD00081E015968C93159785E08C93E091003491
:108FE000F0910134E154F94C108256C06A3031F4EA
:108FF0008091FB338F5F8093FB334EC08091FB33B6
:10900000813089F46D3009F447C08091003490912B
:109010000134FC01E154F94C6083019680930034E3
:109020009093013439C08330B9F56B34A9F581E0F0
:1090300015968C93159785E08C93E0910034F09110
:109040000134E154F94C108216961C92169724C0F4
:109050008091FE339091FF330097F1F0209100341E
:1090600030910134F901E154F94C60832F5F3F4F97
:10907000209300343093013401978093FE33909312
:10908000FF33892B49F481E015968C93159785E081
:109090008C9316961C92169715968C910895409174
:1090A00023346091143430E080E050E090E0E92F08
:1090B000F0E0E154F94C20812C3221F48F5F8230B2
:1090C000A1F531C0823021F4213369F541E02BC094
:1090D000843021F4213339F561E025C0853019F55C
:1090E0002C3209F12032F9F0222369F02053552364
:1090F00039F0330F732F770F770F370F320F01C00F
:10910000322F5F5F10C04093233460931434309348
:109110002434332369F081E0809323346BE970E1D8
:109120000C944B1F08959F5FC2CF8430B9F6FBCFDC
:1091300008956F927F929F92AF92BF92CF92DF92EB
:10914000EF92FF921F93CF93DF9320E0C12CD12C9D
:10915000760130E010E0912C0F2EFCE1AF2EF4E30D
:10916000BF2EF02D0F2EFBE16F2EF4E37F2EF02D9E
:10917000C3E2D4E3E92DF0E0E154F94C80818C3274
:1091800009F41F5F213009F45DC038F0223009F482
:1091900087C0233009F4A3C0DFC0111127C08C326F
:1091A00041F1982F9F7D09F4D7C040ED480F311150
:1091B00005C0C42ED12CE12CF12C16C0CC0CDD1C2A
:1091C000EE1CFF1CD701C601880F991FAA1FBB1FE9
:1091D000880F991FAA1FBB1FC80ED91EEA1EFB1EAF
:1091E000C40ED11CE11CF11C3F5FB6C08C3209F0EB
:1091F000B3C085E0C816D104E104F10448F4F301DA
:109200008081813029F480930F3421E030E0A4C0C4
:1092100010920F34F6E2CF16D104E104F10451F4B8
:1092200081E0F501808363E570E10E944B1F21E03E
:1092300030E092C06DE270E181E00E944B1F21E0BE
:1092400030E08AC0113041F58C3209F47DC0982F8E
:109250009F7D09F481C040ED480F311105C0C42E37
:10926000D12CE12CF12C16C0CC0CDD1CEE1CFF1C0B
:10927000D701C601880F991FAA1FBB1F880F991F0E
:10928000AA1FBB1FC80ED91EEA1EFB1EC40ED11C8E
:10929000E11CF11C3F5F60C08C3209F05DC057C01B
:1092A000123009F059C08C3209F456C0803209F4EA
:1092B00053C0813359F481E0888380930E3469EE82
:1092C0007FE00E944B1F23E030E046C08881813060
:1092D00009F040C010920E3423E030E03DC015305C
:1092E00039F58C32C9F18032B9F1882319F140ED9A
:1092F000480F311105C0C42ED12CE12CF12C16C021
:10930000CC0CDD1CEE1CFF1CD701C601880F991F79
:10931000AA1FBB1F880F991FAA1FBB1FC80ED91EEB
:10932000EA1EFB1EC40ED11CE11CF11C3F5F14C0E1
:10933000811112C0C0922434CD28CE28CF2871F0DC
:1093400081E0809323340AC022E030E005C022E0AF
:1093500030E002C023E030E093940CCFDF91CF9156
:109360001F91FF90EF90DF90CF90BF90AF909F90B4
:109370007F906F900895CF92DF92EF92FF92CF93FC
:10938000DF9320E0C12CD12C760130E0D0E0C0E0AA
:10939000EC2FF0E0E154F94C80818C3209F4DF5F6E
:1093A000222321F0213009F442C083C0D11127C00B
:1093B0008C3241F1982F9F7D09F47BC040ED480F1E
:1093C000311105C0C42ED12CE12CF12C16C0CC0CCF
:1093D000DD1CEE1CFF1CD701C601880F991FAA1FB8
:1093E000BB1F880F991FAA1FBB1FC80ED91EEA1EDC
:1093F000FB1EC40ED11CE11CF11C3F5F5AC08C3215
:1094000009F057C0C114D104E104F10441F46EEC39
:109410007FE081E00E944B1F21E030E04AC064EA17
:109420007FE081E00E944B1F21E030E042C0D1305C
:1094300031F58C3221F1982F9F7D09F140ED480FD5
:10944000311105C0C42ED12CE12CF12C16C0CC0C4E
:10945000DD1CEE1CFF1CD701C601880F991FAA1F37
:10946000BB1F880F991FAA1FBB1FC80ED91EEA1E5B
:10947000FB1EC40ED11CE11CF11C3F5F1AC0A8EEFC
:10948000B3E0A70196010E94FF632AEF30E040E0BD
:1094900050E00E94AC6320931D3430931E344093FF
:1094A0001F345093203469E87FE081E00E944B1F15
:1094B00002C0CF5F6DCFDF91CF91FF90EF90DF9033
:1094C000CF90089530E0832F90E0FC01E154F94CF7
:1094D00020812C32C9F02032B9F02E3649F4109296
:1094E0001734109218341092193410921A340895C7
:1094F0008154994CD2D5609317347093183480936B
:10950000193490931A3408953F5FDDCF409125348C
:10951000509126344115510589F0AFEBB6E3EFE9E0
:10952000F4E320E030E080E090E06D916193260F5D
:10953000311D019684179507C0F304C020E030E088
:1095400080E090E0FC01E154F94C408150E0542F60
:1095500044278181482B81E02417350709F080E0FA
:109560000895CF93DF938091073490E0893091057F
:1095700008F061C2FC01ED52FE4F0C94EA63809149
:109580000E348823C9F08091143481111092143460
:1095900081E08093922283E08093073488E790E013
:1095A0008093403890934138109206346AE474E115
:1095B00081E00E944B1F0BC081E08093073488E755
:1095C00090E0809340389093413810920634109286
:1095D000103410920E34D0E03AC2809115348823B2
:1095E000D9F080911434882321F081E08093F22116
:1095F00003C081E08093FA2182E08093073488E7FA
:1096000090E0809340389093413867E374E181E0C3
:109610000E944B1FD0E01BC261E074E181E00E9418
:109620004B1F81E00E94B23C80ED92E08093403875
:109630009093413887E080930734809106348F5FA0
:109640008093063468EE73E181E00E944B1FD0E006
:10965000FEC180911434882341F068EB71E282EFFF
:1096600091E20E942441C82F07C068EB71E28AEFA3
:1096700091E20E942441C82F80911034882309F47C
:1096800057C08091143481111092143480910E349B
:109690008823C9F01092103410920E3481E0809328
:1096A000922283E08093073488E790E080934038EB
:1096B000909341381092063469EC73E181E00E9486
:1096C0004B1FD0E0C2C1809115348823C9F010929D
:1096D000103410920E3481E08093FA2188E790E0F4
:1096E0008093403890934138809106348F5F809307
:1096F00006346DEA73E181E00E944B1FD0E0A5C102
:1097000067E773E181E00E944B1F81E00E94B23C59
:1097100080ED92E0809340389093413887E08093C9
:109720000734809106348F5F80930634D0E08DC17A
:109730002091403830914138232B09F07FC110929D
:10974000103410920E3481E08093FA2188E790E083
:109750008093403890934138809106348F5F809396
:1097600006346EE573E181E00E944B1FD0E06DC1CD
:1097700068EB71E282E992E20E942441C82F8130B5
:1097800081F481E0809348388093222284E08093A2
:10979000073488E790E080934038909341381092E6
:1097A00006342091403830914138232B09F048C1CC
:1097B0006CE273E181E00E944B1F81E08093922272
:1097C00028E730E0209340383093413880910634C8
:1097D0008F5F80930634D0E038C162E478E382E2A0
:1097E00092E20E942441C82F813079F58FDE8823D0
:1097F000A9F066E073E181E00E944B1F81E0809355
:109800009A2285E08093073488E790E0809340387F
:109810009093413810920634D0E019C165EE72E1A0
:1098200081E00E944B1F81E0809348388093222280
:1098300088E790E0809340389093413880910634D7
:109840008F5F80930634D0E002C120914038309180
:109850004138232B09F0F6C081E08093483880938B
:10986000222288E790E0809340389093413880919D
:1098700006348F5F8093063464E972E181E00E94D0
:109880004B1FD0E0E2C068EB71E28AE992E20E94ED
:109890002441C82F813071F481E08093C22286E098
:1098A0008093073488E790E0809340389093413864
:1098B000109206342091403830914138232B09F022
:1098C000C3C062E672E181E00E944B1F81E0809399
:1098D0009A2228E730E02093403830934138809135
:1098E00006348F5F80930634D0E0AFC068EB71E23E
:1098F00082EC92E20E942441C82F813061F482E020
:10990000809323341092073461E472E181E00E9475
:109910004B1FD1E001C0D0E0209140383091413858
:10992000232B09F092C06FE072E181E00E944B1F8F
:1099300081E08093C22228E730E0209340383093C2
:109940004138809106348F5F809306347EC08091C9
:109950001534882391F01092103410920E3481E067
:109960008093FA2188E790E08093403890934138C3
:1099700082E080930734D0E06AC0809140389091B3
:109980004138892B09F06BC0C3E0C0930B3441E030
:1099900050E06BE074E38AE00E94EC2865ED71E131
:1099A00081E00E944B1F109240381092413881E0B4
:1099B0008093C22268EB71E282EC92E20E94244121
:1099C000C0932334109207346CEB71E181E00E9464
:1099D0004B1FD1E03CC080914038909141380497B2
:1099E00010F084E001C085E080930B3441E050E04A
:1099F0006BE074E38AE00E94EC28C1E0C093C222CD
:109A000068EB71E282EC92E20E942441C0939A22B8
:109A100068EB71E28AE992E20E94244183E080933C
:109A2000233410920734109240381092413810922B
:109A30000634D1E00CC0C0E0D0E007C0D0E005C0E3
:109A4000D0E003C0D0E001C0D0E0C23021F080916E
:109A50000634843030F088E08093073402C0D0E0D0
:109A6000F6CF8D2FDF91CF910895CF93DF9300D064
:109A7000CDB7DEB78091113490E08930910508F0C0
:109A8000E4C0FC01E452FE4F0C94EA63E0EAF6E025
:109A9000848184FF02C080E1868380911234882310
:109AA00009F4EBC081E0809311341092153465E223
:109AB0007BE10E944B1FE1C00E94A141813009F06F
:109AC000D7C068E07BE10E944B1F83E08093113494
:109AD000D4C068EB71E282EA92E20E9424418130B4
:109AE00009F0C6C068EE7AE10E944B1F1092113453
:109AF00081E001D780E1E0E6F6E08683BEC0809198
:109B000027348F3F49F484E08093113467EC7AE185
:109B100081E00E944B1FB1C085E080931134ADC03D
:109B20000E94F244813009F0A3C00E94B23C86E05A
:109B3000809311346BEA7AE181E00E944B1F67E762
:109B40007AE181E00E944B1F98C08091123481110C
:109B50001AC080911B34811116C080912334811169
:109B600021C080910C3481112CC082E0809311348B
:109B700081E08093A22269E57AE10E944B1F80E098
:109B80000E94B23C7AC080911B34813059F40E940B
:109B9000B23C87E08093113468E27AE181E00E9470
:109BA0004B1F6BC080912334813059F40E94B23C2A
:109BB00088E08093113468EF79E181E00E944B1FC7
:109BC0005CC080910C34882361F081E00E94B23C3B
:109BD00086E08093113465EC79E181E00E944B1FAF
:109BE0004CC0809127348F3F09F047C084E08093B8
:109BF00011341092273462EA79E181E00E944B1F10
:109C00003CC08ED88130A1F56EE679E10E944B1FF1
:109C100085E08093113410920C342FC00E941B42B7
:109C2000813031F56EE379E10E944B1F85E080932E
:109C3000113423C096DC8130D9F46FE079E10E94C1
:109C40004B1F85E08093113418C06AEF78E181E002
:109C50000E944B1F0E941F401092113481E04BD68E
:109C600080E1E0E6F6E086838FEF8093273405C03D
:109C7000823019F489E08093113481E00E947C568F
:109C8000892B09F4E6C041E050E0BE016D5F7F4FD3
:109C900081E07ED78111DDC08B8189831A82BE016C
:109CA0006F5F7F4F81E00E94211F6B818AEA91E202
:109CB000B6D88823A9F081E0809314341092AA21A9
:109CC0001092AF218093233440E050E060E070E0D8
:109CD00084E10E94EC2863ED78E181E00E944B1F53
:109CE0006B8184ED91E29BD88823D1F08091BF36BF
:109CF000805380931634882341F081E0809315349B
:109D000069EB78E10E944B1F07C0109215346DE992
:109D100078E181E00E944B1F1092D4211092D9214A
:109D20006B818DEC91E27BD88823D1F08091BF3696
:109D3000805380931634882341F081E0809315345A
:109D400063E878E10E944B1F07C01092153467E664
:109D500078E181E00E944B1F1092CD211092D22118
:109D60006B818BED91E25BD8882349F08091BF36FF
:109D70008053809313341092DB211092E0216B8189
:109D80008EE891E24CD8882329F09CDB10928E213A
:109D9000109293216B818FEB91E241D8882361F07F
:109DA0001092BF211092C42189E08093113469E29E
:109DB00078E181E00E944B1F6B8186EC91E22FD805
:109DC000882361F01092C6211092CB2189E0809304
:109DD000113466EF77E181E00E944B1F6B8185E9CA
:109DE00091E21DD8882329F05AD91092952110921A
:109DF0009A216B8183EA91E212D8882341F099D9A4
:109E000081E0809310341092A3211092A8216B81DD
:109E10008CE991E204D8882341F0ADDA81E08093A7
:109E20000D3410929C211092A1216B8188EB91E25C
:109E30000E940F476B8181EB91E20E940F476B817B
:109E400089E498E30E940F476B8182E498E30E94C3
:109E50000F472396CDBFDEBFDF91CF91089581E0FC
:109E60000E94B23C81E080930C34809112348111C5
:109E700003C081E080931234089581E090910C3406
:109E8000911180E0089527E0EFE6F4E3DC01019012
:109E90000D922A95E1F70895CF93DF93CDB7DEB702
:109EA000C750D140CDBFDEBF9091AF359330B1F5F3
:109EB0009091B035903391F59EEF980F923070F5F8
:109EC00093E09A8390E39B839091B1359C83823099
:109ED00011F481E001C08FEFC95FDE4F8883C75066
:109EE000D1400E94A132813051F4198241E050E00A
:109EF000BE01695F7E4FCE0101960E94DA120E9478
:109F0000F032813059F483E0898341E050E0BE01B2
:109F1000695F7E4FCE0101960E94DA12C95FDE4F63
:109F2000CDBFDEBFDF91CF910895CF93DF93CBE11B
:109F3000D4E38881B1DF1882DF91CF9108950F9328
:109F4000CF93DF931F92CDB7DEB72FB72983F89455
:109F50001BBEFC0108ED04BF608389818FBF0F9099
:109F6000DF91CF910F9108954F925F926F927F9200
:109F7000AF92BF92CF92DF92EF92FF920F931F9317
:109F8000CF93DF93CDB7DEB72B97CDBFDEBF6C018C
:109F9000242F352F862F972F8E010F5F1F4F5801CB
:109FA0007E014CE0E40EF11C0F2EFAE04F2E512CF6
:109FB000612C712CF02D622F732FA30192010E944E
:109FC000AC63F80161938F01842F952FEE15FF0587
:109FD00091F7FE013C964FEFA41AB40A90E020E0FE
:109FE0008291811102C0222339F0D601A90FB11D3F
:109FF000805D8C939F5F21E0EA15FB0589F7F601F0
:10A00000E90FF11D8981805D80839F5FF601E90F73
:10A01000F11D10822B96CDBFDEBFDF91CF911F9136
:10A020000F91FF90EF90DF90CF90BF90AF907F9017
:10A030006F905F904F900895FC01862F82958F70EE
:10A040008A3018F4805D808302C0895C80836F70E1
:10A0500077276A3018F4605D618302C0695C6183B0
:10A0600012820895CF93DF93FC01423098F0A62F1F
:10A07000B72FED012D91842F90E00197C80FD91FC4
:10A0800038813083EF01C80FD91F288342503196A1
:10A09000423078F7DF91CF9108950F931F93FC0121
:10A0A0008081882309F485C040E04F5FDF01A40F61
:10A0B000B11D8C918111F9CF442309F47EC060E079
:10A0C00070E0CB0150E0DF01A40FB11D11970C919E
:10A0D000023640F010E007551109222717FD2095A0
:10A0E000322F11C0023440F010E00753110922272B
:10A0F00017FD2095322F07C010E0005311092227C9
:10A1000017FD2095322F552309F44AC0513089F4A8
:10A11000000F111F221F331F000F111F221F331F9B
:10A12000000F111F221F331F000F111F221F331F8B
:10A1300037C0523029F4322F212F102F002730C082
:10A14000533051F40F2EFCE0000F111F221F331F5C
:10A15000FA95D1F7F02D24C0543021F4980111273D
:10A1600000271EC0553051F40F2EF4E1000F111FCF
:10A17000221F331FFA95D1F7F02D12C0563029F463
:10A18000302F2227112700270BC0573049F40F2EFC
:10A19000FCE1000F111F221F331FFA95D1F7F02D9C
:10A1A000602B712B822B932B5F5F415009F08BCF7B
:10A1B00007C060E070E0CB0103C060E070E0CB015D
:10A1C0001F910F910895982F92959F70990F292FA5
:10A1D000220F220F920F8F70890F08952DEC829F0E
:10A1E000312D1124932F969596959695990F492F79
:10A1F000440F440F940F891B982F832F86958695C3
:10A200008695829F212D1124269526952695220F2D
:10A21000322F330F330F230F821B20E1829F900DCB
:10A220001124892F0895CF92DF92EF92FF920F931E
:10A230001F93423019F0443069F034C00027162FC4
:10A24000272F382F2227332768017901C72AC70112
:10A25000B60128C0F62EEE24DD24CC24092F1127C8
:10A26000222733270C291D292E293F296B017C0128
:10A27000CC24DD24FF24CD2CDE2CEF2CFF240C2954
:10A280001D292E293F29DC01CB018827AA27BB27BE
:10A29000BA2FA92F982F8827BC01CD01602B712BD5
:10A2A000822B932B1F910F91FF90EF90DF90CF9017
:10A2B0000895E0E0F6E083EA808380E2858383E826
:10A2C0008683E0E2F6E083E0808315828683E0E423
:10A2D000F6E090EB908315829683E0E6F6E093E358
:10A2E000908315829683E0E8F6E0808381E08583A1
:10A2F00082E08683E0EAF6E080E48083158286834C
:10A300000895E0E7F0E08BE5808385E08183828338
:10A3100087E283838FE484838FE685838683089531
:10A32000CF93DF931F92CDB7DEB7EBDFC2DF7FD0D5
:10A330008983F9D10E94BE60B0D20E946D3F0E9415
:10A340008A110BD20E949C240E94FC1E0E941F4076
:10A350000E94E83A0E9491320E94C8600E947F2CBD
:10A360000E949B2581E00E941E1FE0EAF0E08281AE
:10A370008160828385E598E30E94176084E598E315
:10A380000E94176078940E944E230E947C5A0E947B
:10A390009F310E947C350E9427260E94D8320E945D
:10A3A00083610E9415260E94A12E882371F041E04E
:10A3B00050E0BE016F5F7F4F82E00E94EC280E9458
:10A3C0002E290E94585B0E94895B11E004E0809175
:10A3D000543881110AC0109354380E94F7600E94CB
:10A3E000AD250E94E45B0E94E22D809155388111D9
:10A3F0000CC00093553861E074E283E00E94211F95
:10A4000051D080E598E30E94E12F0E94652C2DDB5E
:10A410000E949A3D0E94A4320E94F3320E94C41E00
:10A420000E9483408111D3CF0E94A037D0CF80916A
:10A430007800811103C01092563827C085FF04C0F0
:10A4400091E09093563821C084FF04C092E090932D
:10A4500056381BC083FF04C093E09093563815C054
:10A4600082FF04C094E0909356380FC081FF04C06F
:10A4700095E09093563809C080FF04C096E0909311
:10A48000563803C097E090935638E8E7F0E09081A3
:10A490008095892380836BE280E890E050DD809195
:10A4A00056380895A89508958091583890E0FC0199
:10A4B0003197E930F10520F4EB51FE4F0C94EA633B
:10A4C00020E011C02CE00FC024E10DC02CE10BC036
:10A4D00024E209C02CE207C024E305C02CE303C03A
:10A4E00020E401C024E080915938823031F083307B
:10A4F00031F0813031F060E005C062E003C063E01C
:10A5000001C061E08091573890E08930910508F0F2
:10A51000B0C0FC01E251FE4F0C94EA63E0E5F0E0CC
:10A52000808184608083622B81E490E008DDE0E537
:10A53000F0E0818182FFFDCF62E080E490E0FFDC0B
:10A54000AAC0E0E5F0E0808182608083622B81E434
:10A5500090E0F5DCE0E5F0E0818181FFFDCF61E096
:10A5600080E490E0ECDC97C0E0E5F0E082E08283FC
:10A57000808188608083622B81E490E0E0DCE0E50C
:10A58000F0E0818183FFFDCF63E080E490E0D7DCE1
:10A5900082C0E0E5F0E080E482838081886080838F
:10A5A000622B81E490E0CBDCE0E5F0E0818183FF89
:10A5B000FDCF63E080E490E0C2DC6DC080915C3848
:10A5C000806CE0E5F0E08583808180618083622B90
:10A5D00081E490E0B4DCE0E5F0E0818184FFFDCF30
:10A5E00064E080E490E0ABDC56C080915C38806C25
:10A5F000E0E5F0E08583808180618083622B81E4E7
:10A6000090E09DDCE0E5F0E0818184FFFDCF64E037
:10A6100080E490E094DC3FC080915C388068E0E5A5
:10A62000F0E08583808180618083622B81E490E00B
:10A6300086DCE0E5F0E0818184FFFDCF64E080E42A
:10A6400090E07DDC28C080915C38E0E5F0E0858317
:10A65000808180618083622B81E490E070DCE0E5A2
:10A66000F0E0818184FFFDCF64E080E490E067DC6E
:10A6700012C0E0E5F0E0808181608083622B81E49C
:10A6800090E05DDCE0E5F0E0818180FFFDCF60E0FF
:10A6900080E490E054DC80915A388823E1F0809186
:10A6A0005B38823049F0833061F0813079F483E0A7
:10A6B000E0E4F0E0838312C085E0E0E4F0E083832F
:10A6C0000DC08BE0E0E4F0E0838308C081E0E0E4CB
:10A6D000F0E0838303C0E0E4F0E0138280915D3812
:10A6E000882341F0E0E5F0E082E0828381E0868328
:10A6F0008093680080915E38882341F0E0E5F0E0C7
:10A7000082E0828381E086838093680080915F3855
:10A71000882341F0E0E5F0E082E0828381E08683F7
:10A7200080936800089589E0E3E1F4E2A7E5B8E3E7
:10A7300001900D928A95E1F7B7CE0895EF93FF93BC
:10A740000F932F93EBECF1E008ED21E004BF2083A1
:10A750002F910F91FF91EF910895E0ECF1E0878543
:10A760008823ECF3E0ECF1E0848588608487089529
:10A770009B01E0ECF1E067856623ECF3BC01705FC0
:10A78000C9010E942F6481E008957F928F929F9269
:10A79000AF92BF92CF92DF92EF92FF920F931F93EF
:10A7A000CF93DF93EC017B015A01E0ECF1E0878568
:10A7B0008823ECF3E0ECF1E0878581FF03C086E3BA
:10A7C0008287BCDF9E012F713327D695C795D2951E
:10A7D000C295CF70CD27DF70CD27A114B10409F445
:10A7E0004DC06E01CC0CDD1CCC0CDD1CCC0CDD1C7A
:10A7F000CC0CDD1CCC0CDD1CC0ECD1E068948824B2
:10A8000085F8912C0F2EF5E37F2EF02D8F85882370
:10A81000ECF38401021B130BA016B10608F48501AA
:10A8200001151105A1F02C0D3D1D80E090E040E0E8
:10A83000F701E80FF91F5081820F931FFC01F05FB1
:10A8400050834F5F842F90E08017910788F38F85A6
:10A850008823ECF3C8828D2D8F7189831A827A86C2
:10A860006DDFA01AB10AE00EF11E80E2C80ED11C05
:10A87000A114B10419F020E030E0C8CF81E0DF91ED
:10A88000CF911F910F91FF90EF90DF90CF90BF90ED
:10A89000AF909F908F907F90089580E698E30C94FE
:10A8A000176008951F93CF93DF931FB7F894411556
:10A8B0005105D9F0460F571FEB01A0ECB1E031E094
:10A8C000861B970B1F962C911F972223DCF31A9659
:10A8D0003C931A97FC01EC0FFD1FE491E9931A9643
:10A8E0001C921A97C417D50769F71FBF7894DF9198
:10A8F000CF911F910895843008F048C090E025E67C
:10A9000032E0829FF001839FF00D929FF00D1124A1
:10A91000EF59F74C20812223D9F125E632E0829FBE
:10A92000F001839FF00D929FF00D1124EF59F74C29
:10A930002181222379F125E632E0829FF001839F75
:10A94000F00D929FF00D1124EB53F54C2081222342
:10A9500019F1FC01EE0FFF1FE80FF91FEE0FFF1FAB
:10A96000E45EFB4D0190F081E02D2481277E24835D
:10A9700025E632E0829FF001839FF00D929FF00D5B
:10A980001124EF59F74C118280E008958BEF089560
:10A990008BEF08958BEF08958DEF0895843008F0C4
:10A9A00060C090E025E632E0829FF001839FF00DC9
:10A9B000929FF00D1124EF59F74C2081222309F4C6
:10A9C00052C025E632E0829FF001839FF00D929FF6
:10A9D000F00D1124EF59F74C2181211146C025E6D5
:10A9E00032E0829FF001839FF00D929FF00D1124C1
:10A9F000EF59F74CDF01A25DBE4F1C9211961D92DC
:10AA00001C92119712961D921C921197A25DBE4F37
:10AA10001C9211961D921C92119712961D921C92D7
:10AA20001197129621E02C93DC01AA0FBB1F8A0F0D
:10AA30009B1FDC01AA0FBB1FA45EBB4D0D90BC91F8
:10AA4000A02D11968C911197806C11968C93119773
:10AA500014968C911497886114968C93218380E0CE
:10AA600008958BEF08958BEF08958BEF08951F9352
:10AA7000CF93DF93843008F082C090E025E632E087
:10AA8000829FF001839FF00D929FF00D1124EF59EA
:10AA9000F74C2181211175C0FC01EE0FFF1FE80F5B
:10AAA000F91FEE0FFF1FE45EFB4DA281B38121E091
:10AAB00030E0E901048002C0CC0FDD1F0A94E2F708
:10AAC0001296CC931297058002C0220F331F0A946E
:10AAD000E2F711962C93119715962C930190F08123
:10AAE000E02D2381246123832481277E24832581F3
:10AAF00023602583403825E252076105710511F175
:10AB000060F4403629E052076105710529F1403CA7
:10AB1000524161057105D9F036C041152BE4520749
:10AB20006105710551F04115514E6105710559F5E9
:10AB300026E9268320E9278313C021EC268322E916
:10AB400027830EC023E0268326E9278309C025E852
:10AB500026832CE9278304C025EC26832CEA27834F
:10AB600025E632E0829FF001839FF00D929FF00D69
:10AB70001124EF59F74C81E0808380E005C08BEF12
:10AB800003C08BEF01C08CEFDF91CF911F9108952F
:10AB9000AF92BF92CF92DF92EF92FF920F931F93EB
:10ABA000CF93DF93843008F095C0E82FF0E085E67E
:10ABB00092E0E89FD001E99FB00DF89FB00D1124FD
:10ABC000AF59B74C8C91882309F486C085E692E092
:10ABD000E89FD001E99FB00DF89FB00D1124AF5947
:10ABE000B74C11968C91882309F478C085E692E0E1
:10ABF000E89FD001E99FB00DF89FB00D1124A15737
:10AC0000B64C8C9181116CC085E692E0E89FD00132
:10AC1000E99FB00DF89FB00D1124A157B64C81E00B
:10AC20008C934115510509F446C08B015B01A40EBC
:10AC3000B51E85E692E0E89FA001E99F500DF89FC0
:10AC4000500D11244F59574CEA01CF5CDE4F0F2EA7
:10AC5000FCE2CF2EDD24D394F02DA881B981A40F7E
:10AC6000B51F12968C91D8018D938D01E880F980E3
:10AC7000BFEFEB1AFB0A9701369527953695279576
:10AC8000ABE3BDE60E94F063969587959295829519
:10AC90008F7089279F7089278C9D90018D9D300D25
:10ACA0009C9D300D1124C701821B930B88839983CF
:10ACB0000A151B0591F625E632E0E29FC001E39FED
:10ACC000900DF29F900D1124FC01E157F64C10827B
:10ACD00080E007C08BEF05C08BEF03C08BEF01C096
:10ACE0008DEFDF91CF911F910F91FF90EF90DF904B
:10ACF000CF90BF90AF900895843008F078C090E076
:10AD000025E632E0829FF001839FF00D929FF00DC7
:10AD10001124EF59F74C2081222309F46BC025E65A
:10AD200032E0829FF001839FF00D929FF00D11247D
:10AD3000EF59F74C2181222309F45FC0FC01EE0F8B
:10AD4000FF1FE80FF91FEE0FFF1FE45EFB4D0190A0
:10AD5000F081E02D23812F7E238345E652E0849FFE
:10AD60009001859F300D949F300D11242F59374C41
:10AD7000D901A15DBE4F4D915C91119712962D9115
:10AD80003C9142175307C8F445E652E0849F900176
:10AD9000859F300D949F300D11242F59374CD901C8
:10ADA000A15DBE4F8D919C91119712962D913C9172
:10ADB000845D9E4F821B930B16C045E652E0849F34
:10ADC0009001859F300D949F300D11242F59374CE1
:10ADD000D901A15DBE4F8D919C91119712962D9135
:10ADE0003C91821B930B23812061238308958BEF79
:10ADF0009FEF08958BEF9FEF08958BEF9FEF0895DE
:10AE0000843050F590E025E632E0829FF001839F88
:10AE1000F00D929FF00D1124EF59F74C2081222361
:10AE2000E9F025E632E0829FF001839FF00D929FCA
:10AE3000F00D1124EF59F74C2181222389F025E6EA
:10AE400032E0829FF001839FF00D929FF00D11245C
:10AE5000EB53F54C808108958BEF08958BEF0895A7
:10AE60008BEF0895843008F065C090E025E632E06D
:10AE7000829FF001839FF00D929FF00D1124EF59F6
:10AE8000F74C2081222309F455C025E632E0829F49
:10AE9000F001839FF00D929FF00D1124EF59F74CB4
:10AEA0002181222309F446C0FC01EE0FFF1FE80FA9
:10AEB000F91FEE0FFF1FE45EFB4D0190F081E02DC6
:10AEC000608145E652E0849F9001859F300D949FFC
:10AED000300D1124C9018F59974CFC01E15DFE4FE3
:10AEE00020813181DC01A20FB31F12966C93408147
:10AEF00051814F5F5F4F9A0136952795369527957B
:10AF0000ABE3BDE60E94F063969587959295829596
:10AF10008F7089279F7089276CE271E0869F90016E
:10AF2000879F300D969F300D1124CA01821B930B11
:10AF30008083918308951F920F920FB60F92112470
:10AF40000BB60F922F933F934F935F936F937F9323
:10AF50008F939F93AF93BF93EF93FF9380E082DF34
:10AF6000FF91EF91BF91AF919F918F917F916F91E1
:10AF70005F914F913F912F910F900BBE0F900FBE9D
:10AF80000F901F9018951F920F920FB60F921124D9
:10AF90000BB60F922F933F934F935F936F937F93D3
:10AFA0008F939F93AF93BF93EF93FF9381E05ADF0B
:10AFB000FF91EF91BF91AF919F918F917F916F9191
:10AFC0005F914F913F912F910F900BBE0F900FBE4D
:10AFD0000F901F9018951F920F920FB60F92112489
:10AFE0000BB60F922F933F934F935F936F937F9383
:10AFF0008F939F93AF93BF93EF93FF9382E032DFE2
:10B00000FF91EF91BF91AF919F918F917F916F9140
:10B010005F914F913F912F910F900BBE0F900FBEFC
:10B020000F901F9018951F920F920FB60F92112438
:10B030000BB60F922F933F934F935F936F937F9332
:10B040008F939F93AF93BF93EF93FF9383E00ADFB8
:10B05000FF91EF91BF91AF919F918F917F916F91F0
:10B060005F914F913F912F910F900BBE0F900FBEAC
:10B070000F901F901895CF93DF93843008F07EC017
:10B0800090E025E632E0829FF001839FF00D929FD1
:10B09000F00D1124EF59F74C2081222309F46EC0E2
:10B0A00025E632E0829FF001839FF00D929FF00D24
:10B0B0001124EF59F74C2181222309F45FC0E05A93
:10B0C000FD4F4081518132962081318142175307D3
:10B0D00009F447C0FC01EE0FFF1FE80FF91FEE0F48
:10B0E000FF1FE45EFB4DA081B18145E652E0849FE5
:10B0F0009001859F300D949F300D1124C9018F5907
:10B10000974CFC01EE59FD4FC081D1818C0F9D1FE2
:10B11000EC01CD5CDE4F88818C93408151814F5F83
:10B120005F4F9A013695279536952795ABE3BDE697
:10B130000E94F06396958795929582958F708927E6
:10B140009F7089276CE271E0869F9001879F300D88
:10B15000969F300D1124CA01821B930B808391832B
:10B160000DC025E632E0829FF001839FF00D929F93
:10B17000F00D1124EB53F54C81E08083DF91CF91EA
:10B1800008956F927F928F929F92AF92BF92CF92CB
:10B19000DF92EF92FF921F93CF93DF93182F8430AB
:10B1A00008F0C8C0C82FD0E085E692E0C89FF00143
:10B1B000C99FF00DD89FF00D1124EF59F74C8081F5
:10B1C000882309F4B9C085E692E0C89FF001C99FC1
:10B1D000F00DD89FF00D1124EF59F74C8181882391
:10B1E00009F4ACC085E692E0C89FF001C99FF00D5C
:10B1F000D89FF00D1124E054F54C80818111A0C03E
:10B2000085E692E0C89FF001C99FF00DD89FF00D30
:10B210001124E054F54C81E080834115510509F477
:10B220005FC0FE01EE0FFF1FEC0FFD1FEE0FFF1FB3
:10B23000E45EFB4D0190F081E02D7B015B01A40EEB
:10B24000B51E85E692E0C89FA001C99F500DD89F0A
:10B25000500D11244F59574C4A0180EA881A8DEF3E
:10B26000980A0F2EFCE26F2E77247394F02DD401F0
:10B270002D913C91D7018D917D01D901A40FB51F6E
:10B28000AD5CBE4F8C9383818B7F8383D401CD9043
:10B29000DC90BFEFCB1ADB0A9601369527953695E1
:10B2A0002795ABE3BDE60E94F0639695879592954E
:10B2B00082958F7089279F708927869DB001879D11
:10B2C000700D969D700D1124C601861B970BD4013D
:10B2D0008D939C93838184608383EA14FB0439F605
:10B2E00085E692E0C89FF001C99FF00DD89FF00D50
:10B2F0001124EB53F54C8081813071F485E692E0A6
:10B30000C89FF001C99FF00DD89FF00D1124EB5399
:10B31000F54C1082812FAFDE85E692E0C89FF001E8
:10B32000C99FF00DD89FF00D1124E054F54C108208
:10B3300080E007C08BEF05C08BEF03C08BEF01C02F
:10B340008DEFDF91CF911F91FF90EF90DF90CF9025
:10B35000BF90AF909F908F907F906F900895DF92F5
:10B36000EF92FF920F931F93CF93DF931F92CDB76E
:10B37000DEB7D82E41155105A9F07A01062F172FF7
:10B38000F8019491998341E050E0BE016F5F7F4FD7
:10B390008D2DF7DE0F5F1F4FF1E0EF1AF108E1147A
:10B3A000F10471F780E00F90DF91CF911F910F9121
:10B3B000FF90EF90DF9008951F920F920FB60F92BB
:10B3C00011240BB60F922F933F934F935F936F937C
:10B3D0007F938F939F93AF93BF93EF93FF9380E0FF
:10B3E0004ADEFF91EF91BF91AF919F918F917F9135
:10B3F0006F915F914F913F912F910F900BBE0F90E6
:10B400000FBE0F901F9018951F920F920FB60F92BC
:10B4100011240BB60F922F933F934F935F936F932B
:10B420007F938F939F93AF93BF93EF93FF9381E0AD
:10B4300022DEFF91EF91BF91AF919F918F917F910C
:10B440006F915F914F913F912F910F900BBE0F9095
:10B450000FBE0F901F9018951F920F920FB60F926C
:10B4600011240BB60F922F933F934F935F936F93DB
:10B470007F938F939F93AF93BF93EF93FF9382E05C
:10B48000FADDFF91EF91BF91AF919F918F917F91E5
:10B490006F915F914F913F912F910F900BBE0F9045
:10B4A0000FBE0F901F9018951F920F920FB60F921C
:10B4B00011240BB60F922F933F934F935F936F938B
:10B4C0007F938F939F93AF93BF93EF93FF9383E00B
:10B4D000D2DDFF91EF91BF91AF919F918F917F91BD
:10B4E0006F915F914F913F912F910F900BBE0F90F5
:10B4F0000FBE0F901F901895E0E0F6E080E4868381
:10B5000081838183868383EF91E00197F1F700C007
:10B51000000080E4858383EF91E00197F1F700C09C
:10B52000000080E48683828389E092E480D588E00D
:10B530008093094287E092E4A6D50E948B2C660F87
:10B54000771F660F771F609307427093084286E06B
:10B5500092E46DD51092064208950F931F93CF93F6
:10B56000DF93CDB7DEB7A597CDBFDEBF8C010E94BC
:10B57000A037811102C00E948C3761E0CE01019694
:10B580000E94A7378130F9F4CE0101960E947D1FF9
:10B5900089818130D1F4BE016F5F7F4FC8010E9465
:10B5A000D21C0E9488378A81813031F465E77DE1C1
:10B5B0000E944B1F81E00AC063E57DE181E00E94AB
:10B5C0004B1F81E003C080E001C080E0A596CDBFA5
:10B5D000DEBFDF91CF911F910F910895CF93DF933D
:10B5E000CDB7DEB72897CDBFDEBF6B017C016BE323
:10B5F0007DE181E00E944B1FCE0101960E94E12F68
:10B6000069817A818B819C8146015701860E971E44
:10B61000A81EB91EA70196010E94AC63861A970A5C
:10B62000A80AB90A8D829E82AF82B886BE016B5F7E
:10B630007F4FCE0101960E949D30882391F16CE2EC
:10B640007DE181E00E944B1FCE0101960E94002304
:10B650006FE17DE181E00E944B1FCE0105960E94C3
:10B6600000230E9461318FE097E20197F1F700C05B
:10B670000000E0E0F6E080E8858380E48183868353
:10B6800083EF91E00197F1F700C0000080E485832B
:10B6900083EF91E00197F1F700C0000080E486831A
:10B6A00005C066EE7CE181E00E944B1F0000FECFEA
:10B6B00081E090E0A0E0B0E08093024290930342EA
:10B6C000A0930442B09305420E94AD2C80930042A7
:10B6D000909301420E94982C8093FC419093FD41ED
:10B6E00044E050E062E072E483E399E00E945B246E
:10B6F00042E050E060E072E483E39AE00E945B2461
:10B7000042E050E06CEF71E483E39BE00C945B2437
:10B710000895CF93DF9300D01F92CDB7DEB7198283
:10B720001A821B821C8244E050E0BE016F5F7F4F93
:10B7300083E398E00E945B242496CDBFDEBFDF91B7
:10B74000CF910895CF93DF9300D01F92CDB7DEB78E
:10B7500044E050E0BE016F5F7F4F83E398E00E94BA
:10B76000332489819A81AB81BC810196A11DB11DD1
:10B7700089839A83AB83BC8344E050E0BE016F5F52
:10B780007F4F83E398E00E945B242496CDBFDEBF09
:10B79000DF91CF910895CF93DF9300D01F92CDB763
:10B7A000DEB744E050E0BE016F5F7F4F83E398E077
:10B7B0000E94332469817A818B819C812496CDBF3C
:10B7C000DEBFDF91CF910895CF93DF93CDB7DEB782
:10B7D0006097CDBFDEBF8091FA4190E0883091053F
:10B7E00008F093C3FC01E950FE4FF4C70E94842C7B
:10B7F000882351F16DE170E281E00E944B1F58DF18
:10B800000E948B2C6093F6417093F7418093F8412E
:10B810009093F9416D3271408105910560F08CE2A1
:10B8200091E0A0E0B0E08093F6419093F741A093BF
:10B83000F841B093F9416091F6417091F7418091E0
:10B84000F8419091F941CADE66E070E281E00E9421
:10B850004B1F81E08093FA4175DF0E94A32C8093F7
:10B86000F541813009F061C08091094281114DC3D9
:10B8700043D5813009F050C064EE7FE10E944B1F38
:10B8800017DF89DF6D30710581059105E8F48CE2E1
:10B8900091E0A0E0B0E08093F6419093F741A0934F
:10B8A000F841B093F94161ED7FE181E00E944B1FC7
:10B8B00072DFAB01BC0181E00E946D1F61EB7FE193
:10B8C00081E00E944B1F1FC00E948B2C6093F641A9
:10B8D0007093F7418093F8419093F94169E87FE1D3
:10B8E00081E00E944B1F4091F6415091F7416091D9
:10B8F000F8417091F94181E00E946D1F6EE77FE190
:10B9000081E00E944B1F6091F6417091F741809158
:10B91000F8419091F94162DE60E57FE181E00E94AB
:10B920004B1F82E08093FA41F0C263E27FE181E045
:10B930000E944B1F82E08093FA41E7C2F0D40E943C
:10B94000A12E81110E94EC320E94B82C90E08093CD
:10B95000FE419093FF411FDF6D3071058105910518
:10B96000A8F481E090E0A0E0B0E0809302429093E0
:10B970000342A0930442B093054280930042909307
:10B9800001428093FC419093FD4148C044E050E067
:10B9900062E072E483E399E00E94332442E050E0E5
:10B9A00060E072E483E39AE00E94332442E050E0D6
:10B9B0006CEF71E483E39BE00E94332481E090E02C
:10B9C000A0E0B0E08093024290930342A09304422F
:10B9D000B09305420E94AD2C20910042309101426B
:10B9E0008217930718F40E94AD2C02C0822F932F68
:10B9F00080930042909301420E94982C2091FC4138
:10BA00003091FD418217930718F40E94982C02C0D0
:10BA1000822F932F8093FC419093FD4183E080938C
:10BA2000FA4173C28091024290910342A091044274
:10BA3000B09105420197A105B10549F484E08093D6
:10BA4000FA4180E5809306421092FB415EC20E945B
:10BA5000834081115AC20E948940811156C20E94BE
:10BA60008640811152C20E943D4F882309F44DC285
:10BA70000E946E2E811149C20E94A037811145C2D9
:10BA80000E94682A811141C286DE2AE030E040E04F
:10BA900050E062D6672B682B692B11F40E942E2987
:10BAA0007ADE6D30710581059105F0F401DE8CE2DE
:10BAB00091E0A0E0B0E08093F6419093F741A0932D
:10BAC000F841B093F94160E17FE181E00E944B1FB2
:10BAD00062DEAB01BC0181E00E946D1F60EF7EE180
:10BAE00081E00E944B1F1FC00E948B2C6093F64187
:10BAF0007093F7418093F8419093F94168EC7EE1AF
:10BB000081E00E944B1F4091F6415091F7416091B6
:10BB1000F8417091F94181E00E946D1F6DEB7EE16B
:10BB200081E00E944B1F8091F6419091F741880F70
:10BB3000991F880F991F809307429093084287E0CE
:10BB40008093FA410E94F032882309F4DEC16BE849
:10BB50007EE181E00E944B1FD8C1CE010196FDDC41
:10BB6000882309F454C0CE0101960E94E8288091F0
:10BB7000004290910142019761F48091FE419091C1
:10BB8000FF410E94522A0E947C4085E08093FA4146
:10BB90000FC08091FC419091FD41019731F40E94CA
:10BBA0002F4F86E08093FA4103C083E08093FA41EF
:10BBB0008091024290910342A0910442B0910542CB
:10BBC0000097A105B10559F00197A109B10980932A
:10BBD000024290930342A0930442B09305428091A5
:10BBE000004290910142009729F001978093004212
:10BBF000909301428091FC419091FD41009709F49E
:10BC000084C101978093FC419093FD417EC1809156
:10BC1000F5418250843008F078C18091FB41811158
:10BC200074C10E941B3F813011F48093FB418091CD
:10BC3000064281116AC10E94883765E67EE181E093
:10BC40000E944B1F35DDA7DD6D3071058105910523
:10BC5000F0F42EDD8CE291E0A0E0B0E08093F641BC
:10BC60009093F741A093F841B093F94162E57EE1EA
:10BC700081E00E944B1F8FDDAB01BC0181E00E947F
:10BC80006D1F62E37EE181E00E944B1F51C08091F5
:10BC9000F541843091F0853019F0833041F51AC0B8
:10BCA00080E39AE2A0E0B0E08093F6419093F74100
:10BCB000A093F841B093F94126C080E19EE0A0E056
:10BCC000B0E08093F6419093F741A093F841B09390
:10BCD000F94119C088E097E0A0E0B0E08093F64118
:10BCE0009093F741A093F841B093F9410CC08CE2D6
:10BCF00091E0A0E0B0E08093F6419093F741A093EB
:10BD0000F841B093F9416AE07EE181E00E944B1F67
:10BD10004091F6415091F7416091F8417091F9419D
:10BD200081E00E946D1F6FEF7DE181E00E944B1F5B
:10BD30008091F6419091F741880F991F880F991FC4
:10BD4000809307429093084287E08093FA410E94D3
:10BD5000F032882309F4D9C06DEC7DE181E00E94C6
:10BD60004B1FD3C00E94652A8111CFC00E94894019
:10BD70008111CBC00E9486408111C7C00E943D4FF7
:10BD8000882309F4C2C00E94AD2C80930042909396
:10BD900001420E94982C8093FC419093FD410E94A7
:10BDA000804083E08093FA41B0C00E9489408111B5
:10BDB000ACC00E9486408111A8C00E943D4F8823DC
:10BDC00009F4A3C00E94982C8093FC419093FD41FC
:10BDD0000E94804083E08093FA4197C00E94F03235
:10BDE000811152C061EC7DE181E00E944B1F4091C6
:10BDF000024250910342609104427091054281E0F9
:10BE00000E946D1F6EEA7DE181E00E944B1F409110
:10BE100000425091014260E070E081E00E946D1F9D
:10BE20006CE97DE181E00E944B1F4091FC41509103
:10BE3000FD4160E070E081E00E946D1F69E97DE1F5
:10BE400081E00E944B1F44E050E062E072E483E333
:10BE500099E00E945B2442E050E060E072E483E3FA
:10BE60009AE00E945B2442E050E06CEF71E483E3CF
:10BE70009BE00E945B246091F6417091F7418091B4
:10BE8000F8419091F941AADB8091074290910842D4
:10BE9000892BD9F444E050E062E072E483E399E056
:10BEA0000E945B2442E050E060E072E483E39AE0A9
:10BEB0000E945B2442E050E06CEF71E483E39BE07E
:10BEC0000E945B2481E08093FA4180910742909127
:10BED000084283709927892BC1F48091F641909193
:10BEE000F741A091F841B091F94189379105A10539
:10BEF000B10558F00197A109B1098093F6419093DB
:10BF0000F741A093F841B093F9416096CDBFDEBFF1
:10BF1000DF91CF910895CF93DF93E2EEF2E22AE62C
:10BF200033E28FEF9FEFDC01EF0128971882108238
:10BF3000118212821382148285839683A783B0872D
:10BF40007196E217F30781F781E0DF91CF910895B1
:10BF500048E850E06AED72E283E492E00E94C55343
:10BF600081E008950F931F93CF93DF938B01883067
:10BF7000E8F491E1899FE0011124C652DD4DCE0124
:10BF800077D4F801808588874185528563857485DB
:10BF900049875A876B877C87458556856785708971
:10BFA0004D875E876F87788B81E001C080E0DF91ED
:10BFB000CF911F910F910895FC0180818F3F79F0FF
:10BFC00080858F3F71F081E041855285638574855E
:10BFD0004F3F5F4F6F4F7F4F29F480E0089580E01F
:10BFE000089580E008950F931F93CF93DF9348E85F
:10BFF00050E06AED72E283E492E00E94B853CAED29
:10C00000D2E202E613E2CE01D7DF882329F061965F
:10C01000C017D107C1F702C080E001C081E0DF9105
:10C02000CF911F910F91089580910A4208955091E8
:10C030000C425523A9F02091354230913642281701
:10C040003907D9F0E7E3F2E440E005C021913191EE
:10C0500028173907A1F04F5F4513F8CF543188F402
:10C06000E52FF0E0EE0FFF1FEB5CFD4B808391832B
:10C070005F5F50930C4281E0089581E0089581E074
:10C08000089580E0089550910B425523A9F0209126
:10C090000D4230910E4228173907D9F0EFE0F2E453
:10C0A00040E005C02191319128173907A1F04F5F79
:10C0B0004513F8CF543188F4E52FF0E0EE0FFF1F61
:10C0C000E35FFD4B808391835F5F50930B4281E080
:10C0D000089581E0089581E0089580E00895209119
:10C0E0000C42222371F0A5E3B2E480E0ED91FD91D2
:10C0F0009081992319F09081915090838F5F8217DE
:10C10000A8F330910B42332389F0ADE0B2E420E094
:10C11000ED91FD9180819181892B29F08081918120
:10C120000197808391832F5F231790F308951F92C7
:10C130000F920FB60F9211240BB60F922F933F93CD
:10C140004F935F936F937F938F939F93AF93BF931F
:10C15000EF93FF93C4DFFF91EF91BF91AF919F9158
:10C160008F917F916F915F914F913F912F910F90A0
:10C170000BBE0F900FBE0F901F901895E0E0F4E0FB
:10C180008FEF90E08287938781E080838283089598
:10C190008DE592E40E9486258091754290917642C9
:10C1A000A0917742B091784284369105A105B105FE
:10C1B00040F4E0E0F6E082E0828381E081838683E0
:10C1C00008C0E0E0F6E082E08183868381E081833D
:10C1D00086831092DD421092DE421092DF4210926E
:10C1E000E0421092E14280EE92E44DCF08958091BA
:10C1F000DF42882309F47FC08091DE42882319F052
:10C20000813081F172C08091E0429091E142892BAE
:10C2100099F484E090E08093E0429093E14281E0E1
:10C220008093DE42E0E0F6E092E09283858369EB62
:10C2300070E20C944B1F089581E0E0E0F6E0868305
:10C240008091754290917642A0917742B091784268
:10C2500084369105A105B10508F44DC082E08683BE
:10C26000818308958091754290917642A0917742A2
:10C27000B091784284369105A105B10540F4E0E023
:10C28000F6E080858695817091E0892705C0E0E021
:10C29000F6E0808586958170882381F01092DD42DA
:10C2A00088E290E08093E0429093E1421092DE4277
:10C2B00063E970E281E00C944B1F08958091E042A5
:10C2C0009091E142892BB9F481E08093DD4288E2CC
:10C2D00090E08093E0429093E1421092DE426FE65C
:10C2E00070E281E00C944B1F08951092DE42109290
:10C2F000E0421092E142089581E09091DD42913058
:10C3000009F080E008958091DF42811107C081E04B
:10C310008093DF4268E570E20C944B1F0895809192
:10C32000DF42882339F01092DF4260E470E281E05E
:10C330000C944B1F08955058BB27AA270ED04DC10F
:10C340003ED130F043D120F031F49F3F11F41EF480
:10C3500033C10EF4E095E7FB29C1E92F4FD180F3FB
:10C36000BA17620773078407950718F071F49EF5F2
:10C3700067C10EF4E0950B2EBA2FA02D0B01B90169
:10C3800090010C01CA01A0011124FF27591B99F04B
:10C39000593F50F4503E68F11A16F040A22F232F57
:10C3A000342F4427585FF3CF469537952795A795A7
:10C3B000F0405395C9F77EF41F16BA0B620B730B4E
:10C3C000840BBAF09150A1F0FF0FBB1F661F771FBF
:10C3D000881FC2F70EC0BA0F621F731F841F48F474
:10C3E000879577956795B795F7959E3F08F0B3CFFA
:10C3F0009395880F08F09927EE0F979587950895E4
:10C400000CD0EBC0E3D040F0DAD030F021F45F3F45
:10C4100019F0CCC0511115C1CFC0F0D098F39923B9
:10C42000C9F35523B1F3951B550BBB27AA276217F8
:10C430007307840738F09F5F5F4F220F331F441F3D
:10C44000AA1FA9F333D00E2E3AF0E0E830D0915075
:10C450005040E695001CCAF729D0FE2F27D0660F62
:10C46000771F881FBB1F261737074807AB07B0E8A1
:10C4700009F0BB0B802DBF01FF2793585F4F2AF0B7
:10C480009E3F510568F092C0DCC05F3FECF3983EE0
:10C49000DCF3869577956795B795F7959F5FC9F714
:10C4A000880F911D9695879597F90895E1E0660F9D
:10C4B000771F881FBB1F621773078407BA0720F016
:10C4C000621B730B840BBA0BEE1F88F7E09508957F
:10C4D00004D06894B111B5C0089598D088F09F57E2
:10C4E00090F0B92F9927B751A0F0D1F0660F771FC0
:10C4F000881F991F1AF0BA95C9F712C0B13081F0A0
:10C500009FD0B1E008959CC0672F782F8827B85F2F
:10C5100039F0B93FCCF3869577956795B395D9F700
:10C520003EF490958095709561957F4F8F4F9F4F0A
:10C530000895E89409C097FB3EF490958095709516
:10C5400061957F4F8F4F9F4F9923A9F0F92F96E95F
:10C55000BB279395F695879577956795B795F111D4
:10C56000F8CFFAF4BB0F11F460FF1BC06F5F7F4F71
:10C570008F4F9F4F16C0882311F096E911C0772383
:10C5800021F09EE8872F762F05C0662371F096E88C
:10C59000862F70E060E02AF09A95660F771F881F5B
:10C5A000DAF7880F9695879597F9089597F99F6719
:10C5B00080E870E060E008959FEF80EC089500242B
:10C5C0000A941616170618060906089500240A94F8
:10C5D00012161306140605060895092E0394000C7E
:10C5E00011F4882352F0BB0F40F4BF2B11F460FF0D
:10C5F00004C06F5F7F4F8F4F9F4F089557FD905836
:10C60000440F551F59F05F3F71F04795880F97FB16
:10C61000991F61F09F3F79F08795089512161306D0
:10C620001406551FF2CF4695F1DF08C016161706FF
:10C630001806991FF1CF8695710561050894089534
:10C64000E894BB2766277727CB0197F908950BD08D
:10C65000C4CFB5DF28F0BADF18F0952309F0A6CFD4
:10C66000ABCF1124EECFCADFA0F3959FD1F3950F86
:10C6700050E0551F629FF001729FBB27F00DB11D66
:10C68000639FAA27F00DB11DAA1F649F6627B00DF6
:10C69000A11D661F829F2227B00DA11D621F739FDF
:10C6A000B00DA11D621F839FA00D611D221F749FED
:10C6B0003327A00D611D231F849F600D211D822F34
:10C6C000762F6A2F11249F5750408AF0E1F088237B
:10C6D0004AF0EE0FFF1FBB1F661F771F881F915088
:10C6E0005040A9F79E3F510570F060CFAACF5F3F41
:10C6F000ECF3983EDCF3869577956795B795F795BB
:10C70000E7959F5FC1F7FE2B880F911D9695879542
:10C7100097F90895DB018F939F9371D0BF91AF91EB
:10C72000A29F800D911DA39F900DB29F900D11248B
:10C73000089597FB072E16F4009406D077FD08D0D5
:10C7400068D007FC05D03EF4909581959F4F0895E1
:10C75000709561957F4F0895A1E21A2EAA1BBB1B0D
:10C76000FD010DC0AA1FBB1FEE1FFF1FA217B307BD
:10C77000E407F50720F0A21BB30BE40BF50B661FD3
:10C78000771F881F991F1A9469F760957095809597
:10C7900090959B01AC01BD01CF010895052E97FB3B
:10C7A00016F400940FD057FD05D0D6DF07FC02D059
:10C7B00046F408C050954095309521953F4F4F4F16
:10C7C0005F4F089590958095709561957F4F8F4F3D
:10C7D0009F4F0895EE0FFF1F0590F491E02D1994DF
:10C7E000A29FB001B39FC001A39F700D811D1124B2
:10C7F000911DB29F700D811D1124911D0895F0DFD0
:10C80000A59F900DB49F900DA49F800D911D1124A4
:10C810000895AA1BBB1B51E107C0AA1FBB1FA61787
:10C82000B70710F0A61BB70B881F991F5A95A9F7D9
:10C8300080959095BC01CD010895FB01DC0102C0FB
:10C8400005900D9241505040D8F70895FC01059095
:10C850000020E9F7809590958E0F9F1F0895FB01AA
:10C86000DC0102C001900D9241505040D8F708956C
:10C87000FB01DC0101900D920020E1F708950F9378
:10C880001F93CF93DF93CDB7DEB72E97CDBFDEBF1B
:10C890000E891F8986E08C8309831A838FEF9FE7B7
:10C8A0008D839E83AE01465E5F4F688D798DCE018C
:10C8B00001960DD0EF81F885E00FF11F10822E96C2
:10C8C000CDBFDEBFDF91CF911F910F9108952F92C1
:10C8D0003F924F925F926F927F928F929F92AF9210
:10C8E000BF92CF92DF92EF92FF920F931F93CF935D
:10C8F000DF93CDB7DEB72C97CDBFDEBF7C016B01D8
:10C900008A01FC0116821782838181FFB0C1CE01AA
:10C9100001964C01F7019381F60193FD859193FFF8
:10C9200081916F01882309F49EC1853239F493FD0A
:10C93000859193FF81916F01853221F4B70190E0D9
:10C94000C4D1E8CF512C312C20E02032A0F48B321E
:10C9500069F030F4803259F0833269F420612CC0E0
:10C960008D3239F0803339F4216026C02260246092
:10C9700023C0286021C027FD27C030ED380F3A3092
:10C9800078F426FF06C0FAE05F9E300D1124532E86
:10C9900013C08AE0389E300D1124332E20620CC063
:10C9A0008E3221F426FD5FC1206406C08C3611F45E
:10C9B000206802C0883641F4F60193FD859193FF0B
:10C9C00081916F018111C1CF982F9F7D9554933034
:10C9D00028F40C5F1F4FFFE3F9830DC0833631F05D
:10C9E000833771F0833509F057C021C0F801808189
:10C9F00089830E5F1F4F44244394512C540114C06B
:10CA00003801F2E06F0E711CF801A080B18026FFA2
:10CA100003C0652D70E002C06FEF7FEFC5012C876A
:10CA200049D12C0183012C852F77222E16C0380185
:10CA3000F2E06F0E711CF801A080B18026FF03C0E8
:10CA4000652D70E002C06FEF7FEFC5012C8727D105
:10CA50002C012C852068222E830123FC19C0832DF4
:10CA600090E048165906A0F4B70180E290E02DD17D
:10CA70003A94F5CFF50127FC859127FE81915F015E
:10CA8000B70190E022D131103A94F1E04F1A5108E9
:10CA90004114510479F7DEC0843611F0893631F53E
:10CAA000F80127FF07C060817181828193810C5F4B
:10CAB0001F4F08C060817181882777FD8095982F6E
:10CAC0000E5F1F4F2F76B22E97FF09C0909580956D
:10CAD000709561957F4F8F4F9F4F2068B22E2AE04F
:10CAE00030E0A40124D1A82EA81843C0853729F42A
:10CAF0002F7EB22E2AE030E025C0F22FF97FBF2E24
:10CB00008F36C1F018F4883579F0ADC0803719F050
:10CB1000883721F0A8C02F2F2061B22EB4FE0DC09F
:10CB20008B2D8460B82E09C024FF0AC09F2F966009
:10CB3000B92E06C028E030E005C020E130E002C098
:10CB400020E132E0F801B7FE07C060817181828187
:10CB500093810C5F1F4F06C06081718180E090E07F
:10CB60000E5F1F4FA401E3D0A82EA818FB2DFF775E
:10CB7000BF2EB6FE0BC02B2D2E7FA51450F4B4FE95
:10CB80000AC0B2FC08C02B2D2E7E05C07A2C2B2D9E
:10CB900003C07A2C01C0752C24FF0DC0FE01EA0DE4
:10CBA000F11D8081803311F4297E09C022FF06C067
:10CBB0007394739404C0822F867809F0739423FDD4
:10CBC00012C020FF06C05A2C731418F4530C5718C7
:10CBD000732C731460F4B70180E290E02C8775D059
:10CBE00073942C85F6CF731410F4371801C0312CD0
:10CBF00024FF11C0B70180E390E02C8766D02C851C
:10CC000022FF16C021FF03C088E590E002C088E73C
:10CC100090E0B7010CC0822F867851F021FD02C050
:10CC200080E201C08BE227FD8DE2B70190E04DD09C
:10CC3000A51430F4B70180E390E047D05A94F8CFC0
:10CC4000AA94F401EA0DF11D8081B70190E03DD076
:10CC5000A110F6CF332009F45DCEB70180E290E059
:10CC600034D03A94F7CFF7018681978102C08FEFD5
:10CC70009FEF2C96CDBFDEBFDF91CF911F910F911B
:10CC8000FF90EF90DF90CF90BF90AF909F908F90EC
:10CC90007F906F905F904F903F902F900895FC0190
:10CCA0000590615070400110D8F7809590958E0FD7
:10CCB0009F1F0895FC016150704001900110D8F74A
:10CCC000809590958E0F9F1F08950F931F93CF937C
:10CCD000DF93182F092FEB018B8181FD03C08FEFAC
:10CCE0009FEF20C082FF10C04E815F812C813D816B
:10CCF000421753077CF4E881F9819F012F5F3F4F72
:10CD000028833983108306C0E885F985812F19951A
:10CD1000892B29F72E813F812F5F3F4F2E833F8341
:10CD2000812F902FDF91CF911F910F910895FA01DC
:10CD3000AA27283051F1203181F1E8946F936E7F5A
:10CD40006E5F7F4F8F4F9F4FAF4FB1E03ED0B4E04B
:10CD50003CD0670F781F891F9A1FA11D680F791F8C
:10CD60008A1F911DA11D6A0F711D811D911DA11D9D
:10CD700020D009F468943F912AE0269F11243019AD
:10CD8000305D3193DEF6CF010895462F4770405D48
:10CD90004193B3E00FD0C9F7F6CF462F4F70405DF7
:10CDA0004A3318F0495D31FD4052419302D0A9F752
:10CDB000EACFB4E0A6959795879577956795BA954C
:10CDC000C9F700976105710508959B01AC010A2E12
:10CDD00006945795479537952795BA95C9F7620FE9
:0ECDE000731F841F951FA01D0895F894FFCFA8
:10CDEE00000000002C010000010001000100000005
:10CDFE0000000000002C01000001000100010000F5
:10CE0E000000000000002C010000010001000100E4
:10CE1E00000000000000002C0100000100010001D4
:10CE2E0000000000000000002C01000001000100C5
:10CE3E000100000000000000002C010000010001B4
:10CE4E00000100000000000000002C0100000100A5
:10CE5E0001000100000000000000002C0100000194
:10CE6E000001000100000000000000002C01000085
:10CE7E00010001000100000000000000002C010074
:10CE8E00000100010001000000005D00205B0003B6
:10CE9E0000020252260000780300010002960E05E1
:10CEAE000000000000000000000000029B0E0500C4
:10CEBE000000000000000000000002A00E050000AF
:10CECE0000000000000000000002A50E050000009A
:10CEDE00000000000000000002AA0E050000000085
:10CEEE000000000000000002AF0E05000000000070
:10CEFE0000000000000002B40E050000000000005B
:10CF0E00000000000002B90E050000000000000045
:10CF1E000000000002BE0E05000000000000000030
:10CF2E0000000001C30E0800000000000000000019
:10CF3E00000001CC0E060000000000000000000002
:10CF4E000001D30E060000000000000000000000EB
:10CF5E0001DA0E06000000000000000000000001D3
:10CF6E00E10E060000000000000000000001008F2E
:10CF7E001B0600000100961B06000001009D1B070A
:10CF8E0000000100A51B0600000100AC1B070000FD
:10CF9E000000B41B0500000000BA1B0200000000D8
:10CFAE00BD1B1100000000CF1B0500000000D51BAB
:10CFBE000400000100DA1B0700000100E21B07005D
:10CFCE00000100EA1B090000000000F41B05000030
:10CFDE00000000FA1B090000000000041C080000FD
:10CFEE000000000D1C080000000000161C050000CB
:10CFFE000000001C1C0B0000000000281C09000093
:10D00E00000000321C0800000000003B1C0900005C
:10D01E00000000451C0800000000004E1C0400002B
:10D02E00000000531C0600000000005A1C080000FF
:10D03E00000000631C040000000000681C070000D4
:10D04E00000000701C070000000000781C070000A4
:10D05E00000000801C040000000000851C0400007D
:10D06E000000008A1C0400000000008F1C05000058
:10D07E00000000951C110000000000A71C1100000C
:10D08E00000000B91C040000000000BE1C040000DB
:10D09E00000000C31C050000000000C91C010000B8
:10D0AE00000000CB1C080000000000DD1C08000082
:10D0BE00000000D41C08000000000000000000006A
:10D0CE0000000000000000FFFFFFFF000000000056
:10D0DE000000000000000000FFFFFFFF0000000046
:10D0EE00000000000000000000FFFFFFFF00000036
:10D0FE0000000000000000000000FFFFFFFF000026
:10D10E000000000000000000000000FFFFFFFF0015
:10D11E00000000000000000000000000FFFFFFFF05
:10D12E0000000000000000000000000000FFFFFFF4
:10D13E00FF00000000000000000000000000FFFFE4
:10D14E00FFFF0A080808020000000101D0070000D6
:10D15E008045400200000110000000454002100012
:10D16E000110000080454002000100002F00200049
:10D17E003A004D4D492D353133004D4D492D363147
:10D18E0033004D4D492D30313100556E6B6E6F773A
:10D19E006E0050494425303464001F1C1F1E1F1E94
:10D1AE001F1F1E1F1E1F54656C697420534538388F
:10D1BE003020475053204D6F64756C6500535049B5
:10D1CE00204572726F723A2054696D656F757420C6
:10D1DE006F6E2052656164204275666665720D0A37
:10D1EE0000312073656320486561727462656174F5
:10D1FE000D0A00040000010201010000A008400613
:10D20E000203A00960060203A00A80060203A00B17
:04D21E00A006020361
:00000001FF
